:020000040800F2
:100000000000022085F90008E99C0008EB9C00082C
:10001000ED9C0008EF9C0008F19C00080000000027
:10002000000000000000000000000000F39C000839
:10003000F59C000800000000F79C0008F99C0008EF
:10004000C9F90008C9F90008C9F90008C9F9000888
:10005000C9F90008C9F90008C9F90008C9F9000878
:10006000C9F90008C9F90008C9F900084563000882
:10007000C9F90008C9F90008C9F90008C9F9000858
:10008000C9F90008C9F90008C9F90008C9F9000848
:10009000C9F90008C9F90008C9F90008859F0008D6
:1000A000C9F90008C9F90008C9F90008C9F9000828
:1000B000F59E0008C9F90008C9F90008C9F9000847
:1000C000C9F90008C9F90008C9F90008C9F9000808
:1000D000C9F90008C9F9000899A00008C9F9000881
:1000E000C9F90008C9F90008FD9C0008C9F9000811
:1000F000C9F90008C9F90008C9F90008C9F90008D8
:10010000C9F90008C9F90008C9F90008C9F90008C7
:10011000C9F90008C9F90008C9F90008C9F90008B7
:10012000C9F90008C9F90008C9F90008C9F90008A7
:10013000C9F90008C9F90008C9F90008C9F9000897
:10014000C9F90008C9F90008C9F900082D9D00087F
:10015000C9F90008C9F90008C9F90008C9F9000877
:10016000C9F90008C9F90008C9F90008C9F9000867
:10017000C9F90008C9F90008C9F90008C9F9000857
:08018000C9F90008C9F90008E3
:10018800E4A5050800000020FC0C0020000D00205C
:10019800EC510020064B07481A68074B1A60074BBA
:1001A80000221A70064B01221A7001F0F0B900BF44
:1001B800A83E00207C0F0020AC440020903E002088
:1001C800483E002008B5034801F0E1F9024B00223F
:1001D8001A7008BD54130020483E002008B5054B8E
:1001E800012200201A7004F0D5FB0348BDE808403E
:1001F80001F0CDB9C0440020F81300202DE9F041EA
:10020800144C204602F00BFF00201349134A02F059
:10021800BDFC1349134A0746002002F0B7FC1249F7
:10022800124A0646002002F0B1FCD22105463A46A1
:1002380023460A2002F0C2FDD22132462346FA2084
:1002480002F0BCFD5A20D2212A462346BDE8F041DF
:1002580002F0B4BD0C1200209A940508CD010008E4
:10026800A3940508E5010008AB9405089D01000862
:1002780008B5054B012200201A7004F08BFB0348D7
:10028800BDE8084001F083B9C0440020F8130020FD
:10029800044B054800221A70044B02221A7001F020
:1002A80076B900BF903E00200C120020483E002086
:1002B80008B5034801F06BF9024B00221A7008BD1B
:1002C80054130020483E00202DE9F041144C2046EC
:1002D80002F0A5FE00201349134A02F057FC134907
:1002E800134A0746002002F051FC1249124A0646FA
:1002F800002002F04BFCD22105463A4623460A204C
:1003080002F05CFDD221324623465A2002F056FD07
:10031800AA20D2212A462346BDE8F04102F04EBD6C
:100328007C0F00209A940508B9020008B4940508C7
:1003380099020008BD94050879020008002008B554
:1003480004F028FB064B00221A70064B1B78022B80
:100358000CBF05480548BDE8084001F018B900BFC2
:10036800C0440020483E00200C1200207C0F0020D2
:1003780010B5084C204602F052FE00200649074AF4
:1003880002F004FCD22102462346E620BDE81040D4
:1003980002F014BD40150020C69405084503000866
:1003A80010B5074C4FF6E071206801F043FF206854
:1003B800044901F0EDFEBDE8104003F069B800BF44
:1003C800000D0020CF94050810B5074C4FF6E071DA
:1003D800206801F02FFF2068044901F0D9FEBDE82C
:1003E800104003F055B800BF000D0020E494050844
:1003F80010B5074C4FF6E071206801F01BFF20682C
:10040800044901F0C5FEBDE8104003F041B800BF43
:10041800000D0020F994050810B5074C4FF6E0715F
:10042800206801F007FF2068044901F0B1FEBDE82B
:10043800104003F02DB800BF000D00200E950508F0
:1004480010B51E4CFFF7E8FF002004F0A3FA23794B
:100458000BB9FFF7CDFF63790BB9FFF7A1FFA379BC
:100468000BB9FFF7B1FF154B5A79E2B11A79D2B13E
:10047800997900221A715A7101B19A71104B0F4C77
:100488001A7008F03FFC20684FF6E07101F0D2FEC8
:1004980020680C4901F07CFE07F09DFD02F0F8FF92
:1004A800094803F039F8FFF7B7FF002007F054FDBB
:1004B8000648BDE8104001F06AB800BF000D0020F2
:1004C800483E002023950508809698005413002084
:1004D80008B5002007F040FD0248BDE8084001F0DB
:1004E80056B800BF5413002010B586B04FF07E53A5
:1004F80002930023039308F000FB8DED000ACDED75
:10050800010A9DE8030006AB03E903009DED020A1A
:10051800DDED030A9DED041ADDED051A08F09FFADA
:10052800104C002084ED040AC4ED050A07F024FDF0
:1005380020644FF6E07004F001FAB7206E215E22C5
:10054800002304F00BFB084B1A68084B1A60084B91
:1005580002224FF0804001211A7006B0BDE8104019
:100568000DF043BC20480020983E0020AC440020F9
:10057800150E00201FB508F0C0FA8DED000ACDED6C
:10058800010A9DE80300104A02AB83E8030082E8F1
:1005980003004FF6E07004F0D1F9FFF715FFB7201C
:1005A8003C215E22002304F0D9FA084B1A68084B54
:1005B8001A60084B01214FF08040197005B05DF8B2
:1005C80004EB0DF012BC00BF20480020983E00202C
:1005D800AC440020150E002010B5224B2248234CB5
:1005E80086B002930023039302F096FF08F085FA81
:1005F8002046012184ED080AC4ED090A08F09DFA95
:100608008DED000ACDED010A9DE8030006AB03E974
:1006180003009DED020ADDED030A9DED041ADDEDF0
:10062800051A08F01CFA4FF6E07084ED0C0AC4EDC8
:100638000D0A04F083F9FFF7DBFEB720A0215E2244
:10064800002304F08BFA0A4B1A680A4B1A600A4B0B
:1006580003224FF0804001211A7006B0BDE8104017
:100668000DF0C3BB00004842A086010020480020CE
:10067800983E0020AC440020150E00202DE9F04FD4
:10068800434D444E85B000244FF6FF78284602F0CB
:10069800C6FC4146224623463F480094019401F097
:1006A8008DFD0427B060224623464FF6E0713B4893
:1006B8000097019401F082FD2346306041462246AE
:1006C80037480097019401F079FD3649F060364AC1
:1006D800204602F05BFA3549354A0746204602F0C3
:1006E80055FA3449344A8046204602F04FFA3349D5
:1006F800334A8146204602F049FA3249324A824654
:10070800204602F043FA3149314A84462046CDF862
:100718000CC002F03BFA21468346B2682B462046BD
:1007280002F04CFB214632682B467D2002F046FB46
:100738002321F2682B46B42002F040FB9B213A4665
:100748002B46FA2002F03AFB372142462B46FA2084
:1007580002F034FB69214A462B46FA2002F02EFBB0
:10076800C82152462B466E2002F028FBC8215A4663
:100778002B46AA2002F022FBDDF80CC0F0206246CE
:10078800C8212B4605B0BDE8F04F02F017BB00BFEB
:10079800B0120020000D0020379505083F95050888
:1007A800529505085A950508E1050008629505085F
:1007B8007D0500086A950508F1040008729505088A
:1007C800750B000879950508D90400088095050877
:1007D800490400081FB5134802F09EFE08F08DF981
:1007E8008DED000ACDED010A9DE803000E4A02AB2B
:1007F80083E8030082E803004FF6E07004F09EF8F7
:10080800FFF7E2FD5E220023DF203C2104F0A6F979
:10081800064B01221A71064B1A68064B1A6005B07E
:1008280000BD00BFA086010028480020000D002060
:10083800A83E0020AC44002010B586B04FF07E538F
:1008480002930023039308F058F98DED000ACDEDCB
:10085800010A9DE8030006AB03E903009DED020AC7
:10086800DDED030A9DED041ADDED051A08F0F7F831
:100878000E4C002084ED060AC4ED070A07F088FB39
:1008880060644FF6E07004F059F8DF206E215E22B4
:10089800002304F063F9064B01229A71FFF780FDEB
:1008A800044B1A68044B1A6006B010BD204800209B
:1008B800000D0020A83E0020AC44002070B52DEDAE
:1008C800028B9FED248A88B00A26F0EE488A03E05E
:1008D800B0EE608AF0EE418A08F00FF98DED000A5B
:1008E800CDED010A9DE8030004AB83E80300F0EEB8
:1008F800680AB0EE480A9DED041ADDED051A8DED83
:10090800028ACDED038A08F08FF8CDED010A8DED4E
:10091800000A9DE8030002AD85E80300013E6C462D
:10092800DDED020A9DED031AD2D19FED0B0A08F006
:10093800DBF88DED000ACDED010A9DE8030085E89E
:100948000300DDED030A9DED020A08B0BDEC028B41
:1009580070BD00BF00000000CDCCCC3D2DE9F74FA5
:10096800564D574CDFF86491DFF864814FF6E0701C
:1009780003F0E4FF28680EF089F9064668680F4618
:100988000EF084F93246CDE900013B46494620463F
:1009980012F088FE224600230520372104F0FCF8D7
:1009A8002869484F484E0EF071F9824668698B46AF
:1009B8000EF06CF95246CDE900015B4639462046F7
:1009C80012F070FE224600230520692104F0E4F8A5
:1009D800286B0EF05BF98246686B8B460EF056F971
:1009E8005246CDE900015B464146204612F05AFEC8
:1009F800002305209B21224604F0CEF831462A6CBC
:100A0800204612F04FFE224600239B21A22004F02C
:100A1800C3F84FF4FC6003F091FFA8680EF036F9B4
:100A28008246E8688B460EF031F95246CDE900015E
:100A38005B464946204612F035FE224605205021E5
:100A4800002304F0A9F8A8690EF020F98246E869A5
:100A58008B460EF01BF95246CDE900015B4639463C
:100A6800204612F01FFE224600230520822104F0B2
:100A780093F8A86B0EF00AF98246E86B8B460EF0E5
:100A880005F95246CDE900015B464146204612F081
:100A980009FE00230520B421224604F07DF83146E2
:100AA8006A6C204612F0FEFDA220B42122460023E3
:100AB80003B0BDE8F04F04F06FB800BF2048002035
:100AC800100D002099950508BC950508879505081F
:100AD800AB95050810B51F4B1F48204C86B00293F4
:100AE8000023039302F018FD08F007F820460221BE
:100AF80084ED0A0AC4ED0B0A08F01FF88DED000A10
:100B0800CDED010A9DE8030006AB03E903009DED66
:100B1800020ADDED030A9DED041ADDED051A07F062
:100B28009EFF4FF6E07084ED0E0AC4ED0F0A03F045
:100B380005FFDF20A0215E22002304F00FF8084BF8
:100B480001225A71FFF70AFF064B1A68064B1A6012
:100B580006B010BD00004842A086010020480020D1
:100B6800000D0020A83E0020AC440020F6E600BF9F
:100B7800284B2948062210B51A704FF6E07400F089
:100B880006FD0020214607F099FB3120214607F099
:100B980095FB6320214607F091FB9520214607F03D
:100BA8008DFBC7204FF4FC6107F088FB4EF29C7068
:100BB80003F0C4FE052001210023184A03F0ECFFCE
:100BC800052020210023164A03F0E6FF05205221C4
:100BD8000023144A03F0E0FF842100230520124A71
:100BE80003F0DAFF4FF4F06003F0A8FEB6210F4AD5
:100BF8000023052003F0D0FF4FF6FF7003F09EFEA0
:100C08008720DC210A4A002303F0C6FFBDE8104014
:100C180007F0DABEC044002088160020C1950508F8
:100C2800F6950508EE9505085D9E0508CC9B050818
:100C3800C595050838B5384B3848394D07221A701C
:100C48004FF6E07400F0A3FC0020214607F036FBC5
:100C58003120214607F032FB6320214607F02EFBA6
:100C68009520214607F02AFB2146C72007F026FBDE
:100C78004EF29C7003F062FE052001210023294AF0
:100C880003F08AFF052020210023274A03F084FF70
:100C9800052052210023254A03F07EFF05208421E8
:100CA8000023234A03F078FF2A460520B6210023B3
:100CB80003F072FF40F213144FF4F06003F03EFEAD
:100CC8002046012100231B4A03F066FF204620210D
:100CD8000023194A03F060FF204652212A460023C8
:100CE80003F05AFF204684210023144A03F054FFDE
:100CF800B62100232046124A03F04EFF4FF6FF703C
:100D080003F01CFE7D20DC210E4A002303F044FF83
:100D1800BDE8384007F058BEC044002088160020BF
:100D2800B59A0508CA950508CE950508D29505080F
:100D3800D5950508DE950508DA950508D9950508BD
:100D4800DD950508E295050838B52B4B2B48052499
:100D58001C704FF6E07500F01AFC0020294607F0D9
:100D6800ADFA2720294607F0A9FA4F20294607F0AF
:100D7800A5FA7720294607F0A1FA9F20294607F00F
:100D88009DFA2946C72007F099FA4EF29C7003F0A5
:100D9800D5FD204601210023194A03F0FDFE204617
:100DA80016210023174A03F0F7FE20463E210023B0
:100DB800154A03F0F1FE204666210023134A03F08A
:100DC800EBFE20468E210023114A03F0E5FE204663
:100DD800B621104A002303F0DFFE4FF6FF7003F040
:100DE800ADFD7D20DC210C4A002303F0D5FEBDE8D3
:100DF800384007F0E9BD00BFC04400208816002035
:100E0800B59A0508ED950508F1950508F5950508C5
:100E1800F9950508FD95050801960508394B3A48E6
:100E2800042270B51A704FF6E07400F0B0FB002091
:100E3800214607F043FA3120214607F03FFA6320A4
:100E4800214607F03BFA9520214607F037FA2F4E46
:100E58002F4D2146C72007F031FA4EF29C7003F05F
:100E68006DFD052001213246002303F095FE052083
:100E780020210023274A03F08FFE0520522100235A
:100E8800254A03F089FE052084210023234A03F024
:100E980083FE2A460520B621002303F07DFE40F29A
:100EA80013144FF4F06003F049FD20460121324647
:100EB800002303F071FE204620210023184A03F086
:100EC8006BFE204652212A46002303F065FE204689
:100ED80084210023134A03F05FFEB6210023204635
:100EE800114A03F059FE4FF6FF7003F027FD7D20ED
:100EF800DC210E4A002303F04FFEBDE8704007F0E6
:100F080063BD00BFC0440020881600202296050853
:100F1800B59A05080D9605081D9605081296050848
:100F2800179605081C9605082196050825960508B4
:100F3800F8B5304B3048314F314E03221A704FF616
:100F4800E07400F024FB0020214607F0B7F9632085
:100F5800214607F0B3F9B3204FF4F06107F0AEF97A
:100F68002146C72007F0AAF94FF6FF7003F0E6FC08
:100F78004EF29C75DC2100237D20224A03F00CFEF2
:100F8800284603F0DBFC052001213A46002303F044
:100F980003FE0520522100231B4A03F0FDFDB62164
:100FA80032460023052003F0F7FD40F213144FF4F6
:100FB800F06003F0C3FC204601213A46002303F009
:100FC800EBFD204652213246002303F0E5FDB62111
:100FD800002320460D4A03F0DFFD284603F0AEFC4F
:100FE8000520A2210A4A002303F0D6FDBDE8F840F7
:100FF80007F0EABCC0440020881600203F96050888
:10100800B59A0508309605083A9605083E960508EB
:10101800FE95050808B5064B064802221A7000F02E
:10102800B6FA07F045F8BDE8084007F0CDBC00BFA8
:10103800C044002088160020002008B503F0AAFC50
:10104800064B00221A70064B1B78022B0CBF054872
:101058000548BDE8084000F09ABA00BFC044002027
:10106800483E00200C1200207C0F00202DE9F14F93
:101078002D4C204601F0D3FF00202C492C4A01F0CA
:1010880085FD2C492C4A8146002001F07FFD2B4923
:101098002B4A0746002001F079FD2A492A4A0646CC
:1010A800002001F073FD2949294A0546002001F076
:1010B8006DFD2849284A8046002001F067FD274930
:1010C800274A8246002001F061FDD22183464A4624
:1010D8002346E62001F072FE28203A4623460146C0
:1010E80001F06CFE462132462346282001F066FEB8
:1010F80064212A462346282001F060FE82214246C8
:101108002346282001F05AFE524623462820A021D3
:1011180001F054FE28205A46BE21234601B0BDE8FE
:10112800F04F01F04BBE00BFF8130020C69405082D
:1011380041100008439605081D1000083096050860
:10114800390F000825960508250E00084E96050853
:10115800510D0008599605083D0C0008C59505086D
:10116800790B00080F4A012310B513700E4A0024AA
:1011780014700E4A2046137006F0EEFE204603F067
:1011880009FC0B4B04221A7007F06AFB07F008FCF5
:10119800084B09481C70094B1C70BDE8104000F052
:1011A800F6B900BFC04400200B0E0020090E002035
:1011B800483E002024460020C4100020903E002015
:1011C8000F4A38B5012313700E4A002414700E4AD2
:1011D8002046137006F0C0FE204603F0DBFB0B4BE5
:1011E80002251D7007F03CFB07F0DAFB084B0948A5
:1011F8001D70094B1C70BDE8384000F0C8B900BF2D
:10120800140E00200B0E0020C0440020483E002091
:1012180024460020F8130020903E002008B5064B15
:101228000020187003F0B6FB044B054803221A701F
:10123800BDE8084000F0ABB90B0E0020483E002086
:10124800B0120020034B01224FF4FC601A7003F027
:1012580075BB00BF0B0E00200B4B10B500242046B9
:101268001C7003F097FB07F08DF806F0C7FB074BDF
:101278001C70074B01221A7007F07EF80548BDE87C
:10128800104000F084B900BF0B0E0020C0440020BD
:10129800483E00207C0F00200A4B10B50024204651
:1012A8001C7003F077FB07F06DF8074B1C70074BB9
:1012B80002221A7007F060F80548BDE8104000F0F7
:1012C80066B900BF0B0E0020C0440020483E002035
:1012D8000C1200200C4B10B500220C4C1A7007F0B1
:1012E80051F804F0E5FA06F07CFE07F045F82068AE
:1012F8004FF6E07100F09EFF2068054900F048FFB6
:10130800BDE8104002F0C4B80B0E00202C0D0020E0
:10131800639605080E4B002210B51A700088C8386D
:1013280080B2042805D90B480B4A0C4B912102F0D6
:10133800D7FA0B4CC0B204F045FB20684FF6E071B9
:1013480000F078FF20680749BDE8104000F020BF92
:101358000B0E00207796050874D5030897960508A4
:101368002C0D0020C89605082DE9F04F6448654DFE
:1013780089B0002401F053FE4FF6FF712246234640
:1013880061480094019400F019FF042607464FF6BF
:10139800E071224623465D480096019400F00EFF56
:1013A8004FF6E0718046224623465948009601943C
:1013B80000F004FF4FF6FF71814622462346554848
:1013C8000096019400F0FAFE234628604FF6FF715C
:1013D800224651480096019400F0F0FE4F4968609B
:1013E8004F4A204601F0D2FB4E494F4A82462046DA
:1013F80001F0CCFB4D494E4A8346204601F0C6FB1E
:101408004C4903904C4A204601F0C0FB4B490490DC
:101418004B4A204601F0BAFB4A4905904A4A204601
:1014280001F0B4FB49490690494A204601F0AEFB59
:101438003A4607902146324B204601F0BFFC214630
:1014480042462F4BC82001F0B9FC0A214A462C4BD2
:10145800C82001F0B3FC2A68294B5521782001F0F7
:10146800ADFC6A68264B7820692101F0A7FCC825E5
:1014780005262327E0B204F0D5F9364A0146284666
:1014880001F084FB94FBF6F106FB114179431E3110
:10149800024689B200201A4B0134013501F08EFC56
:1014A800042CADB2E6D1D22152460520144B01F0EE
:1014B80085FCD2215A464C20114B01F07FFCD221E9
:1014C800039A0F4B9C2001F079FCD221049A0C4B13
:1014D800EC2001F073FCB421059A094BEC2001F0D3
:1014E8006DFCB421069A064B9C2001F067FC079A14
:1014F800034B4C20B42109B0BDE8F04F01F05EBCAD
:10150800541300202C0D0020D8960508E2960508F3
:10151800EF960508FA9605080F9505080E97050831
:10152800DD12000816970508251200081F97050800
:10153800A1120008289705086112000831970508CC
:101548004D1200083A970508C91100084397050885
:101558006D1100081D13000808B500F051FBFEF7D7
:101568004DFE00F083F8FFF789F8FEF7ADFEFFF7B0
:101578007DFD00F0EFFCFFF7F7FEFEF7F9FE00F047
:10158800D3FB00F049FABDE8084000F011BB10B5E4
:10159800044628B90F48104A104B492102F0A0F917
:1015A8000F4B1868844213D010B1C36900219847C3
:1015B800002003F0EFF9002003F0D6F94FF6FF7092
:1015C80003F0BCF9E369204601219847044B1C60ED
:1015D80010BD00BF4C97050883D503086897050818
:1015E800340D00200048D2E75413002008B5124BF0
:1015F800124A1B780D2B8CBF002101211170142277
:101608005A430F4988588B184FF47A720D49504342
:10161800086059684A430C490A609A680B4B1A607B
:1016280006F058FC06F0A8FE094B0A4800221A707A
:10163800BDE80840FFF7ABBFAE3E0020380F0020E2
:1016480000000020B03E0020CC440020A44400202C
:10165800483E002054130020024B034800221A7011
:10166800FFF795BF483E0020541300202DE9F347AB
:101678003A4DDFF804913A4E00244FF6FF7728469A
:1016880001F0CDFC394622462346364800940194A1
:1016980000F094FD4FF0040882463946224623465E
:1016A8004846CDF80080019400F088FD3946306046
:1016B800224623464846CDF80080019400F07EFD7E
:1016C80039467060224623464846CDF8008001948A
:1016D80000F074FD2346B060394622464846CDF8EE
:1016E8000080019400F06AFD1F49F0601F4A2046FF
:1016F80001F04CFA1E491F4A0746204601F046FAF7
:101708002146804652462B46204601F057FB3C2195
:1017180032682B465A2001F051FB5A2072682B463A
:10172800014601F04BFB7821B2682B465A2001F0A4
:1017380045FB9621F2682B465A2001F03FFBD22147
:101748003A462B46EC2001F039FB9C20D221424638
:101758002B4602B0BDE8F04701F030BBC4100020B2
:10176800380D002078970508859705086116000848
:101778008E970508F51500080F95050870B5474EB2
:10178800474C327847492DED028B142592B005FB62
:1017980002420C320FA811F085FF33780D2B05FBA0
:1017A80003F504EB050332D8D3ED016A9B6807EE15
:1017B800103A6359B8EEE68A06EE903ADFED3A7AC7
:1017C800F8EEC78AB8EEE67A88EE278AC8EEA78AC6
:1017D800C7EE277A17EE900A0DF058FA02460B4624
:1017E8006846324911F05EFF18EE100A0DF04EFA05
:1017F80002460B4605A82E4911F054FF18EE900A30
:101808000DF044FA02460B460AA82A4929E093ED4E
:10181800017A9B6807EE903A635906EE903AF8EE23
:10182800E78AF8EEE67AB8EEC78A17EE900A0DF066
:101838002DFA02460B4668461F4911F033FF18EE91
:10184800100A0DF023FA02460B4605A81B4911F0B1
:1018580029FF18EE900A0DF019FA0B4618490246AE
:101868000AA8184C11F01EFF2068174900F090FCD8
:1018780020680FA900F08CFC6068694600F088FCBD
:10188800A06805A900F084FCE0680AA900F080FCC3
:1018980001F0FEFD12B0BDEC028B70BDAE3E002023
:1018A800000000209797050800007A44A2970508D1
:1018B800B3970508C4970508D5970508E69705085E
:1018C800F7970508380D0020189505084FF6FF70A2
:1018D80070474FF6FF70704713B5002944D04FF298
:1018E800DE7003F057F8002003F01EF90F2003F014
:1018F80025F81E4C1E4A412101230A2003F04CF909
:10190800042003F011F9236828209621042B21DCF8
:101918000123184A03F040F901A90DF106022068D5
:1019280003F0C2FB0F2003F009F8BDF80400BDF86E
:10193800061014382822002380B203F02FF8BDF8CF
:101948000610BDF80400143989B22822012303F0D7
:1019580025F809E0084A012303F01EF91E20A521F5
:10196800064A012303F018F91CBD00BF480D0020EA
:10197800089805081B980508379805084D98050824
:1019880037B51E4C2368042B05462BDC01A80DF146
:10199800060103F087FBBDF80630BDF8042018499E
:1019A80004200AF027FA2368002B04DA1548164A9F
:1019B800164B592105E0042B05DD1248124A144B39
:1019C8005A2101F08DFF04EB8302BDF804100133A6
:1019D8009180BDF806102360052BD18008D1201D09
:1019E80003F0E2FB00230B482360FFF7D0FD03E080
:1019F80028460121FFF770FF3EBD00BF480D0020BB
:101A080064980508A998050895D50308CB98050892
:101A1800E29805089C14002037B50B4C204601F0CD
:101A2800FEFA0A4B0A49009300250120094A0A4B8D
:101A3800019501F09CF9294602462346284603B041
:101A4800BDE8304001F0BAB968110020E11800087B
:101A5800D5180008DB180008891900084FF6FF7030
:101A680070474FF6FF7070471FB54FF6E07002F0F1
:101A780091FF002003F058F80F2002F05FFF0021CB
:101A8800294A2A4C01230A2003F086F8002002F094
:101A980055FF042003F048F80A201921244A01239D
:101AA80003F07AF82521234A01230A2003F074F869
:101AB8001F2002F043FF01230A2037211E4A03F0AA
:101AC8006BF8237873B301231E2096211B4A03F079
:101AD80063F862881A49684611F0E4FD01231E2064
:101AE800A2216A4603F058F8A2881649684611F000
:101AF800D9FDAE216A4601231E2003F04DF80F20C0
:101B080002F01CFF6088A188143880B228220023C4
:101B180002F044FFA1886088143989B22822012381
:101B280002F03CFF1FBD00BF10990508600D0020A2
:101B380022990508429905086299050885990508BA
:101B480097990508A499050801B18DE7704713B561
:101B58000DF1060101A803F059FA144B01221A707D
:101B68005988BDF80420891A0E311C2919460AD84B
:101B78009C88BDF80600201A0E301C2803D89968E6
:101B88000131996001E000238B60084B99680129B5
:101B980005DD00229A601A70FFF724FD05E05A80DF
:101BA800BDF806209A80FFF75FFF1CBD600D00207E
:101BB80037B50B4C204601F032FA0A4B0A4900931C
:101BC80000250120094A0A4B019501F0D0F8294661
:101BD80002462346284603B0BDE8304001F0EEB87F
:101BE8009C140020511B0008651A00086B1A000895
:101BF800571B00080148FFF7CABC00BF201000208F
:101C080010B50B4C204601F00AFA00200146224686
:101C180000F034FB00200749074A00F0B7FFD22143
:101C2800024623464FF48270BDE8104001F0C6B862
:101C380088160020B1990508FD1B000810B5064C50
:101C48004FF6FF71206800F0F5FA044B2068196818
:101C5800BDE8104000F09CBA6C0D0020EC0200209A
:101C680008B5FFF7EBFF0020014606F055F8BDE880
:101C7800084001F00DBC08B5002002F08BFE054BB2
:101C88001868054B196800F083FA0448BDE8084055
:101C9800FFF77DBC6C0D0020E802002054130020E3
:101CA8000088A0F5C87080B2092808B505D9084889
:101CB800084A094B902101F013FE084B1880084B85
:101CC800FF21197006F028F8BDE80840B6E700BF04
:101CD800B6990508A7D50308D99905082C17002037
:101CE8002E1700200088A0F5967080B2092808B544
:101CF80005D90848084A094B842101F0F1FD084B31
:101D08001880084B0121197006F006F8BDE8084054
:101D180094E700BFB6990508BCD50308D99905080A
:101D28002C1700202E170020F7B500243648374D11
:101D380001F075F9224623464FF6FF7134480094A6
:101D4800019400F03BFA04262246234607464FF644
:101D5800FF7130480096019400F030FA234628605D
:101D680022464FF6FF712B480096019400F026FAA0
:101D780029496860294A204600F008FF204628497A
:101D8800284A00F003FF214606463A4620461E4BE5
:101D980001F014F82A681C4B2046282101F00EF89F
:101DA8003246AA20D221184B01F008F80F254FF42B
:101DB800967440F2351620461B491C4A00F0E6FE90
:101DC80001340246782128460F4BA4B2233500F08F
:101DD800F5FFB442ADB2EED10F254FF4C87440F20E
:101DE800991620461249134A00F0D0FE01340246E3
:101DF8009B212846044BA4B2233500F0DFFFB442F0
:101E0800ADB2EED1FEBD00BFE41500206C0D002080
:101E18000A9A050820950508169A0508691C0008FD
:101E28001F9A05087F1C0008289A0508ED1C000861
:101E38002A9A0508A91C000808B5FFF7FFFE00202C
:101E4800014605F069FFBDE8084001F021BB00BF6D
:101E580008B506F00DFD164A00230220CA2102F03B
:101E68009BFE144B1A68144B1A60144B1B78023BE8
:101E7800052B1CD8DFE803F003070B13170FBDE889
:101E88000840FFF7C7B8BDE80840FFF751B8BDE8FC
:101E98000840FEF7C3BFBDE80840FEF7CBBEBDE86B
:101EA8000840FEF751BFBDE80840FEF761BE08BD17
:101EB8000E950508A83E0020AC440020C044002030
:101EC80008B5084B01221A70074B1A68074B002007
:101ED8001A6002F05FFD06F0C3FC0548BDE8084043
:101EE800FFF755BB140E0020A83E0020AC4400208C
:101EF800F813002038B50E4B0E4D00241C700E4B05
:101F08001C700E4B1C700E4B1A680E4B20461A6044
:101F180002F040FD0C4B1B78022B0CBF0B480C4801
:101F2800FFF735FB2C70BDE8384006F099BC00BFC0
:101F3800140E002024460020C0440020903E0020BB
:101F4800A83E0020AC440020483E00200C1200208F
:101F58007C0F00202DE9F041144C204601F05FF879
:101F680000201349134A00F011FE1349134A07468B
:101F7800002000F00BFE1249124A0646002000F02D
:101F880005FED22105463A462346E62000F016FF14
:101F98004B2132462346642000F010FF642069215B
:101FA8002A462346BDE8F04100F008BF2010002073
:101FB800C6940508FD1E00082C9A0508C91E0008CD
:101FC800389A0508591E000808B508B143682BB9A6
:101FD8000348044A044B9B2101F082FC586908BD60
:101FE800459A0508D0D50308679A050808B5FFF78C
:101FF800EBFF8068123080B208BD08B5FFF7E4FF38
:102008004068063080B208BD2DE9F84F044688467E
:10201800FFF7DAFF6689E589074606F1030905F146
:102028000F0AB8F1000F1FD01F2002F087FC2046CE
:10203800FFF7DCFF83462046FFF7DFFF294603460C
:102048005FFA8BF2F0B202F0ADFC042002F06CFDF6
:102058000B364FF6FF70033502F070FCB0B2A9B230
:102068003A68012302F098FD3D69204641464A46F8
:102078005346A847BDE8F88F13B504460DF106018D
:1020880001A802F0C3FF2046FFF79EFF6389BDF851
:102098000410BDF80620C91AE389D21A0339C368A7
:1020A8000F3A204698471CBDF7B5044614200D4644
:1020B80016461F4610F084FF089BC7600361064B55
:1020C8000649074A80E8700000930190054B0020FC
:1020D80000F04DFEFEBD00BF1120000803200008DF
:1020E800F51F000881200008704708B508B143684B
:1020F8002BB90448044A054BAD2101F0F1FB58699E
:1021080008BD00BF869A0508E8D50308679A050840
:10211800F8B505460E46FFF7E8FF836B04461BB18A
:1021280028463146984700E018466F8994F83C30B5
:10213800ED890EB9034310D0208E02F0FFFB608EAC
:1021480002F012FC94F8350002F0EEFC94F83430FA
:1021580038462946224602F01FFD002384F83C3009
:10216800F8BD08B5FFF7C1FF90F83500BDE8084095
:1021780002F0EFBC38B5FFF7B8FF044611F018FBC2
:10218800054694F8350002F0DFFC684380B238BD9C
:1021980038B50D46FFF7A9FF29462E22044611F04F
:1021A80037FB50B1204629462E2211F083FB00232D
:1021B80084F82E30012384F83C3038BD2DE9F743EC
:1021C800074640200E461546984610F0F9FE04468C
:1021D80028B91148114A124B4E2101F081FB114BCD
:1021E800114A12498DE818000020114B00F0BFFD7C
:1021F80039468146FFF7CCFF9DF82830268684F8BB
:1022080035300B9B6586A363002384F8348084F8FB
:102218003C304846BDE8FE83869A050800D6030888
:10222800A49A0508192100086B2100087D210008DF
:10223800F120000810B50C46FFF757FF012304866C
:1022480080F83C3010BD00BF4FF4A0707047C82024
:1022580070477047074B1B78022B07B508D1064B10
:102268001B78022B04D001A80DF1060102F0CEFE66
:102278000EBD00BF24460020C044002073B50A4BA1
:1022880006460D461446009300200849084A094BA3
:10229800019000F06CFD294602462346304602B004
:1022A800BDE8704000F08ABD5B220008512200089A
:1022B800572200085D22000813B502AB03E90600A7
:1022C800436843B1027C0124082A9C7004D11B692D
:1022D8002146984700E01C4620461CBD30B5002822
:1022E8002BD0058B002425E0036A1A7C012A05D12E
:1022F8005B681A888A421BD1187F30BD052A06D12F
:102308005B681A888A4213D193F82C0030BD032ADF
:1023180006D15B681A888A420AD193F8250030BD35
:10232800062A05D15B681A888A4201D1D87A30BD5D
:1023380001340430AC42D7D3002030BD08B18175D8
:1023480001207047F8B504460D46D0B1E175D0F8C4
:1023580098309847012D0DD12746002606E0F869E8
:1023680000F10802436906CA98470136238B0437EF
:102378009E42F4D3D4F89830204629469847012045
:10238800F8BDF8BDF8B50546084617460E4611F0E3
:102398000FFA013FB84234BF04463C463CB12846D8
:1023A8003146224611F086FA00232B55F8BD2C70D1
:1023B800F8BDF7B5044600200090019000296CD0C4
:1023C8000E8B68E000F1080351F823301D7C042DC2
:1023D80004D15D682D88954247D0013000F108038B
:1023E80051F823301D7C012D04D15D682D8895425C
:1023F8003BD0013000F1080351F823301D7C052D36
:1024080004D15D682D8895422FD0013000F1080372
:1024180051F823301D7C032D04D15D682D88954229
:1024280023D0013000F1080351F823301D7C022D20
:1024380004D15D682D88954217D0013000F108035A
:1024480051F823301D7C072D04D15D682D8A9542F3
:102458000BD0013000F1080351F823301D7C062D04
:1024680008D15D682D88954203D103F10801204603
:1024780015E0013000F1080351F823502B7C082B9C
:1024880009D16F683F88974204D105F108012046B9
:102498001A4605E00130B04294D320466946082226
:1024A80011F03EF82046FEBDF8B505460F46164623
:1024B800002830D04388032B2FD0202010F080FD37
:1024C800044600282BD040F80C5B39460C22FFF755
:1024D80059FF1820E66110F073FD0646B8B10223D3
:1024E8000374012363760F4B446063600E4BA36053
:1024F800002323766B8805EB830201339BB2012B03
:1025080050606B800CD16A685268137608E02046E8
:1025180010F05EFD04E0064602E0002600E00646F4
:102528003046F8BD4C550408EA51040837B54568EB
:1025380002AB03E906003DB3037C0124042B85F8B4
:10254800314022D1688E02F0F9F995F8300002F096
:10255800EBFA95F8343043B9BDF80200BDF806101F
:10256800AA1C234602F018FB0FE0012B03D10848F0
:1025780040F2395104E0022B07D1054840F241519D
:10258800044A054B01F0ACF92C4620463EBD00BF7D
:10259800B79A0508C0200408B59A0508F8B5044696
:1025A8000F46164610B3838A0A2B20D0202010F03D
:1025B80007FD0546E8B14460102200F108003946DD
:1025C800FFF7E0FE4FF6FF73A08A2B801F236B8076
:1025D80000232B76831D013080B20128EE6144F878
:1025E8002350A08207D1A3691876F8BDF8BD002052
:1025F800F8BD0120F8BD0120F8BD2DE9F0411D46C8
:102608004B1C984280460C4617460CDD95420ADC66
:10261800013208F101035B1A521BC8B2D2B29BB255
:10262800294602F0BDF9A8F10208BDF81800C4EB6C
:10263800080802F083F901261FFA88F808E0A919AA
:10264800601C80B289B24246002302F0A7F9013625
:102658007B1B9E42F3D3BDE8F081F8B5C7B21446A0
:1026680038461E460D4602F09FF9621E92B2384661
:10267800294602F099F9304602F060F9022606E090
:10268800A21B92B23846294602F08EF90136A642BC
:10269800F6D3F8BD70B5044600F11E003C220023B5
:1026A80080B20D4602F07AF91E3DA9B220463C22BE
:1026B8000123BDE8704002F071B970B504460138D5
:1026C8000322002380B20D4602F068F9013DA9B249
:1026D800204603220123BDE8704002F05FB9F7B538
:1026E800089D2E7BEF7A1C463604AB7A06EB07264C
:1026F800F618431A687B06EB00602D18002001903D
:10270800121B08462146009501F098FEFEBD30B523
:10271800456885B004AB03E906007DB101242C733C
:102728006D68BDF80800BDF80A109DF80C209DF8EA
:102738000E300095FFF7D3FF204600E0284605B08D
:1027480030BD2DE9F04385B004AB03E906004468C9
:10275800BDF80860BDF80C70002C41D0012384F846
:10276800263094F825300BB9A26800E06268FFB201
:10277800BDF80A109DF80E30009230463A46FFF731
:10278800AEFF04F10C08022002F0CEF9404611F029
:102798000FF8054600B1451E0F3F0024153E1FFAED
:1027A80087F90DE002F0CAF902F0CEF904FB1061D6
:1027B80089B248462022002302F008FA0134E4B224
:1027C800AC42EFD3002002F0B9F8B8B2B1B2424639
:1027D800012302F0FBF9002002F0A6F9012000E035
:1027E800204605B0BDE8F0832DE9F04385B004AB81
:1027F80003E906004568BDF80860BDF80C70002DB7
:102808003CD001236B762B7EBDF80A10012B0CBF40
:102818006A68AA689DF80E300092FFB23A463046C0
:10282800FFF75DFF0C35022002F07EF9284610F014
:10283800BFFF0E3F81460024163E1FFA87F80DE0C1
:1028480002F07CF902F080F904FB106189B240467D
:102858002022002302F0BAF90134E4B24C45EFD942
:10286800002002F06BF8B8B2B1B22A46012302F098
:10287800ADF9002002F058F9012000E0284605B023
:10288800BDE8F0832DE9F04F85B00546DDF84090AE
:10289800029148469046039310F08AFFDDF838A06D
:1028A800DDF83CB00646294600242F4611E024B145
:1028B800B4420CBF5B46534600E0039B01F1080598
:1028C800ADB200932846029A4346FFF708FF013449
:1028D8002946B442EBDD002002F030F8022002F075
:1028E80023F97D1D08F10508A8B21FFA88F14A46A8
:1028F800012305B0BDE8F04F02F04EB970B540684D
:1029080086B006AB03E9060000282ED0012380F824
:102918002D308668164BF21A534243EB020390F8A7
:102928002C205AB1002B134D134B144A08BF1D46D7
:10293800134B00F11C0418BF13460AE0002B0D4D81
:102948000D4B0E4A18BF1D460D4B00F10C0408BF75
:102958001346BDF81200BDF81410BDF816200096F5
:1029680001950294FFF78EFF012006B070BD00BFED
:10297800302A04086C260408122C04084E2804087F
:10298800F42D040870B5446886B006AB03E9060068
:1029980004B301236377A668104B227FF11A4B42D8
:1029A80043EB01030AB10BB904E01BB966680C4D8F
:1029B8000C4B01E00C4D0D4BBDF81200BDF8141086
:1029C800BDF8162000960C3401950294FFF75AFFC3
:1029D800012000E0204606B070BD00BF7C35040829
:1029E800B83104089A33040852370408283904080F
:1029F8002DE9F04385B004AB03E906004468BDF84F
:102A08000860BDF80A90BDF80C50BDF80E80002C87
:102A180000F08C800123A3740220676802F084F818
:102A28004FF6FF7001F0A0FF002001F087FFEDB224
:102A38005FFA88F8A6F1160189B230462A4643465D
:102A48000097FFF74CFE277A002F2ED1A28A234643
:102A580000E00137974204D29969097E04330029BE
:102A6800F7D002F06BF802F06FF8A9F116091FFA17
:102A780089F90E2101FB10914FF6FF7208F1010848
:102A88005FFA88F389B2009248462A46FFF7B5FDF7
:102A9800022002F049F81F2001F050FFA38A002B02
:102AA80038D0103DE8B2303E2CE0E3685C68A28A7A
:102AB8002346013A002700E00137974204D299697A
:102AC800097E04330029F7D002F038F802F03CF808
:102AD8000E2101FB10914FF6FF7208F101085FFA11
:102AE80088F389B2009248462A46FFF786FD0220FD
:102AF80002F01AF81F2001F021FFA38A53B1103DFC
:102B0800E8B21A3E0637B1B254F82720012308323A
:102B180002F05CF8002002F007F84FF6FF7001F0B1
:102B280023FF1F2001F00AFF012000E0204605B026
:102B3800BDE8F0832DE9F041054636208846144665
:102B48001F4610F03DFA0646E0B120F8025B414608
:102B58002E22FFF717FCBDF8183086F8344073862C
:102B68001820012386F8307086F8313010F028FAE2
:102B7800044618B104234660037404E0304610F09C
:102B880027FA00E004462046BDE8F081F8B506467D
:102B980024200F46154610F013FA0446D8B10F4BFF
:102BA800068083600E4B39464360102200F10C000A
:102BB800FFF7E8FB012600231820256223776677B4
:102BC80010F0FEF9054610B14460067404E0204692
:102BD80010F0FEF900E005462846F8BD7C350408EB
:102BE800D62F0408F8B506462C200F46154610F0D7
:102BF800E7F90446E8B120F80C6B39461922FFF7CB
:102C0800C1FB0D4BA562A3600C4B6360002384F8E5
:102C180025301820012384F8263010F0D1F9054614
:102C280018B103234460037404E0204610F0D0F97F
:102C380000E005462846F8BD884E0408264B0408DF
:102C480010B50446142010F0BBF920B100234380CE
:102C5800014B0480036110BDB124000838B5054656
:102C6800442010F0ADF90446C0B10E4B0582436014
:102C78000D4B0360012383740023037283820B4B83
:102C88000364182010F09CF9054618B10723446026
:102C9800037404E0204610F09BF900E0054628463E
:102CA80038BD00BF1C47040812430408A5250008C6
:102CB8002DE9F04105463420884614461F4610F099
:102CC8007FF9064620B3144B05808360134B4146B9
:102CD8004360102200F10C00FFF754FB214606F177
:102CE8001C001022FFF74EFB002386F82C3018201A
:102CF8000123376386F82D3010F062F9044618B1C5
:102D080005234660037404E0304610F061F900E0E2
:102D180004462046BDE8F081302A04088A240408C5
:102D28002DE9F041044614200D461646984610F049
:102D380047F90746B8B1069B048003610023C372B4
:102D480001234560068180F80A800373182010F07B
:102D580037F9044618B106234760037404E038467F
:102D680010F036F900E004462046BDE8F0812DE970
:102D7800F041044618200D461646984610F020F9F2
:102D88000746B8B101238370069B04800361079B43
:102D980045608660C0F80C804361182010F010F977
:102DA800044618B108234760037404E0384610F05D
:102DB8000FF900E004462046BDE8F0812DE9F34113
:102DC80098461B8B1D2B05460C4617464FF00000F6
:102DD80000F2B480B5F5A07F0090019000F2AE80BB
:102DE800F02900F2AB80127CADF80610511EADF848
:102DF8000250072900F28A80DFE801F045595E0495
:102E0800456A14767B684E4A7A611A8893F834309A
:102E18003A80013BDBB2012B7FD8ADF80240ADF818
:102E280006507AE005F11602ADF8002004F116020A
:102E3800ADF8042002AE434A16E903007A6107F1AF
:102E4800080282E8030003F10802013348F82270FF
:102E5800A8F818307B681A8A187A3A8000286CD14A
:102E6800FFF7FCFE3849436859603849DF6001269E
:102E7800163D196002461E72A8B2E1B24346FFF73A
:102E88009DFF30465AE0012A0CBF314B314B786820
:102E98007B6130F80C3B3B8010F08AFC431CDB0064
:102EA8001A34ED18ADF80440ADF8005035E07B68F1
:102EB800294A1B687A6102E0284A7B687A611B8884
:102EC80014353B80ADF800501434ADF8044024E0CC
:102ED8007B68234A7A611A883A801A899B7AAD18E6
:102EE800ADF80050E418F0E77E681E4B7B6133882C
:102EF80038463B8073689847013D4519ADF8005046
:102F0800B36838469847013C0419DEE71648174A63
:102F1800174B40F21A3100F0E3FC02AA12E9030051
:102F280007F1080383E80300B8F8183003F1080232
:102F3800013348F82270A8F818300120BDE8FC8158
:102F480035250008F9290008083F0408FE3A040856
:102F58008D29000805290008F12700084B270008DB
:102F680017270008C1220008B79A0508D0200408CE
:102F7800B59A0508F8B51646002834D01378002B02
:102F88002ED0028B002327E0046A257C042D21D152
:102F980065682F888F421DD195F8313053B16F8EF7
:102FA80001F0F2FC04F1080268866369204606CA4B
:102FB80098476F86A81C31462E22FFF7E3F995F84B
:102FC80031307BB104F108026369204606CA98478C
:102FD8000120F8BD013304309342D5D30020F8BD59
:102FE8001846F8BD0120F8BD70B5B8B1068B044687
:102FF800002310E0256A287C04280AD16D682888F7
:10300800884206D11046A91C2E22FFF7BBF90120E1
:1030180070BD01330434B342ECD3002070BD38B521
:10302800044620B3134BC361134BC0F89830134BBD
:10303800C0F89C30124B00257822C0F8A030857566
:10304800C5750583294600F1200010F0ABFAD4F8C5
:1030580098302046294698470A4A1388312B07D8C2
:10306800094941F8234001331380012038BD38BD98
:10307800284638BD4D23000845230008E5220008EE
:10308800BB230008740D0020301700202DE9F04103
:103098000446002800F0B380078B02460025A8E00C
:1030A800136A1E7C042E00F08780012E23D15868F5
:1030B80003888B4240F09B8005F108070FF088FFDA
:1030C80054F827004FF00008C0F804800FF080FF84
:1030D800228B531E9D4208D00732238354F82210B6
:1030E80044F8271044F8228002E044F8278025831A
:1030F8003046BDE8F081052E5ED0032E5CD0022E4E
:1031080013D15B68186803888B4270D14388013BF0
:103118009BB243800BB90FF05BFF05F1080654F82A
:10312800263058680FF054FF4EE0072E21D15E6814
:10313800338A8B425BD1002706E0BB1D013756F866
:1031480023000FF045FFFFB2B38ABB42F5D8002732
:10315800B78205F1080654F8263058680FF038FF92
:1031680054F8260033E044F8267025830120BDE892
:10317800F081062E1ED1586803888B4237D105F19D
:1031880008060FF025FF54F82600002747600FF0C7
:103198001FFF228B531E9D4209D00833013A54F871
:1031A8002310228344F8261044F82370DEE744F8FD
:1031B80026701AE0082E1AD1586803888B4216D157
:1031C8000FF006FF05F1080654F8260000274760AF
:1031D8000FF0FEFE228B531E9D42C4D0073254F8D6
:1031E800221044F8261044F822702383BEE70135E4
:1031F8000432BD42FFF454AF0020BDE8F081BDE8C1
:10320800F08170B5044600282AD0068B751E083652
:1032180000EB86061EE056F8043D1A7C042A13D0FB
:10322800012A11D0052A0FD0032A0DD0022A02D173
:103238005B681B6809E0072A02D15B68198A05E008
:10324800062A01D0082A04D15B6819882046FFF7AE
:103258001DFF013D681CDED100232383012070BDC2
:1032680070BDF0B528B30023068B1A461EE0046A29
:10327800257C072D18D16468258A8D4214D1A78A28
:10328800002504EB83040DE004EB050C0435DCF8A1
:1032980018C09CF818C0BCF1010F03F1010301D15B
:1032A800D8B2F0BDBB42EFD301320430B242DED314
:1032B8000020F0BD70B508B3048B00231BE0026A40
:1032C800157C072D15D15268158A8D4211D100231E
:1032D800958A11461C46012007E013B99669307695
:1032E80001E08E69347601330431AB42F5D3012015
:1032F80070BD01330430A342E1D3002070BD2DE935
:10330800F04128B30023078B1A461EE0046A257C87
:10331800072D18D16468258A8D4214D1B4F814C0D9
:10332800002504EB83040CE066190435B66996F8A9
:103338001880B8F1010F03D106F10800BDE8F0814B
:1033480001336345F0D301320430BA42DED30020A2
:10335800BDE8F0812DE9F04700282FD00023B0F810
:1033680018C01D4627E0046A267C072E21D1646810
:10337800268A8E421DD1B4F81480002604EB8309F6
:1033880015E009EB0604A7693C7E012C0DD192F8E3
:1033980000A0BAF1000F08D007F10800114610226A
:1033A800FEF7F0FF2046BDE8F087013304364345B9
:1033B800E7D3013504306545D5D30020BDE8F08753
:1033C800F0B5B0B1068B002510E0046A277C062F03
:1033D8000AD1646827888F4206D123819DF814306A
:1033E8006260A3720120F0BD01350430B542ECD310
:1033F8000020F0BD10B500210446FEF7A3FF2046CB
:103408000121BDE81040FEF79DBF38B598B1048B87
:10341800024600230CE0106A058804328D4206D16A
:1034280000F10802436906CA9847012038BD0133F4
:10343800A342F0D3002038BD10B50C460021FEF79A
:1034480081FF20460121BDE81040FEF77BBF13B580
:1034580002AC04E90C00BDF80230834206D8BDF87E
:103468000030834234BF0020012000E00020BDF876
:1034780006308B4206D8BDF804308B4234BF002199
:10348800012100E00021002818BF0846C0B21CBD79
:1034980038B5114B114A1988002319E052F8045F16
:1034A800A87D012812D100240CE004F1080355F886
:1034B8002300037C082B03D1436800211B6998472C
:1034C8000134A4B22B8BA342EFD838BD01339BB291
:1034D8008B42E3D138BD00BF740D00202C170020AB
:1034E800704770B5094CA5787DB9094B1E78012E37
:1034F8000BD16368013363606268064B9A4204D952
:10350800284601F0D3FAA670656070BD740D0020DE
:103518008401002040420F00054A9060134602E0F3
:1035280099680139996091680029F9D1704700BFFD
:10353800740D0020F0B585B001F066FD002800F09C
:103548004981002502A80DF10A01ADF80850ADF82F
:103558000A5001F05BFD03A80DF10E01ADF80C5007
:10356800ADF80E5001F09EFDBDF80C10BDF8082016
:103578000091BDF80E10BDF80A3001912C46964D09
:103588009649082008F036FCA878012803D101F0F4
:103598008DFAAC7019E1924B5B78012B40F01581E4
:1035A800AB78002B40F011816B6029888D4A09E1C6
:1035B80052F8046FB07D012840F002810025FAE03E
:1035C80005F10803BDF8080056F82340BDF80A10B5
:1035D80004F108030CCBFFF73AFF002800F0E9805C
:1035E800237C013B062B00F29F80DFE803F00429CF
:1035F800159D1F9D4C006668012304F1080533776B
:1036080095E80600636920469847002333772046EB
:10361800636995E8060086E0636893F8252012F14F
:10362800FF3218BF012283F8252077E0636893F8FA
:103638002C2012F1FF3218BF012283F82C206DE0F4
:103648006268137E1568002B6ED16E882F46294656
:10365800184606E051F804EFDEF804E001338EF86E
:103668001800B342F6D301231376002607E057F873
:10367800040F00F10802436906CA984701366B88AF
:103688009E42F4D350E0656820892E68A37B227B94
:103698000096A0F1160189B2FFF721F81420FFF770
:1036A8003BFF2B7AC3B9AF8A29461A461E4609E062
:1036B800886990F818E00676BEF1010F08BF134636
:1036C80004310132BA42F3D301220BB9AB6924E0C9
:1036D800053355F8233020E06368DB685A68002317
:1036E800908A154619461F4609E0AE6996F818E013
:1036F8003776BEF1010F08BF0B4604350131814210
:10370800F3D3411E8B4203D1053052F8203003E039
:1037180004D2073352F8233001221A7604F1080242
:1037280006CA636920469847237C013B072B4CD87F
:10373800DFE803F00410074B0A0D123A63681B6AAE
:1037480034E063689B6A2DE063681B6B2AE063685A
:103758001B6927E0636824E063681A7A7AB9988A53
:103768001946013800E00132824204D28C69247E75
:103778000431002CF7D0063253F8223011E0DB6810
:103788005A68908A11460138002300E001338342C9
:1037980004D28C69247E0431002CF7D0063352F809
:1037A8002330DB69984710E06368DB682046984758
:1037B8000BE00135ADB2338BAB423FF601AF04E00D
:1037C80001339BB28B427FF4F3AE01F063FC0F2010
:1037D800FFF7A2FE05B0F0BD740D0020DD9A0508C4
:1037E800840100202C170020034B9A6812B19A68B4
:1037F800013A9A60704700BF740D00202DE9F34725
:103808000120DFF8D080DFF8D090014609F08CFE67
:103818000025012403234FF4807602274046694699
:103828008DF8053000968DF804708DF806508DF8E7
:10383800074009F0D1FA40460821224609F04CFB1E
:10384800234BDFF898801A6844F2A243B2FBF3FADC
:103858000AF1FF3A204621461FFA8AFA09F094FE37
:10386800C8F804A048464146A8F80050A8F80250F5
:10387800A8F8085088F80A500AF022FA7023A8F825
:103888000C300423A8F810300AF1FF3A63236422AD
:1038980003FB0AF3B3FBF2F39BB2C8F8143008F148
:1038A8000C014846A8F80E40A8F81870A8F81A5055
:1038B800A8F81C60A8F81E500AF020FB48462146CC
:1038C8000AF093FA484621460AF099FDBDE8FC87BC
:1038D800F00200200000024000000140840D00209A
:1038E80083B50E460746154910201C46154608F0B4
:1038F80081FA1020124908F07DFA1020114908F0C9
:1039080079FA10200E4908F075FA002310200E49A4
:10391800019308F06FFA334610200C493A4608F034
:1039280069FA10200A492A4608F064FA1020094961
:10393800224608F05FFA019B0133E7E7179B050869
:103948001C9B05083C9B05084C9B05085C9B0508CF
:10395800719B0508829B050808B5164B1A6A013247
:103968001A621A6A012A1A4603D013484FF4A07142
:103978000FE05862194602E04B6A013B4B62506AFD
:103988000C4B0028F8D11A6A012A06D00A4840F2DE
:103998004B110A4A0A4BFFF7A3FF1A6A013A1A6247
:1039A8001B6A2BB10448054A064B40F24D11F2E759
:1039B80008BD00BF840D0020939B0508AE5804087D
:1039C800BD9B0508CE9B05080C4B0D491A6844F2AF
:1039D800A2436428B2FBF3F3D4BF20EAE07064206A
:1039E800013B9BB24B60013B58436422B0FBF2F0B1
:1039F80080B2486103480C310AF003BAF002002093
:103A0800840D00200000014010B5134B93F82820C6
:103A18002AB11248124A134B4FF40A710EE00122E0
:103A280083F8282066234FF0C042013BDBB21080A8
:103A380033B90A480A4A0C4B40F23221FFF750FFCB
:103A48001488A4B28442F0D1084B1980024B00229A
:103A580083F8282010BD00BF840D0020939B050823
:103A6800B8580408DF9B0508B59A050800000260ED
:103A780010B5FFF7C3FE6420FFF7A6FFE5204FF45B
:103A88000041FFF7C1FF00200121FFF7BDFF012022
:103A98004FF48071FFF7B8FF02204FF4E061FFF7A1
:103AA800B3FF032041F23001FFF7AEFF04200021ED
:103AB800FFF7AAFF082040F20221FFF7A5FF09201F
:103AC8000021FFF7A1FF0A200021FFF79DFF0C202E
:103AD8000021FFF799FF0D200021FFF795FF0F2028
:103AE8000021FFF791FF10200021FFF78DFF112023
:103AF8000021FFF789FF12200021FFF785FF13201F
:103B08000021FFF781FF102041F2B071FFF77CFF21
:103B180037211120FFF778FF3220FFF71DFF122011
:103B280040F23B11FFF770FF3220FFF715FF13201B
:103B38004FF4C051FFF768FF0F212920FFF764FFFA
:103B48003220FFF709FF20200021FFF75DFF212029
:103B58000021FFF759FF30200021FFF755FF3120E2
:103B68000721FFF751FF322040F20311FFF74CFF06
:103B7800352040F20741FFF747FF40F20444362062
:103B880040F60F11FFF740FF37202146FFF73CFFB3
:103B980038204FF48061FFF737FF39202146FFF7BF
:103BA80033FF3C200021FFF72FFF3D204FF48061B9
:103BB800FFF72AFF50200021FFF726FFEF215120B1
:103BC800FFF722FF52200021FFF71EFF532040F28B
:103BD8003F11FFF719FF60204FF41C51FFF714FF46
:103BE80061200121FFF710FF6A200021FFF70CFF79
:103BF80080200021FFF708FF81200021FFF704FF44
:103C080082200021FFF700FF83200021FFF7FCFE40
:103C180084200021FFF7F8FE85200021FFF7F4FE3D
:103C280090201021FFF7F0FE92200021FFF7ECFE14
:103C380093200321FFF7E8FE95204FF48871FFF7E2
:103C4800E3FE97200021FFF7DFFE98200021FFF711
:103C5800DBFE072040F27311BDE81040D4E610B532
:103C6800FFF7CCFD6420FFF7AFFE21210720FFF707
:103C7800CBFE3220FFF770FE01210020FFF7C4FEC3
:103C88003220FFF769FE23210720FFF7BDFE32200F
:103C9800FFF762FE00211020FFF7B6FE41F28830E0
:103CA800FFF75AFE33210720FFF7AEFE3220FFF759
:103CB80053FE112046F63001FFF7A6FE3220FFF72B
:103CC8004BFE4FF4C0610220FFF79EFE3220FFF743
:103CD80043FE122046F6EB41FFF796FE3220FFF72F
:103CE8003BFE03204AF6A401FFF78EFE3220FFF7C1
:103CF80033FE00210C20FFF787FE3220FFF72CFE51
:103D08000D2040F60C01FFF77FFE3220FFF724FE5E
:103D18000E204FF42C51FFF777FE3220FFF71CFEE0
:103D2800B0211E20FFF770FE3220FFF715FE01209C
:103D380042F63F31FFF768FE3220FFF70DFE0520FF
:103D48000021FFF761FE3220FFF706FE0021062062
:103D5800FFF75AFE3220FFF7FFFD16204EF61C71C2
:103D6800FFF752FE3220FFF7F7FD172040F203114C
:103D7800FFF74AFE3220FFF7EFFD00210B20FFF787
:103D880043FE3220FFF7E8FD00210F20FFF73CFE3D
:103D98003220FFF7E1FD41200021FFF735FE3220F8
:103DA800FFF7DAFD42200021FFF72EFE3220FFF751
:103DB800D3FD00214820FFF727FE40F23F143220B0
:103DC800FFF7CAFD21464920FFF71EFE3220FFF704
:103DD800C3FD00214A20FFF717FE3220FFF7BCFD84
:103DE80000214B20FFF710FE3220FFF7B5FD4420DD
:103DF8004FF46F41FFF708FE3220FFF7ADFD0021B9
:103E08004520FFF701FE3220FFF7A6FD2146462098
:103E1800FFF7FAFD3220FFF79FFD302040F20771CF
:103E2800FFF7F2FD3220FFF797FD31204FF40171C3
:103E3800FFF7EAFD3220FFF78FFD32204FF40171C2
:103E4800FFF7E2FD40F202543220FFF785FD2146DC
:103E58003320FFF7D9FD3220FFF77EFD342040F2F2
:103E68000751FFF7D1FD3220FFF776FD35204FF4DB
:103E78000171FFF7C9FD3220FFF76EFD36204FF4C0
:103E88000171FFF7C1FD3220FFF766FD214637209B
:103E9800FFF7BAFDA4F500743220FFF75DFD214657
:103EA8003A20FFF7B1FD3220FFF756FD2F2041F2EF
:103EB800BE21FFF7A9FD3220FFF74EFD21463B202A
:103EC800FFF7A2FD3220FFF747FD00212320FFF76F
:103ED8009BFD3220FFF740FD00212420FFF794FDD1
:103EE8003220FFF739FD25204FF40041FFF78CFD04
:103EF8003220FFF731FD00214F20FFF785FD3220EA
:103F0800FFF72AFD4E200021FFF77EFD3220BDE895
:103F1800104021E508B5124B93F829202AB1114821
:103F2800114A124B40F242210FE0012283F8292066
:103F3800222166234FF0C042013BDBB2118033B926
:103F48000848094A0A4B40F25B21FFF7C9FC108870
:103F580080B22228F0D1024B002283F8292008BD24
:103F6800840D0020939B0508C5580408DF9B0508AD
:103F7800B59A050810B5224B49F22032032823D8F8
:103F8800DFE800F0021A0B111C8846F6280041F2FF
:103F98002801944218BF01461AE01C8841F2080023
:103FA80046F6080104E01C8841F2300046F630016C
:103FB800944208BF01460BE0188846F6200190425B
:103FC80008BF4FF4815103E00E4840F2792113E015
:103FD8001B8848F68912934205D049F22032934251
:103FE80007D1032000E01120FFF70EFDBDE81040C7
:103FF80090E7044840F28521034A044BFFF770FC20
:1040080086010020939B0508DA580408B59A05082C
:10401800014B18800A209FE4000002604FF0C04363
:10402800188003F500331A881A88188880B27047F8
:104038002DE9F041022098B00121002409F074FA1A
:10404800012502268C488DF85C5016A98DF85E4033
:104058008DF85F4016968DF85D6008F0BDFE18205B
:10406800294609F061FA2846294609F075FA2146D9
:104078000C22824808F030FF29460C227F4808F0BD
:104088002BFF04210C227D4808F026FF05210C2275
:104098007A4808F021FF07210C22784808F01CFF15
:1040A80008210C22754808F017FF09210C227348D3
:1040B80008F012FF0A2171480C2208F00DFF0B21AD
:1040C8006E480C2208F008FF0E210C226B4808F0FD
:1040D80003FF0F210C22694808F0FEFE07210C227D
:1040E800674808F0F9FE08210C22654808F0F4FE3C
:1040F80009210C22624808F0EFFE0A210C226048D0
:1041080008F0EAFE0B210C225D4808F0E5FE0C21C0
:104118000A465B4808F0E0FE0D210C22584808F0DA
:10412800DBFE0E210C22564808F0D6FE0C2254481D
:104138000F2108F0D1FE03274CF6B3734F481693AE
:1041480016A98DF85D708DF85E408DF85F408DF88A
:104158005C6008F041FE4FF6807316A94848169334
:104168008DF85D708DF85E408DF85F408DF85C606D
:1041780008F032FE40F6B830FFF7EEFB2246314633
:104188003D4808F09EFE44F6FF70FFF7E5FB2A461F
:104198003146394808F095FE40F6B830FFF7DCFBA9
:1041A8004FF48053102709930DF13C084FF4002376
:1041B80068460F94109412941395149415940094CF
:1041C8000194029404940694079408940A9405941C
:1041D8000B940C9311960397CDF8348008F075FB77
:1041E800042368461193109412941395149415940B
:1041F8000F96CDF8388008F068FB2946204608F06D
:10420800E4FB40F6B830FFF7A7FB2046FFF706FFB0
:1042180004461C491C4D3846224607F0EBFD48F67B
:1042280089139C421AD049F220339C420DD041F2A6
:1042380089239C4212D03846144907F0DBFD144804
:10424800144A154BA621FFF74BFB38461349224663
:1042580007F0D0FD2C80FFF70BFC0AE0FFF7FFFC0E
:1042680048F689122A8010200D4941F2892307F067
:10427800C1FD18B0BDE8F08100040240000C024006
:1042880000100240F49B0508860100200B9C0508DD
:10429800939B0508F2580408B59A0508429C05083E
:1042A800779C05084FF0C04322221A8003F500339B
:1042B80082B01A8892B2ADF806201B889BB2ADF87E
:1042C8000630BDF8060080B202B07047134B1B8859
:1042D80048F68912934210B504460BD049F22032B1
:1042E800934213D1C1F1EF01202089B2FFF78CFB73
:1042F800212006E0C1F1EF014E2089B2FFF784FBCF
:104308004F202146BDE81040FFF77EBB0448054A10
:10431800054B40F2F321FFF7E3FA00BF86010020C6
:10432800939B0508FB580408B59A05082DE9F04148
:104338000D46C5F1F008411E5E18C2EB0802C5F132
:10434800EF039BB292B2B6B29A422CBF90469846FF
:104358009A4234BF11461946864234BF374607464B
:1043680040F23F13864238BF06469E4228BF1E468B
:104378001B4B1B8848F68912B8F1EF0F28BF4FF086
:10438800EF089342044610D049F2203293421FD1DD
:104398005020FFF739FB51204146FFF735FB5220EB
:1043A8003946FFF731FB53200AE041EA082189B278
:1043B8004420FFF729FB45203946FFF725FB462017
:1043C8003146FFF721FB20462946BDE8F0417DE74D
:1043D8000448054A054B40F2DD21FFF781FA00BF8A
:1043E80086010020939B050809590408B59A050819
:1043F80000200146F0224FF4A07397E7072040F20F
:104408007311FFF701BB07200021FFF7FDBA10B5B4
:104418001446FFF75BFFFFF77DFD2046BDE810401F
:10442800F6E508B5FFF752FF4FF0C04322221A8085
:1044380003F500331A88188880B208BDF8B580B231
:1044480002FB03F589B292B29BB2069C9DF81C60F0
:10445800FFF76CFF0020FFF78DFD002709E034F817
:10446800020B1EB1030A43EA002080B2FFF7D0FD19
:104478000137AF42F3DBBDE8F840B9E72DE9F74F64
:1044880016469DF834200C9F01920546B2B280B2C0
:104498000C46984689B29BB2FFF748FF4FF0000BD5
:1044A8000020FFF767FDDA463DE0002D30DB09EB21
:1044B800050340F23F1293422ADC002C28DB0BEB69
:1044C8000403EF2B24DC19F00F0F04D1B9F1000F0E
:1044D800C8BF0AF1010A174B09EA0303002B03DAE4
:1044E800013B63F00F030133019A0AB1C3F10F03D3
:1044F800012202FA03F337F81A2013401BB213B152
:104508000D4B588D01E00D4A508880B2FFF780FDB1
:1045180009F1010901E04FF00009C145C5DB0AF1C5
:10452800010A0BF1010BB345F5DB03B0BDE8F04F11
:104538005EE700BF0F000080840D00208601002088
:104548002DE9F04F85B004469DF83C000292002703
:104558008A46039088463E4640F23F1C9B463AE016
:10456800002C2FDBE1452DDCBAF1000F2ADBB8F176
:10457800EF0F27DC2A0702D1002DC8BF01361B49DF
:104588002940002903DA013961F00F010131039A4A
:104598000AB1C1F10F010E9830F8162003FA01F1A3
:1045A8000A4012B272B112494A8D019392B21FFAAF
:1045B80089F01FFA88F1CDF800C0FFF728FFDDF871
:1045C80000C0019B013509F101095D45C8DB0136D1
:1045D800013708F10108029A974203DAA14600253B
:1045E8000123F2E705B0BDE8F08F00BF0F0000809F
:1045F800840D002082B0044BADF80600BDF80620FB
:1046080092B25A8502B07047840D002082B0044BE4
:10461800ADF80600BDF8062092B25A8002B0704785
:104628008601002070B50646FFF7E2FE0020FFF77E
:10463800A1FCF02409E0013D3046ADB2FFF7E8FCEB
:10464800002DF8D1013CA4B214B14FF4A075F2E7E3
:1046580070BD70B51D461446FFF738FE2846FFF7B3
:1046680089FC0025054E05E0708D80B2FFF7D0FC6F
:104678000135ADB2A542F7D170BD00BF840D002051
:104688002DE9F0410C4616461F461A4600230546FA
:10469800FFF7DFFF611E711828463A46002389B2EA
:1046A800FFF7D7FF2846214632460123FFF7D1FFFF
:1046B800013D7F19B8B2214632460123BDE8F041D9
:1046C800C7E770B580B202FB03F489B292B29BB21D
:1046D800FFF72CFE0020FFF74DFC0025054E04E0F7
:1046E800708D80B2FFF794FC0135A542F8DBBDE878
:1046F80070407DE6840D0020F8B5561A0C4601314D
:1047080089B21F460546FFF7E1FD0120FFF732FC9D
:104718004FF0C04322221A800E4A0F491388B6B2BE
:10472800002304E01088013321F8020B9BB2B34246
:10473800F8D121462846FFF7C9FD0120FFF71AFCEA
:10474800002404E03846FFF763FC0134A4B2B44205
:10475800F8D1F8BD000002602646002070B5194B5C
:10476800194AD98D92F9004064180025A4B2AC42C8
:1047780008BF0124C62C28BFC6240F2615704FF683
:10478800FF7288B09E85DC855A8519200A222B463F
:104798002146FFF75EFF21463046FFF742FE2246DC
:1047A80003460A4968460EF07DFF6A4604A8084990
:1047B8000EF078FF3220D22104AA2B4600F0ECF943
:1047C80008B070BD840D0020E42D0020B69C0508BB
:1047D800BE9C05082DE9F0431F2093B0FFF722FF88
:1047E8004FF47840FFF71EFF4FF6E0754FF4FC607A
:1047F800FFF718FF2846FFF715FF0020494CFFF781
:1048080011FF00200146642203464FF6FF79A4F801
:104818002A90FFF71EFF00200A2164220346FFF7B3
:1048280018FF00200146642201234FF4784765856C
:10483800FFF70FFF7720EF21C82200234FF4FC6613
:104848006785FFF706FFBD213222012340F23F10A2
:104858006685FFF7FEFEA0203222002378216785B7
:10486800FFF7F7FEA0207821322201234FF01F081E
:104878006685FFF7EEFEA020782132220223A4F8F5
:104888002A80FFF7E6FEA0207821322203236585DF
:10489800FFF7DFFE244B2549A3F8028002AD3C2236
:1048A80028460EF03DFEEB20C3210522302300955B
:1048B8000025A4F82A900195FFF7E0FD32210A208F
:1048C80096220B466785FFF7DBFE32213C209622B5
:1048D8000B466685FFF7D4FE32210B4696226E20E2
:1048E800A4F82A80FFF7CCFEFFF78DFDFFF786FDC1
:1048F8003220FFF769F82846FFF766F86420FFF7CB
:1049080063F80B4B03F110028DE8240028465A681F
:104918001B682946FFF792FD1195119B01331193EE
:10492800FBE700BF840D0020860100201E59040803
:10493800607D010800487047FC17002082B0064BD4
:10494800ADF80600BDF8062092B21A80188880B229
:1049580002B0FFF74FBE00BFF8170020014B1888C0
:1049680080B27047F817002082B0064BADF80600F9
:10497800BDF8062092B21A80188880B202B0FFF7FC
:1049880045BE00BFFA170020014B188880B2704757
:10499800FA170020FFF746BEFFF7C8BCFFF759BE5D
:1049A800FFF76EBEFFF78DBE2DE9F04F4FEA4208C4
:1049B80000253D4C85B082468B46C8F10308174652
:1049C8002E461FFA87F909EB0B0C228805EB0A0320
:1049D8001FFA8CFC9BB26146184692B2CDF804C00F
:1049E8000293FFF714FDC9EB0B0292B20392029BEC
:1049F80022880399184692B2FFF709FDDDF804C032
:104A08002288C5EB0A039BB26146184692B202930C
:104A1800FFF7FDFC029B22880399184692B2FFF724
:104A2800F6FC05EB0B0292B2039209EB0A0322880B
:104A380003999BB2184692B20293FFF7E8FC029BD7
:104A48002288C5EB0B0C1FFA8CFC1846614692B203
:104A5800CDF804C0C9EB0A09FFF7D9FC22880399ED
:104A68001FFA89F992B24846FFF7D1FC2288DDF88F
:104A780004C092B248466146FFF7C9FCB8F1000F7E
:104A880004DA08EB860808F1060805E0F31B08F1CC
:104A98000A0808EB8308013F01360135BE42ADB272
:104AA8008FD905B0BDE8F08FF817002008B9FFF7D7
:104AB800AABC012801D1FFF7A1BC704770470020AC
:104AC8000146F0224FF4A073FFF730BC704708B5D9
:104AD80005280CD8DFE800F0121403050709094877
:104AE80008BD094808BD094808BD094808BD094866
:104AF800094A0A4B40F24111FEF7F2FE084808BD88
:104B0800084808BD74010020640100205C010020F1
:104B180054010020C39C05085A590408B59A050891
:104B28007C0100206C01002010B50446FFF7CFFF80
:104B3800014B18601C7110BD8C010020014B1879C5
:104B4800704700BF8C01002008B5FFF7C0FF8088C0
:104B580008BD08B5FFF7BBFFC08808BDF7B51F46FD
:104B68000B4B0C4E1D681446EA882B68203C5443B6
:104B7800A4B2AE1B03EB440418BF0126AB888DE832
:104B8800500017B1FFF7DCFC01E0FFF777FCFEBD32
:104B98008C0100207C0100202DE9F0410F46984649
:104BA80015460446084E08E0204643463946FFF7B6
:104BB800D5FF33689B88E418A4B215F8012B002AA6
:104BC800F2D1BDE8F08100BF8C01002010B5044689
:104BD80008462146BDE81040DEE7094B70B504469B
:104BE80018790E461546FFF7B4FFC6F1F001091A09
:104BF80089B220462A460023BDE87040CCE700BFB2
:104C08008C010020704700BF044B1A680AB9044A97
:104C18001A601A681018186010467047B40D002002
:104C2800EC5100204FF0FF30704708B50248034AA6
:104C3800034B3721FEF754FEE29C0508705904081F
:104C4800B59A05080120704710B504460A480221A4
:104C580008F0F0FE0028F9D00748214608F0B3FE16
:104C68000548012108F0E6FE0028F9D00248BDE811
:104C7800104008F0A5BE00BF0038004010B5194824
:104C8800022108F0D7FE0028F9D01648002108F0C4
:104C98009AFE1448012108F0CDFE0028F9D01148E9
:104CA80008F08EFE0402A4B2002301E001339BB297
:104CB800002BFBD00B48022108F0BCFE0028F9D0DD
:104CC8000848002108F07FFE0648012108F0B2FEDE
:104CD8000028F9D0034808F073FE2043C0F3CB0046
:104CE80010BD00BF003800402DE9F0478AB00AAF78
:104CF8000A20012108F018FC4FF4604347F8143DDE
:104D0800474EDFF824A1012400254FF00208304661
:104D180039468DF81A508DF818808DF819808DF85D
:104D28001B4008F059F830460D21052208F0D4F848
:104D380030460E21052208F0CFF8052230460F2113
:104D480008F0CAF821464FF4804008F011FC50469C
:104D580008F0ECFC4FF48273ADF802304FF40073A6
:104D6800ADF80A303823ADF80C30504607236946B1
:104D7800ADF81030ADF80050ADF80450ADF806505D
:104D8800ADF80850ADF80E5008F002FD5046214627
:104D980008F099FDA9468DF81A5030464FF4805511
:104DA800394605958DF818408DF819808DF81B4007
:104DB80008F012F83046294608F07FF840253946B1
:104DC80018488DF818908DF819808DF81A908DF87C
:104DD8001B40059508F000F821464FF4804008F084
:104DE800D3FB0621032008F05DFE0C2307A88DF8ED
:104DF800213007958DF820908DF8224007F0E0FCCF
:104E080017238DF8243009A80F238DF825308DF845
:104E180026308DF8274002F06BFB0AB0BDE8F0871A
:104E280000040240000C024000380040014B187892
:104E3800704700BFB80D0020024B5A889B8802803B
:104E48000B807047B80D0020014B00221A70704784
:104E5800B80D0020F0B593B06846002148220EF046
:104E6800A1FB6D46002464484FF4805108F027F8F0
:104E7800002301E001339BB2002BFBD09020FFF709
:104E8800E3FE002301E001339BB2002BFBD0FFF7C8
:104E9800F5FE4FF480510746574808F00EF80023F6
:104EA80001E001339BB2002BFBD053484FF48051F3
:104EB80008F005F8002301E001339BB2002BFBD07A
:104EC800D020FFF7C1FE002301E001339BB2002B85
:104ED800FBD0FFF7D3FE4FF480510646464807F053
:104EE800ECFF45F8047B01342E6244484021E4B2CB
:104EF80007F0D1FF10B9092CB5D101E0092C78D100
:104F08009DE80C00D218029B03980699D218049BBE
:104F1800C018059BC018079BCB180899032490FB61
:104F2800F4F092FBF4F25B1893FBF4F3151AC11A30
:104F38009C1A002DB8BF6D420029B8BF4942002C09
:104F4800B8BF6442502D03DD502909DD502C50DCD8
:104F58008D4205DAAC424FF0020405DB111806E079
:104F68008C424FF0020401DAD11800E0C1180A9B04
:104F7800099A0C980F9DD2180B9BD2180D9BC0183C
:104F88000E9BC018109BEB18119D91FBF4F10324A4
:104F980092FBF4F290FBF4F05B1993FBF4F3161A0E
:104FA800C41A9D1A002EB8BF7642002CB8BF6442BE
:104FB800002DB8BF6D42502E89B203DD502C09DD9B
:104FC800502D16DCA64205DAB5424FF0020405DB87
:104FD800131806E0A5424FF0020401DAD31800E0E6
:104FE800C318074A93FBF4F39BB2938001235180C3
:104FF800137013B0F0BD00BF00040240000C024063
:10500800B80D002000000000FFF710BFF7B50546F7
:105018000C4601A80DF10601FFF70EFF1B4BBDF86A
:105028000660BDF8040093E80600724301FB002205
:1050380099685218164992FBF1F207EE102AF8EE19
:10504800C77A40F23F17FCEEE77A17EE902A92B241
:10505800B2F5207F28BF3A462A801D69DA685B6965
:105068006E4302FB0060C01890FBF1F107EE101AC6
:10507800F8EEC77AFCEEE77A17EE903A9BB2B3F5F2
:10508800F07F28BFEF232380FEBD00BFC00D0020A6
:1050980040420F00FFF7D8BE014B187E704700BF93
:1050A800C00D0020FFF7C8BE042808B505D9074879
:1050B800074A084B7D21FEF713FC054B03EB8000E4
:1050C800038B0B80438B138008BD00BF039D05082D
:1050D80076590408219D050808B5082001F094F9BF
:1050E80042F69643C31A584240EB030008BD10B578
:1050F8000A2001F0B1F90C4C20600E2001F0ACF947
:105108006060122001F0A8F9A060162001F0A4F94F
:10511800E0601A2001F0A0F920611E2001F09CF93E
:1051280001236061237610BDC00D002010B5FFF784
:10513800DBFD01F033FA044601F03CFA0749034667
:105148002246202006F056FEFFF7C6FF28B101F0E0
:105158003FFA10B9BDE81040C9E710BD5D9D0508CC
:1051680010B5104C0A20216801F05DF961680E2025
:1051780001F059F9A168122001F055F9E1681620EB
:1051880001F051F921691A2001F04DF961691E20D9
:1051980001F049F9082042F69641BDE8104001F0B7
:1051A80025B900BFC00D00202DE9F04F0346A7B078
:1051B800B0F800C01C898688DF885D89CDF810C0EA
:1051C800B249B0F802C0B3F80C90B3F80E80CDF82D
:1051D80024C00FFA84FB30B201220FFA87FE0BEBD2
:1051E800000C0A7629B20FFA89FACDF888C001EBCB
:1051F8000E0C0FFA88F2CDF890C00AEB0B0CCDF824
:1052080030C002EB010CCDF858C0B3F810C05B8A6F
:10521800CDF800C00FFA8CFC06910CEB00010A9146
:1052280002930CEB0A011BB2239103EB0E010E91C2
:1052380099182591049900FA81F058445044604423
:10524800DDF824C006990EFA8CFEDDF810C01FFAAE
:1052580080FB1CFB0CF08E4416FB0600964414FBE6
:105268000400009A19FB09009E4412FB02001FFA71
:105278008EFA09F0E9FCDDF824C0029ACDE91201A2
:105288001CFB0CF017FB070015FB050018FB0800BA
:1052980012FB020009F0D8FCDDF824C0029ACDE91F
:1052A800140104991CFB01F317FB063615FB046671
:1052B800009B18FB096612FB036009F0C5FCDDE9D9
:1052C8001423CDE90001DDE9120109F033FD04469C
:1052D8000D46DDE9000102460B4609F02BFD0246AA
:1052E8000B462046294609F071FBCDE918015846BE
:1052F80009F0BAFCCDE91001DDE91023DDE9000170
:1053080009F018FDCDE90601504609F0ADFC8046CC
:1053180089464246DDE912014B4609F00BFDDDE9FD
:105328001023CDE91C01DDE9140109F003FD002279
:1053380006460F46564BDDE9180109F0FBFC4246CC
:1053480004460D464B46DDE9060109F0F3FC02462A
:105358000B4609F03DFB02460B462046294609F05C
:1053680037FB424604460D464B46DDE91C0109F071
:10537800E1FC02460B462046294609F027FBDDE9F9
:10538800102304460D463046394609F0D3FC024640
:105398000B462046294609F019FBDDF828C0CDE95F
:1053A80002014FEA8C10DDF830C000EB0C20DDF86C
:1053B80010C0A0241CFB040009F046FCDDF838C02E
:1053C800CDE90A014FEA8C10DDF858C000EB0C203B
:1053D800DDF824C01CFB040009F036FCCDE90C0103
:1053E800504609F031FCDDE91023CDE91601DDE96D
:1053F8000C0109F09FFC4246CDE91E014B46DDE950
:105408000A0109F097FC4246CDE920014B46DDE947
:10541800000109F08FFC32463B4609F0D7FACDE986
:105428000E01584609F010FCDDE91C23CDE91A01EC
:10543800DDE9060109F0CAFADDF88CC0C024CDE91F
:10544800060104FB0CF0DDF888C0302505FB0C00D4
:10545800DDF810C078261CFB060009F0F5FBDDF826
:1054680094C0824604FB0CF0DDF890C005FB0C00EC
:10547800DDF824C01CFB06008B4609F0E5FBDDE9DE
:10548800102306460F4609F055FC03E0C00D002026
:10549800000014404246CDE904014B4650465946A7
:1054A80009F048FCDDE9142380468946DDE90A0154
:1054B80009F040FCDDE9002304460D46DDE90C0156
:1054C80009F038FC02460B462046294609F07EFAC8
:1054D8000022A14B09F02EFCDDE9202304460D46ED
:1054E800DDE91E0109F072FA02460B46DDE91601F4
:1054F80009F020FC02460B462046294609F068FAC6
:10550800002204460D46954BDDE90E0109F012FC18
:1055180002460B462046294609F05AFADDE90223DD
:1055280009F032FD88A3D3E9002309F003FC09F050
:105538009BFE8B490860DDE91223DDE90C0109F0C7
:10554800F9FBDDE9002304460D46DDE90A0109F00F
:10555800F1FB02460B462046294609F037FA00229D
:105568007D4B09F0E7FBDDE91E2304460D46DDE926
:10557800200109F02BFA02460B46DDE91A0109F071
:10558800D9FB02460B462046294609F021FA00229B
:1055980004460D46714BDDE9060109F0CBFB0246D6
:1055A8000B462046294609F013FADDE9022309F0E3
:1055B800EBFC65A3D3E9002309F0BCFB09F054FE1A
:1055C800674A5060DDE90E23DDE90A0109F0B2FB04
:1055D800DDE9062304460D46DDE90C0109F0AAFBC6
:1055E80002460B462046294609F0F2F900220446F5
:1055F8000D465A4BDDE9180109F09CFB02460B46A3
:105608002046294609F0E4F9DDE9022309F0BCFC4B
:105618004DA3D3E9002309F08DFB09F025FE504B7B
:1056280059469860DDE91423504609F083FBDDE90B
:10563800002304460D463046394609F07BFB0246F6
:105648000B462046294609F0C1F90022424B09F0D1
:1056580071FB424604460D464B46DDE9040109F05C
:10566800B5F902460B46DDE9160109F063FB02466F
:105678000B462046294609F0ABF935A3D3E90023A8
:1056880004460D46DDE90E0109F054FB02460B46BF
:105698002046294609F09CF9DDE9022309F074FC4B
:1056A80029A3D3E9002309F045FB09F0DDFDDFF864
:1056B800B0C0DDE91223CCF80C003946304609F0B9
:1056C80039FBDDE9002304460D465046594609F0EA
:1056D80031FB02460B462046294609F077F900229D
:1056E8001D4B09F027FBDDE9042304460D4640461F
:1056F800494609F06BF902460B46DDE91A0109F043
:1057080019FB02460B462046294609F061F910A309
:10571800D3E9002304460D46DDE9060109F00AFB3A
:1057280002460B462046294609F052F9DDE90223D4
:1057380009F02AFC04A3D3E9002309F0FBFA09F0D5
:1057480093FD074908610DE00000000080842E41A8
:105758000000000000C082400000144000008940A2
:10576800C00D0020DDE90E235046594609F0E2FA43
:10577800DDE9062304460D463046394609F0DAFAD3
:1057880002460B462046294609F022F911A3D3E91F
:10579800002304460D46DDE9180109F0CBFA02465C
:1057A8000B462046294609F013F9DDE9022309F0E2
:1057B800EBFB0AA3D3E9002309F0BCFA09F054FD76
:1057C800034A506127B0BDE8F04FC9E4AFF3008049
:1057D800C00D00200000000000C082400000000052
:1057E80080842E41AFF30080064B074A5968116048
:1057F8001969064A1160D969054A11609A6A054B08
:105808001A60704794010020B03E0020CC4400206C
:10581800A4440020603E0020014B1878704700BF68
:10582800DC0D0020032808B505D90548054A064BB4
:105838007321FEF755F80C235843044B185808BD3C
:10584800989D0508A2590408B29D050894010020F6
:10585800032808B505D90648064A074B7821FEF7FC
:105868003FF8064B0C2202FB0030406808BD00BF21
:10587800989D0508B2590408B29D050894010020B6
:10588800034B044A1B780C2101FB032398687047DB
:10589800DC0D002094010020034B044A1B780C20E7
:1058A80000FB032399607047DC0D00209401002061
:1058B800144B1B78012B10B5134B144C0ED11968DF
:1058C800C82000F0B0FD2168CC2000F0ACFD104BE2
:1058D800D020196800F0A7FDD4200DE01968D82061
:1058E80000F0A1FD2168DC2000F09DFD084BE020C0
:1058F800196800F098FDE420064B1968BDE81040CF
:1059080000F091BD380F0020B03E0020CC440020AC
:10591800A4440020603E0020144B1B78012B10B5D6
:10592800134C0FD1C82000F097FD2060CC2000F068
:1059380093FD104B1860D02000F08EFD0E4B1860C0
:10594800D4200EE0D82000F087FD2060DC2000F095
:1059580083FD084B1860E02000F07EFD064B1860C0
:10596800E42000F079FD054B186010BD380F0020C9
:10597800B03E0020CC440020A4440020603E00201B
:1059880008B502F01DFB10B1BDE80840C4E7BDE84A
:10599800084029E70148FBF7FABD00BFE4150020DD
:1059A8000148FBF7F4BD00BFE41500200148FBF7F0
:1059B800EEBD00BFE41500200148FBF7E8BD00BFBD
:1059C800E4150020032808B505D91648164A174BD0
:1059D8004F21FDF785FF164B1870164B1870164BA4
:1059E800012202281A70154B0FD0032813D09042B9
:1059F80005D0134A12681A60BDE80840CAE7114A80
:105A080012681A60BDE80840CAE70F4A12681A60AF
:105A1800BDE80840CAE70D4A12681A60BDE80840A8
:105A2800CAE700BF989D0508C3590408DC9D05080E
:105A3800DC0D0020A63E0020080E0020EC0200200D
:105A4800E4020020E0020020DC020020D80200204E
:105A5800064B07495960C021002219721E211A708D
:105A6800D9601A745A611A76DA61704728180020CA
:105A780040787D0110B50321FF22C02001F094F881
:105A88001F4C102120608022C02001F08DF81121C8
:105A980020608022C02001F087F812212060802237
:105AA800C02001F081F8132120608022C02001F07D
:105AB8007BF8142120608022C02001F075F81521A0
:105AC80020608022C02001F06FF88022206016211B
:105AD800C02001F069F82060C0201721802201F061
:105AE80063F82060074CC020227AB72101F05CF8E7
:105AF8000023237463612376E3610123237010BDBF
:105B0800843E00202818002038B5C0200321FF2239
:105B180001F04AF80B4D00242B19615D5A78C0201A
:105B2800023401F041F8C82CF6D1B121AC22C020D2
:105B380001F03AF8C0200321002201F035F80020D6
:105B480038BD00BFD75904082DE9F34706460F466C
:105B580092461D461AB90C1FE401914635E005EE40
:105B6800902A06EE903AB8EE657AF8EE667AFC016D
:105B7800C7EE277AA4F500749FED5C7A67EE877A02
:105B880017EE900A09F082F841EC100B0BF0ACF814
:105B980059EC108B4946404609F08EFB24184FEA11
:105BA800CA1009F051F8CDE90001284609F04CF86F
:105BB8004B46424609F0BEF802460B46DDE90001B5
:105BC80008F004FF09F078FB8146002E14BF4FF05F
:105BD80022084FF01A08C5F307224146C02000F0FA
:105BE800E3FF08F10101EAB2C02000F0DDFFC4F3D1
:105BF800014208F10201C02000F0D6FFC4F30722D9
:105C080008F10301C02000F0CFFFE2B208F104015F
:105C1800C02000F0C9FFC9F3034305F4702243EA2A
:105C2800123208F10501C02000F0BEFF08F106019C
:105C3800C9F30722C02000F0B7FF08F107015FFA97
:105C480089F2C02000F0B0FFC020B121A02200F0EE
:105C5800ABFF07EE107A264CF8EEC77A0EBBD4EDF0
:105C6800015A06EE90AAB8EE657A05EE905AB8EE9B
:105C7800666AF8EE656A0123C6EE266A237477EE33
:105C8800A67A67EE277A17EE900A08F0FFFF41EC34
:105C9800100B0BF029F851EC100B09F00DFB6061AB
:105CA80020E005EE90AAD4ED016AB8EE656A05EE2B
:105CB800905AB8EE667AF8EE656A0123C6EE266A4F
:105CC800237677EEA67A67EE277A17EE900A08F021
:105CD800DDFF41EC100B0BF007F851EC100B09F04D
:105CE800EBFAE0610020BDE8FC8700BF000000433C
:105CF800281800200022012326E7012838B50D4680
:105D080004D002280CBF3C242C2400E03424214673
:105D1800C02000F0C3FF05F0070200F00F0040EAC2
:105D280002122146C020BDE8384000F03DBF2DE9F1
:105D3800F3470A9C1D4607468A461646524B01E021
:105D48006D0864089C42FBD82DB906F10076043E24
:105D5800F601A94634E006EE905AB8EE667A06EEE9
:105D6800904AF8EE667AF601C7EE277AA6F500762D
:105D78009FED467A67EE877A17EE900A08F086FF5D
:105D880041EC100B0AF0B0FF59EC108B4946404625
:105D980009F092FA3618E80108F056FFCDE900013B
:105DA800204608F051FF4B46424608F0C3FF024622
:105DB8000B46DDE9000108F009FE09F07DFA81468D
:105DC800022F9BBF324BDB194FF0000893F8C880B5
:105DD800C4F307224146C02000F0E6FE08F10101A5
:105DE800E2B2C9B2C02000F0DFFE08F10201C9B278
:105DF800C6F30142C02000F0D7FE08F10301C9B282
:105E0800C6F30722C02000F0CFFE08F10401C9B292
:105E1800F2B2C02000F0C8FE04F47024C9F30343B2
:105E280008F1050143EA1432C9B2C02000F0BCFEF3
:105E380008F10601C9B2C9F30722C02008F1070812
:105E480000F0B2FE5FFA89F25FFA88F1C02000F034
:105E5800ABFEBAF1010F0CBF2F220F220DB942F091
:105E68004002012F06D002D3022F0AD105E0C0203C
:105E7800102104E0C020112101E0C020122100F00F
:105E880093FE0020BDE8FC87FFFF0F0000000043E1
:105E9800D759040807B5012300930023FFF747FFEC
:105EA8000EBD00280CBFFF22002208B5C020032128
:105EB80000F07AFE002008BD08B5C020B121AC2250
:105EC80000F072FE002008BD08B50420012107F08B
:105ED8002BFB4FF480700121BDE8084007F054BB4C
:105EE80007B50223009303238DF8043003480023E9
:105EF80069468DF8073006F06FFF0EBD00080240B6
:105F080030B5124D8BB0002406A806940794089467
:105F1800099406F02FF900948DF804408DF8054097
:105F28000294039404942846012469468DF8144089
:105F380006F0F1F828460B212246062306F066F9FA
:105F48002846214606F030F90BB030BD002001404C
:105F580010B5002104460122302000F025FEC0B90A
:105F6800012001F041F8002CB8BF4034E4B2102100
:105F78002246302000F018FE012001F035F83020CC
:105F88001121224600F010FE0120BDE8104001F06A
:105F98002BB810BD10B5002104460122302000F0B6
:105FA80003FEC0B9012001F01FF8002CB8BF40342F
:105FB800E4B212212246302000F0F6FD012001F063
:105FC80013F830201321224600F0EEFD0120BDE831
:105FD800104001F009B810BD38B5012205460C463D
:105FE8003020002100F0E0FDF0B9012000F0FCFFB6
:105FF80025EAE5725F2AA8BF5F223B21D2B2302092
:1060080000F0D2FD012000F0EFFF24EAE4725F2ADD
:10601800A8BF5F22D2B230203C2100F0C5FD01208C
:10602800BDE8384000F0E0BF38BD302810B5044660
:106038000ADC10F17F0F02DB002802DB05E06FF0BD
:106048007E0404F5807400E03024002130200A46E4
:1060580000F0AAFDA8B90120E4B200F0C5FF412173
:106068002246302000F0A0FD012000F0BDFF3020C6
:106078004221224600F098FD0120BDE8104000F0C2
:10608800B3BF10BD282810B5044609DC10F1180F5D
:1060980002DB002802DB04E06FF017047F3400E025
:1060A8002824002130200A4600F07EFDA8B90120EE
:1060B800E4B200F099FF53212246302000F074FD2D
:1060C800012000F091FF30205421224600F06CFDA1
:1060D8000120BDE8104000F087BF10BD08B5302092
:1060E8000021012200F060FD60B9012000F07CFF72
:1060F80030203321402200F057FD0120BDE8084040
:1061080000F072BF08BD10B530200021012200F058
:106118004BFD044660B9012000F066FF30203321B2
:10612800224600F041FD0120BDE8104000F05CBFB0
:1061380010BD10B530200021012200F035FD0446C5
:10614800A0B9012000F050FF34212246302000F091
:106158002BFD012000F048FF30203721224600F0B7
:1061680023FD0120BDE8104000F03EBF10BD4020D7
:10617800EEE640200EE708B500210122302000F0AD
:1061880013FD012000F030FF30203421024600F0DA
:106198000BFD012000F028FF30203721024600F0D7
:1061A80003FD0120BDE8084000F01EBF08B500212E
:1061B8000122302000F0F8FC012000F015FF30200B
:1061C80034210C2200F0F0FC0120BDE8084000F06A
:1061D8000BBF000000000000184B1949D3ED006AFE
:1061E80093ED017A00231A469FED166A03E0F0EE5C
:1061F800476AB0EE677A505E05EE900AF8EEE57AE7
:106208000133C7EE867A9BB218B204327F2877EE44
:10621800E67AECDD27EE077A07EEA77A0A49074AFD
:106228000B80BDEEC77A002313605360C2ED027A7B
:1062380017EE102A054B92001A607047E00D0020F7
:10624800E42900200000FA45143E0020B01A00207E
:106258002DE9F84F2E4B2F4A19682F4B19B92F49A2
:1062680011602F4A02E02F4911602F4A1A602F4B04
:10627800DFF8BCA0DFF8BC90DFF8BCB000221A80C1
:10628800244A9846176830E007EB84036500B3F9A1
:10629800023007EE103AF8EEC77A013617EE900A88
:1062A80008F0F4FC18A3D3E9002308F043FD08F034
:1062B800DBFF29F815002AF8140037F9243007EE17
:1062C800103AF8EEC77A013517EE900A08F0DEFCAE
:1062D8000DA3D3E9002308F02DFD08F0C5FF2BF826
:1062E800140029F81500A8F80060B8F8006034B266
:1062F800FF2CC9DD00F05EF800F06AF801F09CF9A7
:10630800BDE8F84F68E700BF9A9999999999E93FCC
:10631800A41A0020981A0020D0180020E631002086
:10632800E62D0020E6390020E6350020143E002046
:10633800E4250020E4290020E427002010B50B4CB8
:10634800204606F096F90A4B18600A4806F091F9BB
:10635800094B1860FFF77CFF084B094901222046CA
:106368009A81BDE8104006F005BA00BF10600240EF
:10637800A41A002088600240C01A0020E00D002006
:1063880020800010014B1868704700BFB01A002029
:1063980008B5054B054819880022012309F096FC29
:1063A800034B187008BD00BFC4010020CC25002095
:1063B800E820002003480449044A4FF4807309F098
:1063C800FDBC00BFC8010020E4250020CA2300202E
:1063D80003480449044A4FF4807309F0EFBC00BF36
:1063E800D4010020E4270020041C002038B505460D
:1063F8000C460135C1F3072100F004FEA8B2E1B252
:1064080000F000FE00B238BD38B5044600F00EFDBD
:1064180001340546A0B200F009FDEDB2C0B240EA71
:10642800052000B238BD37B50B0E8DF804300B0CC3
:106438008DF805300B0A8DF806308DF8071000240A
:1064480000E0284601AB451CE15C013400F0DAFDB0
:10645800042CADB2F5D13EBD37B5002400E0284686
:10646800451C00F0E3FC01ABADB2E0540134042C50
:10647800F5D19DF805009DF80430000440EA03605A
:106488009DF8073018439DF8063040EA03203EBDCA
:1064980038B50446642000F0A7FD25786068AD0093
:1064A800EDB2257006F0FDFC237A40FA03F000F007
:1064B80003000543104B257005F00F055A5D6378FE
:1064C800D218D2B2D3B20132D2B2022A637001D842
:1064D8000022A2705BB2012B03DD0123A37000230D
:1064E800637094F90130013303DAFF23A3700023AA
:1064F800637094F9020038BDA25A0408F7B5042065
:106508000121234F07F010F802AD01214FF480401C
:10651800012407F039F800264FF4B073384669466D
:1065280045F8083D8DF804608DF8074006F054FCE6
:106538001020214606F0F8FF782369461548009395
:106548008DF804608DF8074006F046FC04202146CB
:1065580006F0EAFF21464FF4804007F015F81C23A7
:106568003846694600938DF804608DF8074006F0B8
:1065780033FC0220214606F0D7FFB02306488DF8E9
:10658800046069468DF80740009306F025FCFEBDBF
:10659800000802400010024000040240802108B5B3
:1065A800034806F078FCD0F1010038BF002008BD90
:1065B8000004024008B54FF48071044806F06BFCF3
:1065C800D0F1010038BF002008BD00BF000802401C
:1065D80008B5FFF7E3FF08B1FFF7ECFFC0B208BD4D
:1065E80010B5642000F000FD1D48FFF751FF044678
:1065F80010B91C4B187009E0FFF7DCFF30B9002C0C
:10660800184B01DD012200E0FF221A701648FFF73F
:106618003FFF164B1B78042B16D100281FD0144BB4
:106628001A7806DD0132D2B20F2A1A7008D9102260
:1066380005E0013AD2B2102A1A7001D900221A7064
:10664800BDE81040FBF79AB800280A4B01D1187032
:1066580010BD02DD01221A7010BDFF221A7010BD94
:1066680014020020A844002020020020483E0020F8
:10667800AE3E0020E42D002007B50220012106F0DF
:1066880053FF012300938DF8043002238DF8053061
:106698000448002369468DF806308DF8073006F067
:1066A8009BFB0EBD0004024010B5084C01210022DE
:1066B800204606F006FC40F2FF4000F095FC012160
:1066C80020460A46BDE8104006F0FBBB0004024025
:1066D80008B5FFF7E9FF00210A46302000F064FA08
:1066E800012000F081FC01210A46302000F05CFA0C
:1066F800012000F079FC00210122302000F054FA3A
:10670800012000F071FC01210822302000F04CFA31
:10671800012000F069FC02210122302000F044FA37
:10672800012000F061FC00210A46302000F03CFA0C
:10673800012000F059FC1B21CD22302000F034FA52
:10674800012000F051FC04210322302000F02CFA33
:10675800012000F049FC06210822302000F024FA2C
:10676800012000F041FC07210A46302000F01CFA05
:10677800012000F039FC08218022302000F014FAB2
:10678800012000F031FC1E21B022302000F00CFA6C
:10679800012000F029FC05219122302000F004FAA4
:1067A800012000F021FC0D210322302000F0FCF92B
:1067B800012000F019FC0E210022302000F0F4F92D
:1067C800012000F011FC14218022302000F0ECF9A7
:1067D800012000F009FC0B218822302000F0E4F9A8
:1067E800012000F001FC30200C21822200F0DCF9AD
:1067F800012000F0F9FB12218822302000F0D4F9A2
:10680800012000F0F1FB13218C22302000F0CCF99C
:10681800012000F0E9FB00210122302000F0C4F93A
:10682800012000F0E1FB0C210822302000F0BCF927
:10683800012000F0D9FB0D210822302000F0B4F926
:10684800012000F0D1FB0E210822302000F0ACF925
:10685800012000F0C9FB0F210822302000F0A4F924
:10686800012000F0C1FB00210A46302000F09CF90D
:10687800012000F0B9FB40210222302000F094F9F9
:10688800012000F0B1FB00224121302000F08CF9FA
:10689800012000F0A9FB30203F21D42200F084F928
:1068A800012000F0A1FB00210122302000F07CF93A
:1068B800012000F099FB10210F22302000F074F91C
:1068C800012000F091FB11210F22302000F06CF91B
:1068D800012000F089FB12210022302000F064F929
:1068E800012000F081FB13210022302000F05CF928
:1068F800012000F079FB09213C22302000F054F9F6
:10690800012000F071FB00210122302000F04CF939
:10691800012000F069FB30203421024600F044F9E0
:10692800012000F061FB30203721024600F03CF9DD
:10693800012000F059FB36210322302000F034F901
:10694800012000F051FB39210322302000F02CF9FE
:10695800012000F049FB3B213C22302000F024F9C3
:10696800012000F041FB3C210A46302000F01CF9D0
:10697800012000F039FB00210A46302000F014F90C
:10698800012000F031FB5121C022302000F00CF929
:10699800012000F029FB30205221002200F004F9E8
:1069A8000120BDE8084000F01FBB00BF2DE9F04FF3
:1069B800454E464D93B001214FF4001006F0B4FD4A
:1069C800304605F057FD4FF0C0630293404B0393E8
:1069D800404B002404934FF400794FF400334FF4F4
:1069E80080684FF400674FF4005A4FF4807B3046BC
:1069F80002A90C9301930997CDF818900594079470
:106A0800CDF82080CDF828A0CDF82CB00D9405F055
:106A1800BDFD22463046304905F013FE30460121BF
:106A280005F019FE01210A464FF0402006F0EAFF62
:106A3800284605F01FFD294A019B0392284A0C931A
:106A480004922846402202A9059209970294CDF89B
:106A580018900794CDF82080CDF828A0CDF82CB058
:106A68000D9405F093FD224628461E4905F0E9FDE0
:106A78002846012105F0EFFD42F21077012202219C
:106A8800194806F0BFFF384600F0AEFA304601213B
:106A980005F0B7FD0121284605F0B3FD384600F0A2
:106AA800A3FA0B238DF8443011A801238DF8454033
:106AB8008DF846408DF8473000F01AFD384600F052
:106AC80093FA13B0BDE8F08F10600240886002406E
:106AD8000C400040E6390020E63100200C3C004024
:106AE800E6350020E62D0020003C00400248102139
:106AF800012205F0FDBD00BF1060024013B5022061
:106B0800012106F011FD4FF410730E4C009302237F
:106B18008DF804308DF8053001238DF806302046B5
:106B2800002369468DF8073006F056F920460621FD
:106B3800042206F0D1F920460921042206F0CCF9F6
:106B48001CBD00BF0004024030B5154D85B00121C1
:106B58004FF4001006F00CFD284606F0D3F9002388
:106B6800ADF804304BF6FF73ADF806303323ADF8BB
:106B780008304FF48063ADF80A304FF48043ADF825
:106B88000C3004AC074B2846012144F8103D06F0B0
:106B98005BFA2846694606F0E3F905B030BD00BF48
:106BA80000540040801A060073B54FF49613064649
:106BB8000D461446019304E0019B5A1E0192002BD6
:106BC80057D031484FF4003106F056FB0028F3D176
:106BD8002D48012106F044FA4FF48053019304E054
:106BE800019B5A1E0192002B45D02748274906F0E1
:106BF8002EFB0028F4D024483146002206F048FA3B
:106C08004FF48053019304E0019B5A1E0192002B1C
:106C180033D01D481E4906F01AFB0028F4D01A4844
:106C2800294606F0B8FA4FF48053019303E0019B1C
:106C38005A1E01921BB31448164906F008FB002897
:106C4800F5D01148214606F0A6FA4FF496130193A1
:106C580003E0019B5A1E01929BB10B480E4906F0B6
:106C68000BFB0028F5D00848012106F005FA0020A2
:106C780008E0012006E0022004E0032002E00420EE
:106C880000E005207CBD00BF005400400100030067
:106C980082000700800007000400001037B54FF499
:106CA800961304460D46019305E0019B5A1E019276
:106CB800002B00F09B8056484FF4003106F0DCFAB8
:106CC8000028F2D15248012106F0CAF94FF4805346
:106CD800019305E0019B5A1E0192002B00F0888069
:106CE8004B484C4906F0B3FA0028F3D048482146EF
:106CF800002206F0CDF94FF48053019304E0019B84
:106D08005A1E0192002B75D04148434906F09FFA5C
:106D18000028F4D03E48294606F03DFA4FF4805347
:106D2800019304E0019B5A1E0192002B64D038485D
:106D38003A4906F0A1FA0028F4D03548012106F0B6
:106D48008FF94FF48053019304E0019B5A1E01927E
:106D5800002B53D02E482F4906F079FA0028F4D09A
:106D68002B482146012206F093F94FF480530193F2
:106D780004E0019B5A1E0192002B41D0244C284963
:106D8800204606F079FA0028F3D02046002106F0C4
:106D980087F920460121238B06F06EF94FF48053C2
:106DA800019304E0019B5A1E0192002B2AD0184837
:106DB8001C4906F061FA0028F4D0154806F0EDF9F0
:106DC8004FF480530193124A03E0019B591E01912D
:106DD800D3B113889B05F8D4012104460C4806F06A
:106DE8005FF90B48104906F061FA0EE001240CE047
:106DF80002240AE0032408E0042406E0052404E051
:106E0800062402E0072400E0082420463EBD00BF17
:106E18000054004001000300820007000400001035
:106E280002000010400000100004001013B54FF4D9
:106E380096130446019305E0019B5A1E0192002B0C
:106E480000F0B08061484FF4003106F015FA0028D0
:106E5800F2D15E48012106F003F94FF48053019303
:106E680005E0019B5A1E0192002B00F09D805748B7
:106E7800574906F0ECF90028F3D05448A021002225
:106E880006F006F94FF48053019305E0019B5A1E62
:106E98000192002B00F08A804C484E4906F0D7F941
:106EA8000028F3D0C4F30521484806F074F94FF4DC
:106EB8008053019304E0019B5A1E0192002B77D066
:106EC8004248454906F0D8F90028F4D0E1B23F48D5
:106ED80006F061F94FF48053019304E0019B5A1EB8
:106EE8000192002B66D039483B4906F0C5F90028C5
:106EF800F4D03648012106F0B3F84FF480530193DB
:106F080004E0019B5A1E0192002B55D02F483049AE
:106F180006F09DF90028F4D02C48A121012206F0A2
:106F2800B7F84FF48053019304E0019B5A1E019275
:106F3800002B43D0254C2949204606F09DF900280E
:106F4800F3D02046002106F0ABF820460121238B20
:106F580006F092F84FF48053019304E0019B5A1E07
:106F68000192002B2CD019481D4906F085F90028FC
:106F7800F4D0164806F011F94FF480530193134AE0
:106F880003E0019B591E0191E3B113889905F8D4D8
:106F9800012104460D4806F083F80C48114906F013
:106FA80085F910E001240EE002240CE003240AE035
:106FB800042408E0052406E0062404E0072402E08F
:106FC800082400E0092420461CBD00BF00540040EE
:106FD80001000300820007000400001002000010F6
:106FE800400000100004001082B0002304E0019B60
:106FF80001330193009B01330093009B8342F6D336
:1070080002B0704737B54FF4805304460D460193DC
:1070180004E0019B5A1E0192002B6ED03D484FF4AC
:10702800003106F029F90028F3D13A48012106F089
:1070380017F84FF48053019304E0019B5A1E019204
:10704800002B5CD03348344906F001F90028F4D00D
:107058003048A021002206F01BF84FF4805301931A
:1070680004E0019B5A1E0192002B4AD029482B4963
:1070780006F0EDF80028F4D0C4F30521254806F001
:107088008AF84FF48053019304E0019B5A1E019241
:10709800002B38D01F48224906F0D9F80028F4D030
:1070A800E1B21C4806F077F84FF48053019303E0EF
:1070B800019B5A1E019243B31648194906F0C7F8B6
:1070C8000028F5D01348294606F065F84FF49613C2
:1070D800019303E0019B5A1E0192C3B10D48114967
:1070E80006F0CAF80028F5D00A48012105F0C4FFC7
:1070F8000D48FFF779FF00200AE0012008E0022090
:1071080006E0032004E0042002E0052000E0062059
:107118003EBD00BF0054004001000300820007008C
:107128008000070004000010A0860100F7B54FF4A6
:10713800805304460D461646019304E0019B5A1EEF
:107148000192002B75D041484FF4003106F094F8B5
:107158000028F3D13D48012105F082FF4FF4805308
:10716800019304E0019B5A1E0192002B63D037481B
:10717800374906F06CF80028F4D03448A0210022E2
:1071880005F086FF4FF48053019304E0019B5A1EDB
:107198000192002B51D02D482E4906F058F80028AE
:1071A800F4D0C4F30521294805F0F5FF4FF48053C6
:1071B800019304E0019B5A1E0192002B3FD0234803
:1071C800254906F044F80028F4D0E1B21F4805F03C
:1071D800E2FF4FF48053019304E0019B5A1E019291
:1071E800002B2ED019481C4906F031F80028F4D09D
:1071F80000244FF4961710E0295D144805F0CBFFE2
:10720800019703E0019B5A1E0192E3B10F4813490D
:1072180006F032F80028F5D00134E3B2B342EBD3DC
:107228000A48012105F028FF0D48FFF7DDFE002080
:107238000AE0012008E0022006E0032004E0042020
:1072480002E0052000E00620FEBD00BF005400401B
:1072580001000300820007008000070004000010FE
:10726800A086010013B50520012106F05DF9184C30
:107278004FF4E053009302238DF804308DF8053065
:107288002046002369468DF806308DF8073005F052
:10729800A3FD20460A21062205F01EFE20460C21E9
:1072A800062205F019FE062220460B21A4F50064EB
:1072B80005F012FE4FF4004320466946009305F09E
:1072C8008BFD20460F21062205F006FE1CBD00BFDF
:1072D800000802401FB50446FFF7CEF9FFF734FC5B
:1072E800FFF7F6F9FFF7BEFF01214FF4004006F063
:1072F8003FF902940F4C1023ADF8023020460023CA
:107308006946ADF80430ADF80C30ADF80030ADF892
:10731800063006F05CFA69464FF0402006F02BFB79
:107328002046012106F0DBFA4FF04020012106F04B
:10733800D6FA1FBD003C0040014B1860704700BFE3
:10734800FC0D0020704710B50A4A1379262B04D883
:107358000949C8540133137110BD074A0123591E46
:10736800D45C0133272B5454F9D1034B83F82600FE
:1073780010BD00BFFC0D0020E83D0020704710B58F
:1073880004462078FFF7DFFF14F8013F002BF8D1FF
:1073980010BD38B504460D46013D14F8010BEDB299
:1073A800FFF7D1FF002DF7D138BD00BF014B18788A
:1073B800704700BF040E0020014B5878704700BF8B
:1073C800040E0020024B187880F00100704700BFBF
:1073D800040E0020024B00221A705A70704700BF3A
:1073E800040E0020014B01221A707047040E002081
:1073F800014B01225A707047040E002082B000230E
:1074080004E0019B01330193009B01330093009B2F
:107418008342F6D302B0704707B50420012106F075
:1074280083F801214FF4804006F0AEF84FF4007362
:10743800009300238DF804300348012369468DF832
:10744800073005F0C9FC0EBD000802400D4B07B51A
:107458001A680D484FF47A73B2FBF3F20B4B013AFA
:107468005A600B4AF02182F8231000229A60072202
:107478001A60084B084A00930121084B04F0DAF916
:107488000EBD00BFF0020020B43E002010E000E076
:1074980000ED00E00C040020F00300205803002059
:1074A800054B1A6812B11A68013A1A60034B1A6838
:1074B80001321A60704700BF703E0020883E0020ED
:1074C80082B0044B0190019A1A601A68002AFCD114
:1074D80002B07047703E0020704700BF40F0BE60A9
:1074E800024B40F42020D860704700BF00ED00E058
:1074F800C37810B503B3164B4278DB688478DB4356
:10750800C3F30223C3F10401C9B202FA01F10F2245
:1075180042FA03F2C9B222400A430E4B0178120123
:10752800CB18D2B283F8002303780122590903F05B
:107538001F0302FA03F307E003780122590903F055
:107548001F0302FA03F32031024A42F8213010BD2A
:1075580000ED00E000E100E021F0604121F07F0152
:10756800014B08439860704700ED00E0044B1A692E
:1075780009B1104301E022EA00001861704700BF1A
:1075880000ED00E0044B1A6804280CBF42F0040226
:1075980022F004021A60704710E000E000000000CA
:1075A800034A044B1A60044A044B1A60704700BF30
:1075B8000000FA45B81A0020DB0FC93FB41A0020B2
:1075C800034B00221A60034A034B1A60E8E700BF26
:1075D800D84400200000FA45B019002007EE100A30
:1075E800024BF8EEC77AC3ED007A7047B019002055
:1075F80038B510EE100A07F049FB0DA3D3E90023B4
:1076080007F098FB084B044618680D4607F03EFB48
:107618000B4602462946204607F0B6FC07F06CFEEA
:10762800024B186038BD00BFB81A0020B41A0020F9
:10763800182D4454FB2119402DE9F04F2DED068BF0
:107648008F4CDFF870A289B00027A34637F80A509C
:107658008C4B2580FE5A8C4B6680186807F016FB09
:1076680081A3D3E9002307F065FB07F0FDFD6368FC
:10767800864AC018011101F580610905090D60608D
:10768800C0F30B100DF1200C32F8203032F8212015
:10769800616A238115FB02F0628115FB03F516FB75
:1076A80002F216FB03F60CEB4103E0602561C0F320
:1076B800CF30C5F3CF356261A661C2F3CF32C6F3CE
:1076C800CF3623F8200C23F8105C23F8182C23F865
:1076D800086C6F4BA08301310B40002BE58322849B
:1076E800668403DA013B63F003030133CBF82430EB
:1076F800002B40F0AD806748674A6946042308F0CC
:107708001DFE6648664A04A9042308F017FE65486A
:10771800654A02A9042308F011FE644A644806A9D0
:10772800042308F00BFEB4F9283007EE903AB4F9B8
:107738002A30B8EEE79A07EE903AB4F92C30B8EE52
:10774800E78A07EE903AB4F92E30F8EEE79A07EE9A
:10775800903AF8EEE78A68EE087A49EE097A17EE69
:10776800900A07F093FA41EC100B09F049FC51EC30
:10777800100B07F0C1FD68EEA87A49EEA97A0AEE67
:10778800100A206317EE900A07F080FA41EC100BFC
:1077980009F036FC51EC100B07F0AEFD68EE897A63
:1077A80058EE297A28EE288A0AEE900A606309EED4
:1077B800298A17EE900A07F069FA804618EE100A2F
:1077C800894607F063FA49EC108B41EC110B09F07C
:1077D8008FFB8AEE2A8A51EC100B07F08DFD84EDA1
:1077E8000F8AA06307F052FA21A3D3E9002307F018
:1077F800A1FA8046206C894607F048FA1EA3D3E90F
:10780800002307F097FA02460B464046494607F020
:10781800DFF807F071FD206418EE100A07F036FA59
:1078280013A3D3E9002307F085FA8046606C8946E4
:1078380007F02CFA10A3D3E9002307F07BFA0246DD
:107848000B464046494607F0C3F807F055FD60640B
:107858000237B7F5007F7FF4F9AE09B0BDEC068BAF
:10786800BDE8F08FAFF3008039D6C56D305FC440F6
:107878009A9999999999C93F9A9999999999E93FA2
:10788800180E0020041C0020B41A0020BC5A04085A
:107898000300008008020020400E0020FC010020A8
:1078A800420E0020F0010020440E0020460E002069
:1078B800E4010020CA230020014B93ED0F0A704712
:1078C800180E0020014B93ED0E0A7047180E002089
:1078D800014B93ED110A7047180E0020014B93EDF0
:1078E800100A7047180E0020014B93ED0C0A7047E0
:1078F800180E0020014B93ED0D0A7047180E00205A
:1079080010B5FEF7B7F80020012324210246FEF740
:107918001BF9114B1C780020012C05D10146FEF7FC
:10792800ECF92046002104E00721FEF7E6F90120E2
:107938000721FEF7E2F963221221C020FFF734F98C
:1079480002200121FEF7D9F9FEF7B6FA0120BDE8B9
:107958001040FEF7A6BA00BF380F00200D4B1B7869
:10796800012B05D10C4B0D4A196812688A181A6048
:107978000B4B1B78012B084B196805D1094A91421A
:1079880007DD01321A607047074A914201DD013272
:107998001A607047483E0020AC440020443E002056
:1079A800380F00207FD1F008FF1FA1070E4B1B786E
:1079B800012B05D10D4B0E4A196812688A1A1A60F4
:1079C8000C4B1B78012B094B05D10B4A19689142C6
:1079D80008DC1A6070471A68B2F57A2FDCBF4FF4DA
:1079E8007A221A60704700BF483E0020AC4400204D
:1079F800443E0020380F002040420F00024B1A6816
:107A0800024B1A60704700BFA83E0020AC4400201B
:107A18002DE9F04F824658488BB0B0FBF1F00C4688
:107A280007F012F941EC100B09F05EF951EC100B5C
:107A380007F042FCC307074648BF471E04FB07F090
:107A480007F002F946A3D3E9002307F09DFA04469C
:107A58000D4645EC104B09F047F959EC108B2046C0
:107A680042464B46294606F0B1FFCDE90401494696
:107A7800404607F021FC3CA3D3E900230990DDE947
:107A8800040107F0D3FB00283DD1002401234FF067
:107A98001509224698462046DFF8E4B003E023465D
:107AA80042462C46B04600FB04355D452ED800FB07
:107AB8000826DDE904012EA3D3E9002307F0B6FB6D
:107AC80030BBDDE9042300202C4907F05DFA41ECC6
:107AD800100B0390029109F007F90398029953ECEF
:107AE800102B8DED060B06F071FF09F1FF39CDE97A
:107AF80004015FFA89F9DDE9060107F0DDFBB9F158
:107B0800000FCCD104E00125002601E025464646B9
:107B1800099BD9B2BAF1000F0BD132462B46504619
:107B2800FEF712F801230093504651463A46534651
:107B380009E032462B460120FEF706F801200090A6
:107B480001463A460023FEF7F2F8FEF7B5F90120A0
:107B58000BB0BDE8F04FFEF7A4B900BFAFF300804B
:107B68000000000084D77741956479E17FFDA53D49
:107B7800BBBDD7D9DF7CDB3D00E9A4350000F03F71
:107B8800FFFF0F0038B52A4B1B78022B294B03D176
:107B9800294A12681A6038BD1968284B284A1B6898
:107BA800284CCB189342236018DC0020FFF730FFE5
:107BB80001202168FFF72CFF234B1C780020012CA3
:107BC80005D10146FEF799F82046002104E0072177
:107BD800FEF793F801200721FEF78FF81B4B1B785F
:107BE800022B14D11A4B1B4D1A68124C2B68D31850
:107BF80022689A420BDA184B1B78012B07D1174BD6
:107C0800186800F081F822682B68D3182360084BA5
:107C18001A78012A0AD10E4A11680E4A12688A187F
:107C280004490968914201DB02221A7038BD00BF7D
:107C380024460020AC440020A83E0020C444002074
:107C480080D1F008C8440020380F0020483E0020AA
:107C5800983E0020443E0020903E0020603E0020D8
:107C680008B5FEF79BFC094B5A78187002435A7006
:107C78001AB19A7801329A7030B99B78034A012B6D
:107C880002D900235370937008BD00BF600E002016
:107C980007B50420012105F047FC4FF46043009329
:107CA80001238DF8043002238DF8053004480023A1
:107CB80069468DF806308DF8073005F08DF80EBD51
:107CC80000080240084B1A684FF47A73B2FBF3F2CB
:107CD800064B013A5A60064AF02182F82310002226
:107CE8009A6007221A607047F002002010E000E056
:107CF80000ED00E0034B5A6812B15A68013A5A6025
:107D0800704700BF600E0020024B58605A68002A76
:107D1800FCD17047600E002030B585B004460D4692
:107D280001A85C490A220BF0FBFB5B4B1B78032B79
:107D380010D8DFE803F00205080B01A8574907E04F
:107D480001A8574904E001A8564901E0564901A88D
:107D58000BF0D0FC04AA131913F80C3C5D19EDB212
:107D68002F2D01D80A3502E0392D01D90A3DEDB28F
:107D780004AB1C194FF6FF7004F80C5CFCF7DEFD31
:107D88000020FCF7D1FE0DF103050F242046233413
:107D98005A21002315F8012FA4B2FCF7DFFEB4F531
:107DA800A57FF3D164205A212C220023FCF7D6FEAC
:107DB8000023CD205A212C22FCF7D0FE0020FCF70E
:107DC800BDFD354B1B78032B62D8DFE803F0022892
:107DD8004B5601A931480BF08DFC0A2200212F488F
:107DE8000BF02CFE314A324B12781860012A06D16A
:107DF800304A904201DC01321A602F4A06E0B0F5A1
:107E0800FA5FBCBF4FF4FA521A602C4A1B689342BF
:107E1800C4BF274B1A602A4B1A682A4B20E001A9D5
:107E28001F480BF067FC0A2200211D480BF006FED4
:107E38001E4A254B12781860012A06D11D4A904225
:107E480001DC01321A601C4A06E0B0F5FA5FBCBFDB
:107E58004FF4FA521A60194A1B68934218DD1A4BFC
:107E68001A6015E001A90F480BF044FC0D480021E9
:107E78000A220BF0E3FD154B09E001A90A480BF0B3
:107E880039FC094800210A220BF0D8FD104B186074
:107E980005B030BDDB9E0508A63E0020743E0020DC
:107EA8009C3E0020B1440020643E0020380F002092
:107EB800B03E00203F420F0080D1F00840420F0042
:107EC800A83E0020AC440020CC440020A44400205C
:107ED800603E002010B50D4B0D4C1A680D48214628
:107EE8000BF0E0FB0C4B0D481A6821460BF0DAFB4F
:107EF8000B4B0C481A6821460BF0D4FB0A4B0B4875
:107F08001A682146BDE810400BF0CCBBB03E0020FB
:107F1800E59E0508743E0020CC4400209C3E0020CD
:107F2800A4440020B1440020603E0020643E0020AC
:107F38009FED010A704700BF000000009FED010A95
:107F4800704700BF000000009FED010A704700BFA6
:107F58000000000070477047044B18B1012801D198
:107F6800034A00E0034A12681A607047AC440020D4
:107F7800983E0020A83E002010B9034B18687047AF
:107F8800024B1868704700BFB03E0020A83E002092
:107F980010B9034B18687047024B1868704700BF48
:107FA800CC440020983E002008B54FF49570FEF7A9
:107FB8002BFA40F26523C31A584240EB030008BD70
:107FC80008B5C620FEF720FA40F28D13C21A5042B7
:107FD80040EB020008BD4FF4957040F26521FEF7B2
:107FE80005BAC62040F28D11FEF700BA704760EE60
:107FF800A00AB7EE007AF0EE606A70EE077A40EEFB
:10800800006A47EEA70A36EEC77A08B5C7EE200A17
:1080180010EE900A06F03AFE0022084B06F08AFE9F
:108028000022074B06F0D4FC07F066F907EE900A29
:10803800FDEEE77A17EE900A9F3008BD0000594020
:108048000000E03F38B52DED028BF7EE008AB0EE68
:10805800608A70EE288A10EE900A28EE088A06F0E8
:1080680015FE08EEA88A00220F4B06F063FE0446B0
:1080780018EE100A0D4606F009FE02460B46204689
:10808800294606F081FF0022084B06F0A1FC07F004
:1080980033F907EE900AFDEEE77A17EE900A77308B
:1080A800BDEC028B38BD00BF000069400000E03F16
:1080B800F0B5694D2DED068B95E80F008DB008AE33
:1080C800103586E80F000FCD01AC0FC495E8070006
:1080D8004FF6FF7384E807009F2077216422FAF7A0
:1080E800BCFAA020772164224FF6FF73FAF7B5FA9D
:1080F8009E20772164224FF6FF73FAF7AEFA9F208D
:10810800762164224FF6FF73FAF7A7FA4FF6FF734A
:10811800782164229F20FAF7A0FA0020FCF76AFA77
:108128009F2077216522FCF73FFC9F20772164225E
:10813800FCF73AFC07AD0C36F7EE009A0435F7EE7B
:10814800008A95ED009A4FF49674B0EE68AA18EE7E
:10815800900A06F09BFD3EA3D3E9002306F0EAFD52
:1081680007F0CAF808EE900A38EEE98AB0EE490A34
:10817800F0EE480AFFF73BFFB0EE490AF0EE480A76
:108188000746FFF75FFFBFB281B20F223846FCF700
:108198003EF9013CDBD14FF49674F7EE008A18EEF5
:1081A800900A06F073FD2AA3D3E9002306F0C2FD66
:1081B80007F0A2F808EE900A39EEE88AB0EE490A0C
:1081C800F0EE480AFFF713FFB0EE490AF0EE480A4E
:1081D8000746FFF737FFBFB281B20F223846FCF7D8
:1081E80016F9013CDBD1B542A8D16C4607AE043480
:1081F80094ED009A4FF4C875F7EE008A18EE900ACD
:1082080006F044FD12A3D3E9002306F093FD07F01E
:1082180073F808EE900A38EECA8AF0EE490AB0EE12
:10822800480AFFF7E4FEB0EE480AF0EE490A0746AE
:10823800FFF708FFBFB281B200223846FCF7E7F823
:10824800013DDBD1B442D2D10DB0BDEC068BF0BDFF
:10825800295C8FC2F528F03FBC9A0408121A06EE72
:10826800902A081AB8EEE67A06EE900AF8EEE67A50
:10827800C7EE277A9FED047A67EE877AFDEEE77AF4
:1082880017EE900A704700BF0000A0438A1A06EE56
:10829800902A081AB8EEE67A06EE900AF8EEE67A20
:1082A800C7EE277A9FED047A67EE877AFDEEE77AC4
:1082B80017EE900A704700BF0000484370B50646A5
:1082C8000D460024610704D5A0B231462A46FCF7C2
:1082D8009EF80134B4F5A07FF4D170BD70B50646A0
:1082E8000D460024600704D5A1B230462A46FCF7A3
:1082F8008EF80134C82CF5D170BD114B11481B788C
:108308001149124A0068012B114B09D11268086003
:108318001A60104B1A68104B1A60104B1A680CE060
:108328001268D2011A600B4B1A680B4BD2011A6003
:108338000A4B1A68C0010860D201094B1A607047DD
:10834800380F0020B03E0020A83E0020CC4400207A
:10835800983E0020A4440020443E0020803E002097
:10836800C4440020024B1A68024B1A60704700BFD1
:10837800A83E0020AC44002008B5FFF7BEFFBDE8CA
:108388000840EFE770B500210A222748274D284EFC
:10839800284C0BF053FB00210A22286026480BF0DA
:1083A8004DFB00210A22306024480BF047FB0021D6
:1083B8000A22206022480BF041FB224B32681860E9
:1083C8002B68D31A06EE903A23681F4AB8EEE67A6D
:1083D80006EE903AF8EEE67AC7EE277AFCEEE77AF0
:1083E80017EE903A01339BB207EE903AB8EE677AEF
:1083F800F4EE007A67EE277A1380FCEEE76A134BF7
:1084080016EE901A8AB206EE902AB8EEE67A19802D
:1084180077EEC77AF5EEC07AF1EE10FA01DD013297
:108428001A80BDE87040A7E7743E0020B03E0020E7
:10843800CC440020A44400209C3E0020B1440020ED
:10844800643E0020603E0020EC4700206C4800207D
:108458000022F0B51346202603254FF02C0C00E02F
:108468002646303EF6B217460132092E10F8014B67
:108478000AD897FBF5F605FB16772FB9CE1801F841
:1084880003C07470023301E0CC540133092AE7D1E8
:108498002022CA54CB1848225A707A229A70002295
:1084A800DA70F0BDF0B51F46144B1E788DB0054646
:1084B8000C4606B3A6F1040CDCF1000646EB0C06EC
:1084C800CEB90F4908A80BF0EDF808A86946FFF7E0
:1084D800BFFF0C496A4604A80BF0E4F8BDF8480051
:1084E800FCF72CFA3846FCF73FFA2846214604AA3E
:1084F8003346FCF751FB0DB0F0BD00BF483E0020ED
:10850800BC950508BE9C05082DE9F04F7C4B2DED68
:10851800068B93ED008A78EE087A7A4B85B017EED1
:10852800900A1C6806F0B2FB80462046894606F091
:10853800ADFB68EE088A41EC100BF7EE009ACDE926
:10854800020108F079FB78EEA97A57EC106B17EE68
:10855800900A06F09BFB32463B4682468B464046D5
:10856800494606F0E7FB02460B465046594606F0D8
:108578002DFA06F0C1FE79EEE88A09EE100AC8EE77
:10858800898ADFED617A9DED020B68EEA78A08F013
:1085980053FC404653EC102B494606F0CBFB0646ED
:1085A80019EE100A0F4606F071FB02460B463046DC
:1085B800394606F0E9FC554B002206F0BBFB06F0F5
:1085C8009BFE09EE100A69EE097A48EEA87AB1EE28
:1085D80049AA88EEA77A4E4B5C60D8608AEE27AA33
:1085E80083ED008AC3ED028A83ED047A83ED05AA40
:1085F800484B1B78033B042B6ED8DFE803F00312CB
:10860800254E3C0018EE900A06F040FB044619EE91
:10861800100A0D4606F03AFBCDE900013E483F49F5
:108628000DE017EE100A06F031FB04461AEE100AA8
:108638000D4606F02BFBCDE90001374838492246A4
:108648002B460BF02FF847E018EE100A06F01EFB39
:1086580041EC100B08F04EFC0022324B51EC100B91
:1086680006F068FB06F048FE06F010FB02460B46D3
:1086780029482D492EE018EE100A06F007FB1CA326
:10868800D3E9002304460D46DDE9020106F052FB5A
:10869800CDE9000120482549D1E718EE100A06F077
:1086A800F5FA15A3D3E9002306F0D4FDDFED207A0F
:1086B800002818BFB0EE678A78EE297A79EEC89A52
:1086C800C7EEA99A19EE900A06F0E0FA02460B46A0
:1086D800114818490AF0E6FF0F4A0220CA21002370
:1086E80005B0BDEC068BBDE8F04FFCF755BA00BFEE
:1086F800F6285C8FC2A54C40AE47E17A14AEEF3F36
:108708000C45002010450020000048420000494068
:10871800CC470020C0440020E2440020EB9E05081E
:10872800FB9E0508000034C00B9F05081D9F050827
:10873800A4707D3F399F05082DE9F0434FF47F7001
:108748008DB0FDF761FE00271FFA80F86BE04FEA55
:10875800C7091FFA89F909F580691FFA89F0FEF738
:1087680065FB60F3070409F1010080B2FEF75EFBC8
:1087780060F30F2409F1020080B2FEF757FB60F3A3
:10878800174409F1030080B2FEF750FB60F31F6441
:1087980009F1040080B2FEF749FB60F3070609F10E
:1087A800050080B2FEF742FB60F30F2609F10600D0
:1087B80080B2FEF73BFB09F1070960F307051FFAD2
:1087C80089F0FEF733FB60F30F25B0B206F04CFAE0
:1087D80000221B4B06F0AEFA06F08EFD06F056FAA4
:1087E800CDE90001A8B206F03FFA11A3D3E90023AE
:1087F80006F0ECF810A3D3E9002306F0C5FB06F059
:108808007BFD06F043FA2246CDE902010D4905A891
:108818000AF048FFC1B205A802F0B6FE0120FFF732
:1088280073FA0137BFB2B84591DA0DB0BDE8F083ED
:1088380000000000C0FFDF40E17A14AE47C1664087
:108848000000F03E449F050808B50021C620FDF74A
:10885800CDFD4FF495700021BDE80840FDF7C6BD79
:10886800024B4FF6FF721A80704700BFE0440020A9
:1088780000200146C82240F23F13FBF722BF07B58C
:108888000DF1070002F081FE9DF807000EBD08B546
:10889800FFF7F5FF0028FBD108BD30B5044687B0C7
:1088A80010EE100A0D4606F0F1F902460B4601A833
:1088B80005490AF0F7FE2046294601AA0023FCF7DD
:1088C8006BF907B030BD00BF579F050808B50848C9
:1088D80003F0E4FC0648022103F0B1FD0028F9D0BA
:1088E800034803F007FD07EE900AB8EE670A08BDD3
:1088F8000020014010B50C4C00232DED028B238085
:108908009FED0A8A06E0FFF7E1FF238838EE008A28
:10891800013323802388182BF5D99FED050A28EE0B
:10892800000ABDEC028B10BD143E002000000000C0
:10893800ACC8683910B54FF4C770FDF765FDDB2882
:1089480005D14FF4C870FDF75FFD84B219E041F21C
:10895800E104214644F20100FDF748FD44F201001C
:10896800FDF752FDA04214BF80244FF4007421B2D9
:108978004FF4C870FDF73AFD4FF4C770DB21FDF7DF
:1089880035FD204610BD024B00221A70704700BF0B
:108998000C480020014B01221A7070470C48002037
:1089A800014B00221A60704708450020014B1878D7
:1089B800704700BF0C4800200030024B18BF012050
:1089C800187070470D4800200E4B1A680E4B1A603D
:1089D8000E4A002313700E4A13700E4A01211170BB
:1089E8000D4A4FF6FF7010800C4A13700C4B1A7822
:1089F8000C4B002A14BF052204224FF080401A7045
:108A080005F0F3B9A83E0020AC440020903E0020B9
:108A18000C4800200A0E0020E044002024460020D4
:108A2800140E0020150E002070EEA10A88B030EE5A
:108A3800010A08B0704770EEE10A88B030EE410ACA
:108A480008B07047F0EE407A20EEA10A60EE810A85
:108A580047EEA10A88B017EE810A08B07047D0B572
:108A680061EEA17A41EE017A2DED048B17EE900AA2
:108A780088B0B0EE409AF0EE609AF0EE418AB0EE1F
:108A8800618A06F003F90022002306460F4606F025
:108A9800B9FBE8B969EE887A49EE287A29EE088A9E
:108AA80017EE900A06F0F2F832463B4606F06CFAEA
:108AB80019EEA88A06F020FC044618EE100A06F003
:108AC800E5F832463B4606F05FFA06F015FC01E091
:108AD8000448044600EE900A00EE104A08B0BDECC7
:108AE800048BD0BD0050C347F0EE407A86B020EE2C
:108AF800200A67EE810A06B07047064B93E8030028
:108B080084B004AB03E90300DDED030A9DED020A1E
:108B180004B0704770480020F7EE007A77EEC07A0C
:108B280020EE022A20EE210A07EEA00AF0EE420A01
:108B380047EE810A88B008B0704770B56D4B2DEDCF
:108B4800068B1A786C4B94B00E468DED020ACDED6B
:108B5800030A22B91A68802392FBF3F200E01A682C
:108B6800664C012E236C616CDFED659AB7EE00AAA6
:108B780051D002D3022E60D154E0D21A07EE102A47
:108B8800CB1AB8EEC79A07EE103AF8EEC77AD4EDCA
:108B9800000A89EE279A94ED011AD4ED021A94ED91
:108BA800032AB0EE490AFFF7B7FF8DED000ACDEDB5
:108BB800010A9DE8030006ABD4ED040A94ED051AFA
:108BC800D4ED061A94ED072A83E80300B0EE490AAB
:108BD800FFF7A2FF8DED000ACDED010A9DE8030025
:108BE80008AB83E80300D4ED0C0A94ED0D1AD4ED1C
:108BF8000E1A94ED0F2AB0EE490AFFF78DFF8DED9E
:108C0800000ACDED010ADDED068A9DED078A04AB69
:108C18009DE803000EE0D4ED008A94ED018A08ABCC
:108C2800103405E0D4ED028A94ED038A08AB1834B9
:108C380094E8030083E8030003E0B0EE698AF0EEED
:108C48004A8ADDED030A9DED020A30EEC88A70EE0D
:108C5800688A9DED081ADDED091ACDED0C8A8DEDB7
:108C68000D8AFFF7EFFE8DED000ACDED010A9DE8B4
:108C7800030010AB83E80300DDED111A9DED101A17
:108C880079EEE11A3AEE411AB0EE680AF0EE480AB7
:108C98008DED0E1ACDED0F1AFFF7E1FE8DED000AEE
:108CA800CDED010A9DE803000AAD6C4685E8030096
:108CB8008EB99DED040ADDED050A9DED0A1ADDED7C
:108CC8000B1AFFF7BFFE8DED000ACDED010A9DE8F6
:108CD800030085E803000AAB93E8030014AB03E93B
:108CE8000300DDED130A9DED120A14B0BDEC068BEE
:108CF80070BD00BF380F0020AC4400202048002081
:108D08000000000010B5244C4FF496702168FDF760
:108D18008AFB61684FF49870FDF785FBA1684FF4F2
:108D28009A70FDF780FBE1684FF49C70FDF77BFBC0
:108D380021694FF49E70FDF776FB61694FF4A070CE
:108D4800FDF771FBA1694FF4A270FDF76CFBE169B7
:108D58004FF4A470FDF767FB216B4FF4A670FDF785
:108D680062FB616B4FF4A870FDF75DFBA16B4FF4DC
:108D7800AA70FDF758FBE16B4FF4AC70FDF753FB9D
:108D8800216C4FF4AE70FDF74EFB616C4FF4B07080
:108D9800BDE81040FDF747BB2048002010B54FF450
:108DA8009670FDF759FB224C20604FF49870FDF740
:108DB80053FB60604FF49A70FDF74EFBA0604FF4D0
:108DC8009C70FDF749FBE0604FF49E70FDF744FB93
:108DD80020614FF4A070FDF73FFB60614FF4A27073
:108DE800FDF73AFBA0614FF4A470FDF735FBE06195
:108DF8004FF4A670FDF730FB20634FF4A870FDF721
:108E08002BFB60634FF4AA70FDF726FBA0634FF4B9
:108E1800AC70FDF721FBE0634FF4AE70FDF71CFB6F
:108E280020644FF4B070FDF717FB606410BD00BFFD
:108E38002048002008B5FFF7B7F810B1BDE8084092
:108E4800ACE708BD70B500F58065A8B2FDF7EEFF88
:108E5800294C2070681C80B2FDF7E8FF6070A81CE0
:108E680080B2FDF7E3FFA070E81C80B2FDF7DEFFDB
:108E7800E070281D80B2FDF7D9FF002660F30706D1
:108E8800681D80B2FDF7D2FF60F30F26B6B207EE79
:108E9800906AB8EE677ADFED197A194B67EE277A90
:108EA800A81DC3ED007A80B2FDF7C0FF0026073584
:108EB80060F30706A8B2FDF7B9FF60F30F26B6B254
:108EC800A6F5FE46FF3E07EE106AF8EEC77A17EEE3
:108ED800900A05F0DBFE06A3D3E9002306F054F858
:108EE80006F00AFA074B22681860074B9A6170BDB2
:108EF800CDCCCCCC0C5FC440144600200000803799
:108F08000C45002010450020CC47002073B50446CE
:108F1800002862D0324B18880419A4B222B2002A61
:108F280005DB40F23F139A42C8BF1C4600E000240C
:108F38000121FBF7CBF90120FBF71CF8294E00258E
:108F4800A85B0235FBF764F8B5F5C67FF8D1A0B287
:108F58000121C7224EF29C73FBF7CEFB224D204B1A
:108F6800224A1C8012682B6824B206EE904AD21A54
:108F7800B8EEE67A06EE902AF8EEE67ADC2167EE9D
:108F8800277A9FED1B7AC7EE877A0520FDEEE77AF0
:108F980017EE904A1C194FF6FF73224600930023E0
:108FA800FFF780FA2B68E41A124B1B6894FBF3F462
:108FB80007EE104AF8EEC77AFCEEE77A17EE900A49
:108FC800C00080B2FFF73EFF0B4B0C481A780C49E3
:108FD80002B0BDE87040FFF797BA02B070BD00BF9D
:108FE800E044002026460020B03E0020CC4400206B
:108FF80000809F43A4440020C04400200C4500206A
:1090080010450020114B1B78022B13B51DD0104CB6
:109018002389ADF80630BDF806309BB253B1BDF8D0
:1090280006004EF29C7380B20121C722FBF764FB55
:1090380000232381074B1B78022B06D1064C94F999
:109048000000FFF763FF002323701CBDC04400200D
:10905800600E002024460020E42D00202DE9F04F6A
:10906800314D2DED088B2B78022BCDB009D12F4B2C
:109078001A682F4B42F210701A60FDF7B5FF00F026
:10908800FBBD2C4B1B78F7EE009ADFED2BBA002BBB
:1090980041D02A4C2068C00080B2FFF7D3FE284B8D
:1090A80028491A782848FFF72FFA284B2168D3F85F
:1090B8001880D3F8049093ED008A38EE299A79EE57
:1090C800C87AD3ED038A89EE279A002293ED04BA71
:1090D800D3ED05AA93ED02AA1D4BB4EE6B9ADA60A4
:1090E8001A6100225A61F1EE10FA1A4BC8BFB0EEAD
:1090F8006B9AB4EE699A1B88F1EE10FA48BFB0EE8D
:10910800699A994202DB02232B7022600B4B1A6882
:1091180001321A600BE2104B1A78054BF2B91A6843
:10912800802392FBF3F81BE024460020A83E002091
:10913800AC440020140E0020003C1C4608450020CA
:10914800C0440020104500200C450020CC470020DA
:10915800600E0020EC470020380F0020D3F8008074
:10916800FEF7AAFBCE4D85ED060AFEF7ABFBA86914
:1091780085ED070A10EE104A05F088FD06462046E0
:109188000F4605F083FD41EC100B41EC180B07F07E
:1091980053FD5BEC10ABB0EE480AF0EE680A07F03E
:1091A8004BFE52465B46304639468DED040B05F0C2
:1091B800C1FD06F0A1F8DFEDBB8A07EE900A9FED2E
:1091C800BA8A17EEA88AB94CDDE9042384ED008A2F
:1091D8003046394605F0AEFD06F08EF800EE900AEE
:1091E80060EEA80A0021B248B0EE480AC4ED010AB0
:1091F800FFF7A3FC8DED0E0ACDED0F0A0EAA92E83B
:109208000300AC4B83E80300D3ED018ADFEDAA7AB3
:10921800F4EE6B8AF1EE10FAC8BFF0EE678ADFED64
:10922800A77AF4EE678AF1EE10FA48BFF0EE678A83
:10923800FDEE007AF4EEE78AF1EE10FA93ED00AA5B
:1092480008DDF5EE408ADFED9E7AF1EE10FA48BFB0
:10925800F0EE678A1AEE100A05F018FD0022994B05
:1092680006460F4605F0B2FB28EEA88A044618EE1B
:10927800100A0D4605F00AFD224682468B462B460B
:109288002046294605F056FD52465B4605F0A0FBF0
:1092980041EC100B07F0B4FE002230463946894BEA
:1092A8008DED040B05F094FB02460B4605F042FDDC
:1092B80052465B4605F08CFB41EC100B07F0A0FE14
:1092C800DDE9040155EC104B06F016F8B0EE48BA8B
:1092D800294608EE100A204606F00EF807EE900A16
:1092E80088EE278A784C0AEE0ABAF1EE68AACAEE26
:1092F8008BAA8AEE0BBA18EE100A05F0C7FC62A317
:10930800D3E9002305F088FFDFED707A002818BF45
:10931800B0EE678ADFED6E7A6AEEA77AB4EE698AF4
:109328009FED6C9AF1EE10FA17EE900AC8BFB0EEF6
:10933800498A05F0ABFCDFED687A4BEE4B7A4AEED2
:10934800EA7A06460F4617EE900AC4E9026705F066
:109358009DFC47EC106B41EC110BC4E9000107F0D0
:10936800C7FD51EC100B05F0C7FFB4EE698AF1EEAA
:1093780010FAA8BFB0EE498A79EEC87A38EE299A71
:10938800564B89EE279A1B78DFED4B7AB4EE6B9A31
:10939800F1EE10FAC8BFB0EE679AB4EE699AF1EE32
:1093A80010FAF7EE007A48BFB0EE679A022B80F009
:1093B800004940F0B0804A4B1B78002B00F0AB808E
:1093C800484B494C1B681C40002C03DA013C64F0F4
:1093D80007040134082618EE100A93FBF6F605F088
:1093E80055FC0022414B05F0A5FC05F065FF05463C
:1093F800484605F04BFC26A3D3E9002305F09AFC68
:1094080025A3D3E9002305F0E3FA05F055FF384B0F
:109418002349C3F8008001EBC403C8F3072283F88B
:109428002120C8F30742B60183F8222083F824508C
:109438004FEA1862C5F3072583F82600072CC0F306
:109448000720B6B283F8208083F8232083F82550BC
:1094580083F8270008D106F5806080B220314022C9
:10946800FDF764FE00B1FEE71E4C224B22681B8804
:109478009A424CDB06F58066B0B21F494022FDF7E0
:1094880055FE0546D0B3FEE72D431CEBE2361A3FE6
:10949800CDCCCCCC0C5FC44000000000C0FFDF4046
:1094A800600E00200000F04200008C42704800204E
:1094B800204800201C460020003C1C46003C1CC6DE
:1094C800CDCC4C3D00004940F847002017B7D138B3
:1094D8000AD7233D72F97F3F17B7D139483E00209C
:1094E8000C48002008450020070000800000F040DC
:1094F80014460020EC470020800E0020B4F900102C
:109508004FF47F70FCF772FF914B25601D70914BF3
:109518001A6801321A60FEF7E7F98F4C84ED030AE6
:10952800FEF7E8F984ED040AFCF72CFF60618A4C29
:109538008A49424638A80AF0B5F8E06805F0A6FB63
:1095480002460B4628A886490AF0ACF8206905F0BF
:109558009DFB02460B462CA882490AF0A3F81BEE95
:10956800100A05F093FB82468B4652465B467E49BD
:1095780030A80AF097F81AEE900A05F087FB06461D
:109588000F4632463B46794934A80AF08BF81AEE62
:10959800100A05F07BFBCDE90A01DDE90A237449CD
:1095A80014A80AF07FF818EE900A05F06FFBCDE9D1
:1095B8000601DDE906236F4918A80AF073F818EECA
:1095C800100A05F063FBCDE90801DDE908236A49C3
:1095D8001CA80AF067F8484605F058FBCDE90401D5
:1095E800DDE90423654920A80AF05CF819EE100AA1
:1095F80005F04CFBCDE90C01DDE90C23604924A8FA
:109608000AF050F810A85F4962690AF04BF8F5EEC5
:10961800C08AF1EE10FADFED5CAA37D5404605F0B6
:1096280023FB45A3D3E9002305F084FBF1EE687A18
:10963800044617EE900A0D4605F028FB02460B4635
:109648002046294605F076FB02460B463CA1D1E9A7
:10965800000105F099FC05F04FFE9FED4C7A07EEEE
:10966800900AF4EEC77AF1EE10FAC6BFC7EEAA7AEE
:10967800474C484CF4EEEA7AF1EE10FA36DD9FEDED
:10968800427A454D454CC7EE877A32E02EA3D3E99E
:109698000023DDE9060105F04DFB044640460D4672
:1096A80005F0E2FA24A3D3E9002305F043FB0246C0
:1096B8000B462046294605F067FC05F01DFE07EE1F
:1096C800900AF4EEE97AF1EE10FA46BF67EEAA7A4C
:1096D800334C344CF4EEEA7AF1EE10FA08DD9FEDE3
:1096E8002A7A314D314CC7EE877A02E02A4D00E0E4
:1096F8002D4D17EE900A05F0C9FA2A46CDE900016A
:109708003CA82B49029409F0CDFF2A4B1B78013B5A
:10971800DBB2012B00F2A282274B1B78072B00F249
:109728009D82DFE813F04B009B02DC006301CB0154
:109738001B0271023D0200BF1F85EB51B81E194084
:10974800000000A2941A6D420000000080842E419F
:109758000C48002008450020600E0020719F050875
:109768007B9F0508869F0508919F05089B9F050814
:10977800A59F0508B09F0508BB9F0508C69F05085B
:10978800D19F0508DD9F050800007A44002474492C
:10979800629F05085F9F05088AA005086B9F05085A
:1097A800689F0508659F05084A9705086E9F050884
:1097B800EA9F0508483E0020C0440020AE4B1C78B4
:1097C800002C40F04B820220FBF7AEF94FF6FF70F9
:1097D800FBF7CAF81F20FBF7B1F81921A74A23465F
:1097E8002D20FBF7D9F94FF6FF70FBF7BDF820469F
:1097F800FBF7A4F80F20B42142464FF6FF730094FC
:10980800FEF750FE0F206E2128AA2346FBF7C4F965
:10981800A0206E212CAA2346FBF7BEF90F20382181
:109828001CAA2346FBF7B8F9A020382120AA234612
:10983800FBF7B2F90F205C2130AA2346FBF7ACF9FD
:10984800A0205C2134AA2346FBF7A6F90F204A2161
:1098580014AA2346FBF7A0F9A0204A2118AA2346F8
:10986800FBF79AF90F209B21234624AAFBF794F9CA
:10987800834B1B78012B05D10F2084213CAA23465A
:10988800FBF78AF97F4B5B69B3F57A7FCCBF4FF45E
:10989800FC604FF47840FBF767F80023A0209B2179
:1098A80010AAFBF779F9784B1B78012B08D14FF4F4
:1098B800FC60FBF759F84FF48C700221734A07E0FB
:1098C8004FF6E070FBF750F8714A4FF48C700221A4
:1098D8000023FBF761F91F20FBF746F8BEE152466B
:1098E8005B4646A86B4909F0DDFE32463B4649A86F
:1098F800694909F0D7FEDDE90A2340A8674909F05C
:10990800D1FEDDE9062343A8654909F0CBFEE62030
:10991800022146AA0023FBF73FF9E620162149AAAF
:109928000023FBF739F90220C82140AA0023FBF7DE
:1099380033F943AA00230220DC21FBF72DF9DFEDE0
:10994800597A28EE278A4FF6E07518EE100A05F0C6
:109958009DF99DED040B8B46824607F06DF957EC97
:10996800106B9DED040B07F067FA00208DED040BDA
:10997800FAF7FAFF0A214246002305200095FEF770
:1099880091FD4FF47840FAF7D9FF32463B465046EE
:10999800594605F0CFF934A3D3E9002305F018F8A8
:1099A80005F062FCDDE9042384B25946504605F00F
:1099B800C1F902460B462EA1D1E9000105F006F8CF
:1099C80005F052FC81B22046F8F777FE9D207721FA
:1099D80005220023FAF7E2FF9F20752105220123C3
:1099E800FAF7DCFF2846FAF7A9FF37E12E4B18688B
:1099F8002E4B424619689FED2E8AFEF72FFCB4EED7
:109A0800C8AAF1EE10FA044614D5B5EEC0AAF1EED4
:109A180010FA0FDDBDEECAAA4FF4FA711AEE102A39
:109A28000020FEF733FCA3B281B24FF6FF7218464E
:109A3800FAF7EDFCF4EEC88AF1EE10FA40F10E8167
:109A4800DFED1C7AF4EEE78AF1EE10FA40F30681B6
:109A5800FDEEE88A184818EE902A4FF4FA71FEF7DE
:109A680015FCA4B2CBE000BF0000000000E063409A
:109A78000000000000C05D40140E0020F79F05089C
:109A8800483E0020600E0020380F002016A0050870
:109A98001AA005081EA0050828A0050832A0050878
:109AA8003CA005080000C842B03E0020CC4400207D
:109AB8000000FA430000FAC30CFEFFFF804B186851
:109AC800804B42461968FEF7C9FBB5EEC0BAF1EE05
:109AD80010FA04461DDD504659466BA3D3E900230E
:109AE80005F09AFBA8B16AA3D3E90023504659466A
:109AF80005F020F902460B460020734904F066FF82
:109B080005F0B2FBA5B281B24FF6FF722846FAF70C
:109B18007EFC3046394660A3D3E9002305F09AFB62
:109B2800002800F09B803046394657A3D3E900232C
:109B380005F072FB002800F0918059A3D3E90023B7
:109B48003046394605F0F6F802460B4600205F49D4
:109B5800A4B204F03BFF05F087FB50E0584B1868AF
:109B6800584B42461968FEF779FB4FA3D3E9002307
:109B78000446DDE9080105F06DFB68B19DED080BB1
:109B880007F0B8F9002251EC100B514B05F0D2F850
:109B980005F06AFB014600E0C821A0B289B259E08D
:109BA800474B1868474B42461968FEF757FBDFEDED
:109BB800497A48EE677A84B2FDEEE77A204617EED6
:109BC800901A4FF6FF7289B2FAF721FC38A3D3E94D
:109BD8000023DDE9040105F0ADF837A3D3E900233C
:109BE80005F0D2F905F088FB07EE900AFDEEE77A5A
:109BF8006FF0B30017EE902AB421FEF747FB81B24D
:109C08004FF4FC62204627E0DFED337AB4EEE79AA2
:109C1800F1EE10FA22D52A4B18682A4B42461968E9
:109C2800FEF71CFB9DED0C0B044607F063F953ECA3
:109C3800102B104619460022244B05F07BF80246EB
:109C48000B460020204904F0C1FE05F00DFBA4B22C
:109C580081B220464FF6FF72FAF7D9FB1F4B1B78EB
:109C6800022B09D043B14FF6FF7300930520DC2186
:109C780042460023FEF716FC4DB0BDEC088BBDE84C
:109C8800F08F00BFAFF300809A9999999999B93FDD
:109C98000000000000409F409A9999999999B9BF8E
:109CA8000000000000408F4089B5F81400E3693FC8
:109CB80000000000008076401F85EB51B81E194057
:109CC800B03E0020CC44002000006940000059400C
:109CD800000054C0000048430000C842C0440020AF
:109CE8007047FEE7FEE7FEE7FEE7704770477047FC
:109CF800FEF700B810B5094CA37A4BB1084B1A68A7
:109D080022F006021A6000F013F8204600F06FFEF9
:109D18004FF48020BDE8104002F0BABDB43E0020E8
:109D280010ED00E0014801F031B800BFB43E00205A
:109D3800364BD3F8882042F47002C3F88820344B9D
:109D48001A6842F001021A6000229A60196821F02C
:109D5800847121F4803119602E495960196882B0E4
:109D680021F480211960DA60009201921A6842F4A5
:109D780080321A601A6802F400320192009A0132A5
:109D88000092019A1AB9009AB2F5A06FF2D1204B4D
:109D98001B6813F4003318BF01230193019B012BA7
:109DA8002ED11B4B1A6C42F080521A641A4A116861
:109DB80041F4804111609A689A609A6842F40042BE
:109DC8009A609A6842F4A0529A60144A5A601A68D3
:109DD80042F080721A6019680D4A8901FBD5104B50
:109DE80040F205611960936823F003039360936858
:109DF80043F002039360936803F00C03082BFAD135
:109E0800024B4FF000629A6002B0704700ED00E02C
:109E18000038024010300024007000400854400709
:109E2800003C0240184B194A996801F00C010429BA
:109E380003D0082903D0164B19E0164B17E05968D0
:109E48005A6811F4800F596814BF124B104B02F076
:109E58003F02B3FBF2F30C4A5268C2F30142C1F36A
:109E68008811013252004B43B3FBF2F3074A1360E7
:109E7800054B9A68054BC2F303129A1819681279B0
:109E880021FA02F21A60704700380240F0020020FE
:109E98000024F40000127A0037B51C2301240025A1
:109EA80001A88DF804308DF805508DF806408DF81E
:109EB8000740FDF71DFB2046214603F059FB0A49E0
:109EC8004CF24F334B60A3F542430B800D814D801C
:109ED8004FF0804003F0F4FE4FF0804021462246C8
:109EE80004F0B3FA3EBD00BF7848002038B54FF003
:109EF8008040012104F0BEFA002836D04FF080409F
:109F080001211A4D04F0C1FA4FF08040002103F0FE
:109F18006CFF2B78013B042B27D8DFE803F00307FD
:109F28000B101E00BDE83840F6F754BCBDE83840B9
:109F3800F6F782BCF6F7CEFD00232B7038BD0C4A2D
:109F4800002313702B700B4B01241C70FEF722FDAD
:109F5800FEF726FD084B1C7038BD054B00241C700D
:109F68002C70FEF71DFD044B1C7038BD150E00202B
:109F78000A0E002024460020903E002008B540200C
:109F880002F078FC30B1FAF765FF4020BDE80840E0
:109F980002F07EBC08BD0000014608B5044804F084
:109FA80033FC0348402104F0DCFC0028F9D008BD4C
:109FB80000440040F0B589B04FF4E133012001932B
:109FC80000232B4CADF808301E460146ADF80A3088
:109FD800ADF80C30ADF810300C23ADF80E3003F0AE
:109FE800A3FA4FF40030012103F0C2FA20680221DD
:109FF800072202F071FF07226068032102F06CFF5C
:10A008000125022704232068059305A98DF81A6005
:10A018008DF81B508DF818708DF8197002F0DCFE61
:10A0280008236068059305A98DF8187002F0D4FE1E
:10A03800A06801A904F03EFB2A4640F225510D48CC
:10A0480004F076FC262307A88DF81C308DF81D60D7
:10A058008DF81E608DF81F50FDF74AFAA068294652
:10A0680004F0A5FB044A054B1A6009B0F0BD00BF17
:10A078000403002000440040A19F0008E451002090
:10A08800024B9868002104F092BB00BF0403002033
:10A0980010B5094C40F22551204604F06CFC50B133
:10A0A800A288D2B2112A02D1044B01211970044BA3
:10A0B80019884A401A8010BD004400400C0E002048
:10A0C800C40E00207047704773B50120014603F0A5
:10A0D8002BFA264C4FF4D8530093022303268DF80D
:10A0E80004302046002369468DF806308DF8073085
:10A0F8008DF8056002F070FE204608210A2202F061
:10A10800EBFE204609210A2202F0E6FE20460B213A
:10A118000A2202F0E1FE0A2220460C2102F0DCFEAF
:10A1280001254FF480632046694600938DF8065058
:10A138008DF807508DF8056002F04EFE0A210A4698
:10A14800204602F0C9FE29464FF4804003F01CFA6D
:10A158008020294603F0F4F94FF08050294603F097
:10A1680043FA284602F094FB7CBD00BF0000024081
:10A1780007B54FF4C060FDF7B1F943238DF80430FB
:10A188000322012301A88DF805308DF806208DF8EB
:10A198000730FDF7ADF90EBD782358430723B0FB10
:10A1A800F3F0002301338342FCD970474FF47A73EC
:10A1B8005843F1E737B50023104C019305460320B7
:10A1C800FFF7EAFFEB681A69013C019213D0019A84
:10A1D800002AF4DA019A42F001020192019A1A6106
:10A1E800064A1969013A019102D00199C907F8D4C0
:10A1F8000320FFF7D1FF00203EBD00BF410D030043
:10A2080010B5C47874B900EB820003339B10D0F802
:10A21800D000224603E051F8044C013204600431B6
:10A228009A42F8D1002010BD033230B59210D0F810
:10A23800D0400B46002003E02568013043F8045C59
:10A2480004339042F8D101EB800030BD0122F0B513
:10A258000023827040220129C37082800CD1082318
:10A268000370042343704FF4A073C3800223037266
:10A27800C1724FF0A04309E041B90C2303700623D3
:10A2880043704FF4A063C3801F4BC17203F5006293
:10A298000261C3604678044601461A46002508E074
:10A2A80002F5106C02F530620A65C1F814C0013578
:10A2B8003A460431B54202F12007F1D303F5806232
:10A2C800426103F58862C0F8CC20067803F5A065E2
:10A2D8000146002203E0C1F88C50013220350431D8
:10A2E800B242F8D31946002202E0C4F8CC10013279
:10A2F8000434B24201F58051F7D303F56063C0F826
:10A308000C310020F0BD00BF0000044038B5037ACE
:10A31800C2680025012B044625D1936B417A65F369
:10A32800104309B143F480139363D36823F4800383
:10A3380023F0500343F010036FF3C3036FF3C71305
:10A348006FF351436FF3D343D3602046FFF732FFD7
:10A35800E378012B3ED1052363F34405E36845F018
:10A3680020059D6036E0D36843F04003D360FFF7D3
:10A3780021FF237A627A032B14BF4FF434134FF46E
:10A388003C130AB143F48013E26814209363FFF787
:10A398000DFFE268217AD368032908BF43F48033AC
:10A3A800D360237A032B15D1156B012363F39B65C7
:10A3B8006FF3D7552D2345F0805563F31645156384
:10A3C800C820FFF7F3FEE36845F400051D63C820C5
:10A3D800FFF7ECFEE378012B07D1E3689D680522BF
:10A3E80062F3440545F020059D60002038BDC36830
:10A3F8009A6842F001029A6000207047C3689A6820
:10A4080022F001029A600020704707B500230193EB
:10A41800019B43F020030193019B61F38A1301938D
:10A42800019BC2681361064B1169013B019102D07F
:10A4380001998806F8D40320FFF7AEFE00200EBD70
:10A44800410D030007B500230193019B43F010035E
:10A458000193019BC2681361064B1169013B01918D
:10A4680002D00199C906F8D40320FFF795FE002011
:10A478000EBD00BF410D030008B5C268D3680129AD
:10A488006FF35D736FF39E7302D143F0005302E0E4
:10A4980009B943F080433220D360FFF787FE0020DC
:10A4A80008BDC368586900F001007047C3685B695C
:10A4B80013F0010F14BF002001207047C3685869CA
:10A4C80000F001007047C3685A69986910407047E6
:10A4D800C3685868704703691A6861F301021A6013
:10A4E8007047C268002393614FF0FF335361536094
:10A4F80053610B4B9361C3789169002B14BF4FF4E0
:10A5080000634FF4016343F4701343F4405343F082
:10A51800080321EA03010B4393610020704700BF41
:10A5280000080080F8B5D0F80C3100221A600369E1
:10A5380015461A6865F3CC221A60C37A012B0446C3
:10A548001BD10321FFF7C7FFE36880214FF4800286
:10A5580061F30F0259629A62C02262F30F0561F338
:10A568001F454FF4A072C3F8045162F30F056FF34F
:10A578001F45C3F80851C3F80C5110212046FFF7B6
:10A5880044FF2046FFF75EFF226900234FF0FF31AA
:10A598001361204653611E469161FF25D361214610
:10A5A80010E082691768C7F3076707F08007FFB2F2
:10A5B800002F14BF4FF09047002717600133166132
:10A5C8000430956062789342EBD300231D46FF2048
:10A5D80010E04A6D1668C6F3076606F08006F6B204
:10A5E800002E14BF4FF09046002616600133156107
:10A5F8000431906062789342EBD323691A6942F47C
:10A6080080721A61E278012A04D1054A402161F377
:10A6180059421A632046FFF764FF0020F8BD00BFC7
:10A628000301010003699B68C3F34103013B022B4B
:10A638009ABF024AD05C0320704700BF049B0408FD
:10A6480010B5036981699C680A68C4F3410002284F
:10A6580002D06FF30A0202E0032060F30A020A60E4
:10A668005A6842F480725A60002010BD30B54D78A7
:10A678000B780022012D00EB830405D105FA03F3C2
:10A68800A46963F30F0205E0012505FA03F3646D7D
:10A6980063F31F422368C3F3072505F08005EDB275
:10A6A8006DB98D6865F30A03CD78C98865F393435E
:10A6B80061F3995343F0805343F4004323600369E3
:10A6C800D9690A43DA61002030BD30B54D780B787E
:10A6D8000024012D224600EB830105D105FA03F37E
:10A6E800896963F30F0205E0012505FA03F3496D53
:10A6F80063F31F4203696FF3CF340C60D96921EA11
:10A708000202DA61002030BDF8B54F780B78012FCE
:10A7180000EB830349D19E694C69356833692A4641
:10A7280064F3120314B967F3DC430BE08F68E41990
:10A73800013CB4FBF7F7CC7867F3DC43012C08BF86
:10A7480064F35E733361C378012B06D10B780C690F
:10A7580000EB83039B695C610CE0CB78012B09D08B
:10A768004B693BB103690C785E6B012707FA04F467
:10A7780034435C63CB78012B07D103699B68DB0505
:10A7880054BF45F0005245F080520B7800EB83032C
:10A7980042F004429B691A60CB78012B38D10A78C1
:10A7A8008B8AC968FFF72CFD32E05E6D4F6935680A
:10A7B8008C6833692A462FB964F31203012464F3C1
:10A7C800DC430AE03F19013FB7FBF4F7BF05BF0DB3
:10A7D80067F3DC437C4364F312033361C378012BD2
:10A7E80005D10B780C6900EB83035B6D5C61CB785A
:10A7F800012B06D14B7913B145F0005201E045F029
:10A8080080520B7800EB830042F00442436D1A60DB
:10A818000020F8BD73B54D78012D3DD183694A6993
:10A828001E681C690094E4B242B962F306048DF80C
:10A8380000409DF8024065F3C4040EE08D68AA420A
:10A8480086BF4D6165F3060462F306048DF8004087
:10A858009DF80240012262F3C4048DF80240009A78
:10A868001A61C278012A05D10A780C6900EB8202C4
:10A878009269546146F004421A60C378002B34D1BF
:10A888004B69002B31D003690A78586B012101FA12
:10A8980002F202435A6328E00B784E698C6800EB99
:10A8A80083035B6D1A681D690095EDB206B14C61B2
:10A8B80064F306059DF802408DF80050012565F304
:10A8C800C4048DF80240009C1C61C378012B05D19B
:10A8D8000B780C6900EB83035B6D5C610B7800EB14
:10A8E800830042F00442436D1A6000207CBD4B781F
:10A8F800012B0B7800EB83000AD182691368C3F33C
:10A90800076101F08001C9B221B143F0804301E041
:10A91800426D136843F400131360002070474B78AE
:10A92800012B0B78C97800EB83000CBF8269426D5C
:10A9380002391368C9B26FF35553012998BF43F020
:10A94800805313600020704703699A69D8691040E2
:10A95800000C704700EB810102694B6D9B685069E0
:10A968001840704703699869DB69184080B27047DE
:10A9780082B000230093C0238DF803300122002306
:10A9880062F3C4038DF8023018238DF80030009A62
:10A99800436D1A61C278012A06D100F5B960586181
:10A9A8001A684FF080221A6002B07047D0F814314C
:10A9B80010B50446D3B103699A68D20716D5827ACE
:10A9C80042B1D0F80C21D0F80C116FF341026FF3AB
:10A9D80000020A605A6842F001025A600520FFF737
:10A9E800E5FB23695A6822F001025A6010BD837A98
:10A9F80063B103699B68D90708D5D0F80C31D0F842
:10AA08000C216FF341036FF30003136070470123B8
:10AA180010B5002280F8123104460346FF2104E0F5
:10AA280058698160186D0132816060780433824210
:10AA3800F6D3236900221A615A61DA614FF0FF32B6
:10AA48009A612046FFF7FEFC20461021BDE8104021
:10AA5800DBE44B78012B0B7800EB83000FD1836983
:10AA68001868C0F3074000F02003DBB2CBB900F050
:10AA78000200C0B200280CBF302020207047436D70
:10AA88001868C0F3074000F02003DBB25BB900F0A0
:10AA98000200C0B200280CBF4FF440504FF40050E1
:10AAA8007047102070474FF4805070474B78012B47
:10AAB8000B7810B500EB83030AD19C69102A236830
:10AAC80002D1BDE8104012E7202A0CD0302A0FE04E
:10AAD8005C6DB2F5805F236802D143F400131BE07C
:10AAE800B2F5005F02D143F0006315E0B2F5405FB4
:10AAF8000FD1C3F3074202F02002D2B222B10023E1
:10AB08004B71BDE810400AE743F0806343F08023AF
:10AB180002E00AB962F3CF33236010BDF8B50446EA
:10AB2800FFF794FB0122002384F8122184F81331E3
:10AB380028271646194640250CE007FB03F000F5C8
:10AB48008C7022182354D3805670D1709560D160D0
:10AB58005161013362789342EFD3002328261946C6
:10AB680040250CE006FB03F000F55C702218235426
:10AB7800D3805170D1709560D16051610133627892
:10AB88009342EFD32046FFF739FC2046FFF7BEFB80
:10AB980000212046FFF770FC2046FFF7C3FC204643
:10ABA800BDE8F840FFF723BC70B5CDB20C464FF0B6
:10ABB800280601F07F0106FB010115F0800F14BF84
:10ABC80001F58C7101F55C7104F07F04ED090C70DE
:10ABD8004D708A60CB7005B1CC80022B01D1002367
:10ABE8000B71FFF743FD002070BD10B5CAB201F02C
:10ABF8007F034FF0280404FB030312F0800F14BFF7
:10AC080003F58C7303F55C7301F07F01D2091970A9
:10AC18005A701946FFF759FD002010BD38B501F0EC
:10AC28007F0528246C4304F55C7401194B610023EB
:10AC38008B614B70EBB20355CA60C478012C08BF16
:10AC48000A6113B9FFF7E6FD01E0FFF75DFD00209B
:10AC580038BD70B501F07F042825654305F58C756E
:10AC680041190126E4B2CA600A6100224E704455B7
:10AC78008A614B6114B9FFF7CDFD01E0FFF744FD90
:10AC8800002070BDCAB212F0800F10B54FF0280333
:10AC980006D001F07F0403FB040303F58C7303E083
:10ACA80003FB010303F55C73D209012401F07F0162
:10ACB80019709C705A701946FFF719FE002010BDD4
:10ACC800CAB212F0800F10B54FF0280306D001F079
:10ACD8007F0403FB040303F58C7303E003FB010308
:10ACE80003F55C730024D20901F07F0119709C7090
:10ACF8005A701946FFF713FE204610BD08B50B061B
:10AD080004D501F07F01FFF780FB01E0FFF79AFB14
:10AD1800002008BD0369002261F30A1219680A437A
:10AD28001A60704703695A6803206FF341025A603A
:10AD3800FFF73CBA03695A68032042F002025A60DE
:10AD4800FFF734BA11F0800F4FF0280306D001F056
:10AD58007F0103FB010101F58C7103E003FB010195
:10AD680001F55C71FFF775BE11F0800F4FF02803F5
:10AD780006D001F07F0103FB010101F58C7103E0AE
:10AD880003FB010101F55C71FFF790BE2DE9F74F58
:10AD98000446FFF78BFB002800F03F822046FFF7B0
:10ADA80092FB0546002800F03882C0F3074000F007
:10ADB8000800C0B2002861D02046FFF7C5FDA146B3
:10ADC800824627464FF00008DFF86CB32E4650E065
:10ADD8001AF0010F46D05FFA88F211462046009219
:10ADE800FFF7B8FD10F0010F0546009A20D07B6DE3
:10ADF80001259D60E178A94207D11B69D9F878132C
:10AE0800C3F31203CB1AC9F88833DBF800302046A5
:10AE18001B6811469847E378012B09D1B8F1000F58
:10AE280006D194F81131052B02D12046FFF7A0FD79
:10AE380005F00203DBB213B17B6D02259D6005F0BE
:10AE48000403DBB213B17B6D04259D6005F0080592
:10AE5800EDB23DB1DBF8003020469B6898477B6D2A
:10AE68000820986008F101084FEA5A0A043709F1E6
:10AE78002809BAF1000FABD135460120C5F30743C5
:10AE880003F00403DBB2002B00F0AF802046FFF78D
:10AE980069FD264683464FF0000801959FE01BF0A8
:10AEA800010F00F0978023695FFA88F919695D6BD3
:10AEB80004EB890225FA09F59269ED019268EDB271
:10AEC8000D431540EA071CD55A6B012000FA08F11A
:10AED80022EA01025A63B369974A986013680546E3
:10AEE8005B68204649469847E378AB4209D1B8F1F8
:10AEF800000F06D194F81131042B02D12046FFF738
:10AF080037FD05F00403DBB213B1B36904259D6076
:10AF180005F00803DBB213B1B36908259D6005F09D
:10AF28001003DBB213B1B36910259D6005F020034F
:10AF3800DBB213B1B36920259D6005F04003DBB295
:10AF480013B1B36940259D6005F00203DBB213B16C
:10AF5800B36902259D6025F07F0515F0FF0F39D0F4
:10AF6800282505FB084505F58C75C246AB696A6955
:10AF7800C3EB020CAB689C4528BF9C460CF1030C44
:10AF8800B3694FEA9C0C9B696746A04614E0AA681F
:10AF9800E9681C1B944228BF1446A3B240464A469F
:10AFA800FFF72EF9EB681B19EB60AB69E71C1C195E
:10AFB800AC61B3699B69BF089BB2BB4205D9AC6958
:10AFC8006B699C4201D2002BE1D1B36980254446CC
:10AFD8009D60D04608F101084FEA5B0B0436BBF1CF
:10AFE800000F7FF45CAF019D012005F00203DBB286
:10AFF80013B1E36802225A61C5F3076303F08003C3
:10B00800DBB2CBB1A37A43B1D4F80C31D4F80C211C
:10B018006FF341036FF30003136023695A6822F04A
:10B0280001025A60444B1B6820469B699847E368B5
:10B038004FF000425A610120C5F3072303F00803CB
:10B04800DBB2F3B13C4B1B6820465B699847236928
:10B05800E2689B684FF400615161A27A82B1DB0714
:10B068000ED5D4F80C311A6842F001021A601A6839
:10B0780042F003021A60314B1A6942F006021A6163
:10B08800012005F00803DBB243B12B4B1B682046B7
:10B09800DB689847E36808225A61012005F010032D
:10B0A800DBB2002B33D0E3689A6922F010029A6170
:10B0B8001F6A282607F00F0306FB0346C7F343431E
:10B0C800022B06F55C7602D0062B1AD10EE047F665
:10B0D800F0733B40ABB1C7F30A172046F1683A4614
:10B0E800FFF7A2F8F368DB19F36007E004F5B9612C
:10B0F80020460822FFF798F8C7F30A17B369DF1943
:10B10800B761E3689A6942F010029A610120C5F3B9
:10B11800072303F01003DBB2002B39D023695A68E8
:10B12800002622F001025A6031462046FFF76DF9E9
:10B1380023463246FF2108E0A003002000ED00E08E
:10B1480058698160186D01328160607804338242E9
:10B15800F6D3236901274FF0FF3267F30F069A6190
:10B1680067F31F460F22DE615A612F221A611A689F
:10B178006FF30A121A602046FFF7FAFBE3684FF4F0
:10B1880080525A61264B1B6820461B6998473846EF
:10B19800C5F3072303F02003DBB2EBB12046FFF72A
:10B1A8004FFAE3682046DE68FFF73CFA032806D129
:10B1B8000023A3704FF40073A380092304E0012344
:10B1C800A3704023A380052363F38D26E3684FF41F
:10B1D8000052DE6001205A61C5F3074303F01003F3
:10B1E800DBB24BB10E4B1B682046DB699847E3681E
:10B1F8004FF480125A610120C5F3074505F0200578
:10B20800EDB255B1064B1B6820461B6A9847E368A8
:10B218004FF400125A610120FFE7BDE8FE8F00BF1E
:10B22800A003002043230B80004870471003002030
:10B2380038B51F4B1A68511C052A196035D1197980
:10B24800002201291A6030D09968B1F5006F08BF53
:10B258009A60174B9968DC68A1421A4602D100220D
:10B268001A7122E086BFC1F500631361C1EB0404C3
:10B27800D0F8EC3598BF14611569B3F839300C4C27
:10B288009D428AB204D95918ED1AA160256104E0DB
:10B298006918A1600021ABB22161054901240C7134
:10B2A80004498A188121FFF7D4FC002038BD00BF6B
:10B2B800C80E00201749002038B528230A4D03FB83
:10B2C80001010A4BB1F888131B69044628469847C0
:10B2D800D4F8EC352046B3F8403001212A46FFF770
:10B2E8009DFC002038BD00BFCF4800208C03002003
:10B2F80070B50B7813F0600506460C4625D0202D56
:10B308001FD1CD88B5B113F0800F487808D0214BF4
:10B3180021499B682A469847E2881F49304625E01C
:10B328001E4B1D4958641E4B30465D612A4600F08D
:10B3380022FB1DE0174B48789B6829462A46984708
:10B3480025E000F077FB022521E04B780A2B11D08D
:10B358000B2B14D0062B1AD14B881B0A212B03D197
:10B36800CA883A2A28BF3A220E49304600F0EAFA3B
:10B3780000250CE00C49012200F0E4FA07E08B7884
:10B388001BB9074A1D46936101E000F053FB2846AC
:10B3980070BD00BF8C0300200F490020100300205F
:10B3A800C80E002022030020E00E002010B58121E5
:10B3B8000446FFF71AFC01212046FFF716FC8221FC
:10B3C8002046FFF712FC024B5B689847002010BD2F
:10B3D8008C03002038B5D0F8EC350446B3F8392092
:10B3E80081210223FFF7E0FBD4F8EC350121B3F803
:10B3F800402020460223FFF7D7FB8221082203239F
:10B408002046FFF7D1FB094B022200251A715D7116
:10B41800074B1B689847D4F8EC35064AB3F8403018
:10B4280020460121FFF7FAFB284638BDD00300204B
:10B438008C030020CF48002010B5074C606CFF2813
:10B4480007D0064B064A9B68064952699847FF236E
:10B458006364002010BD00BF100300208C0300208F
:10B46800C80E00200F49002038B510490B79012B70
:10B4780019D10C690CB90C7115E0D0F8EC358D6850
:10B48800B3F839309C42AAB203D95D198D60E41A29
:10B4980003E0A3B22C198C6000240C6104495218F3
:10B4A8008121FFF7D6FB002038BD00BFC80E002061
:10B4B8001749002000207047002070470023F0B58E
:10B4C800084A094E1D4609E01468C75C375501341F
:10B4D8000133B4F5006F146008BF15608B42F3D1D7
:10B4E8000020F0BDD40E002017490020104B114A4F
:10B4F800D3F800C000232DE9F0410F4F16461D4632
:10B508000DE0146810F8038007F804800134802CDB
:10B5180008BF2C4614603468644505D001338B425B
:10B52800EFD10020BDE8F0810220BDE8F08100BF26
:10B5380098510020AC5100201851002021280FD12B
:10B54800084B1A680A701A68120A4A705A888A7070
:10B55800DA78CA701A790A715A794A719B798B71AB
:10B56800002070478403002007B502AB012103F8CF
:10B57800010D1846FFF7A2FF0EBD002100E00131C2
:10B58800435C002BFBD199E798E70B4B0B491A68F2
:10B59800096891420BD00A498A5C02701A68013224
:10B5A800802A1A6005D100221A6001207047002005
:10B5B80070470120704700BF98510020AC5100200F
:10B5C80018510020204B1A68204B1B689A42F0B58E
:10B5D80009D135E00133802B08BF00239A4203D1FB
:10B5E8001A4B1A602CE01A4CE15C0029F2D00A29A7
:10B5F800F0D00D29EED0154C1549134D23600E4699
:10B608000023CF182268BA5CC254226801339F18FD
:10B61800802F08BF53422F689A18974210D0B25C07
:10B628001AB10A2A01D00D2AEBD10022C254074AC6
:10B63800116859187F29116003D98039116000E019
:10B6480000231846F0BD00BFAC51002098510020DF
:10B6580018510020704700BFD0F8E43510B51B69B9
:10B6680004469847032384F81231002010BD08B51A
:10B67800042380F81231D0F8E435DB6898470020BD
:10B6880008BD08B5D0F8E035DB6903B1984700205C
:10B6980008BD08B5D0F8E0351B6A9847002008BDFA
:10B6A80008B5D0F8E0355B6A9847002008BD00214E
:10B6B80010B5402204460B46FFF776FA8021402257
:10B6C80000232046FFF770FA012384F81231D4F8DA
:10B6D800E435A0785B689847002010BD13B569462B
:10B6E800044600F085F99DF8001001F01F03012BB6
:10B6F80007D0022B0AD073B92046694600F026FA13
:10B708000FE02046694600F007FA0AE0204669463D
:10B7180000F0A2F905E021F07F01C9B22046FFF749
:10B72800B1FA00201CBD38B5044600293DD190F877
:10B738001131022B42D1D0F83421D0F820319A426D
:10B7480011D9C178D21A0129C0F8342104D1D0F80E
:10B758002411CB18C0F8243192B22046D4F8241111
:10B7680000F000F92AE0D0F83821B2FBF3F503FB2A
:10B77800152565B99A420AD3D0F83C319A4206D2C7
:10B7880029462A4600F0EEF8C4F83C5116E0D4F8F1
:10B79800E035DB682BB194F81221032A01D1204649
:10B7A8009847204600F00FF908E0D0F8E0355B69CB
:10B7B80023B190F81221032A00D19847002038BD00
:10B7C80010B5044659BB90F81131032B30D1D0F88D
:10B7D8008C23D0F878339A4214D9C178D21A012927
:10B7E800C0F88C2304D1D0F87C13C918C0F87C1396
:10B7F8009A4228BF1A4692B22046D4F87C1300F029
:10B80800CAF815E0D0F8E0351B6923B190F8122189
:10B81800032A00D19847204600F0C6F808E0D0F87F
:10B82800E0359B6923B190F81221032A00D198478B
:10B83800002010BD2DE9F041069F044616469846A3
:10B848000D46FEF741FC20462946C4F8E085C4F8B9
:10B85800E475C4F8E865FFF761F9D4F8E4351B68C6
:10B8680098472046BDE8F041FEF782BC00207047AB
:10B87800D0F8E03510B504461B689847D4F8E4358D
:10B888009B689847002010BD08B5D0F8E0355B6884
:10B898009847002008BD000012230B80004870471D
:10B8A800D003002004230B8000487047E2030020E7
:10B8B80010B5044C04480A46214600F075FA2046A3
:10B8C80010BD00BFB051002046A005080A4608B5C3
:10B8D8000248034900F068FA014808BD59A0050864
:10B8E800B05100200A4608B50248034900F05CFA46
:10B8F800014808BD67A00508B051002008B50A46F0
:10B9080008B9044800E00448044900F04DFA034827
:10B9180008BD00BF72A005087FA00508B05100202F
:10B9280008B50A4608B9044800E00448044900F08C
:10B938003BFA034808BD00BF8CA00508ADA0050868
:10B94800B051002010B513460C46C0F83821C0F895
:10B958003421022280F8112100212246FFF779F9CB
:10B96800002010BD10B50C46134600212246FFF7F3
:10B9780070F9002010BD10B513460C46C0F890238E
:10B98800C0F88C23032280F8112100212246FFF7FA
:10B9980045F9002010BD10B50C461346002122467B
:10B9A800FFF73CF9002010BD0021042310B50A461A
:10B9B800044680F811310B46FFF74BF92046FEF795
:10B9C800D7FF002010BD0021052310B50A46044604
:10B9D80080F811310B46FFF721F92046FEF7C8FF22
:10B9E800002010BD282303FB0100B0F8880370472E
:10B9F80090F8C8350B7090F8C9354B7090F8CB2586
:10BA080090F8CA3503EB02234B8090F8CD2590F8C7
:10BA1800CC3503EB02238B8090F8CF2590F8CE35F8
:10BA280003EB02239BB2CB80C0F83C31012380F8A2
:10BA38001131704710B591F90030002B044601DB35
:10BA4800CB880BB9802100E00021FFF71BF92046C5
:10BA5800BDE81040FEF78CBF38B50D4604466B783C
:10BA68000979012B10D027D3032B51D190F812312B
:10BA7800022B28D0032B47D16B889BB991B1802921
:10BA880010D0FFF7FFF80DE090F81231022B1AD012
:10BA9800032B39D16B88002B3AD149B1802907D0C3
:10BAA800FFF70EF9D4F8E03520469B6829469847F9
:10BAB8002046FFF779FF2BE090F81231022B02D0D5
:10BAC800032B21D106E019B3802921D02046FFF7A6
:10BAD800D9F81DE011F0800F4FF0280306D001F0CF
:10BAE8007F0103FB010393F81A2103E003FB010123
:10BAF80091F87223074B02B101221A6020460549CA
:10BB08000222FFF71FFF03E020462946FFF792FFB6
:10BB1800002038BDE40E002038B590F81231032B10
:10BB280004460D460CD10B79012B09D8D0F8E03525
:10BB38009B689847EB883BB92046FFF735FF03E041
:10BB480020462946FFF776FF002038BD73B54B78AD
:10BB580004460D46092B00F21C81DFE813F0D100E2
:10BB680008011A01E4001A0172000A001A01C00053
:10BB780092004B881A0A013A062A00F20A81DFE885
:10BB880012F007001A00270008010801080108013F
:10BB9800D4F8E835A0781B680DF106019847EB88C2
:10BBA800402B014603D094F81231012B3AD10823D7
:10BBB800ADF8063036E0D4F8E035A0789B6A0DF190
:10BBC80006019847022343700146C4F8EC0529E0B2
:10BBD800DBB2052B00F2DD80DFE803F003080D126D
:10BBE800171CD4F8E835A0785B6817E0D4F8E83576
:10BBF800A0789B6812E0D4F8E835A078DB680DE0FF
:10BC0800D4F8E835A0781B6908E0D4F8E835A078BE
:10BC18005B6903E0D4F8E835A0789B690DF106016B
:10BC280098470146BDF80630002B00F0B680EA8838
:10BC3800002A00F0B2809A4228BF1A46ADF80620C2
:10BC48005CE08B88002B40F0A480CB88002B40F070
:10BC5800A08094F812214B88032A00F09A8003F000
:10BC68007F05204684F813512946FFF753F82046EC
:10BC7800FFF79AFE0DB1022300E0012384F8123188
:10BC88008BE08978464E0129317100F2828094F860
:10BC98001231022B02D0032B7BD108E0002962D09D
:10BCA8000121032384F8101184F8123113E041B9FB
:10BCB800022384F8123184F810112046FFF7E4FDBE
:10BCC80051E094F81011012920464DD0FFF7DCFD12
:10BCD800317984F810112046FFF7CAFD43E0CA887D
:10BCE800012A56D194F81231022B02D0032B50D1DD
:10BCF80002E020462B4913E004F5887120460FE046
:10BD080094F81231023B012B43D8D4F8143124495A
:10BD1800002B0CBF0123032341F80C3F20460122CE
:10BD2800FFF710FE39E04B88012B29D0022B34D1C4
:10BD38008B8813F0FF0F30D121691B0A013B4A6839
:10BD4800042B0FD8DFE803F0030507090B000123D4
:10BD580006E0022304E0032302E0042300E00523B5
:10BD680063F306124A602046FFF71EFE15E094F8BA
:10BD78001231023B012B0CD84B88012B0DD100232B
:10BD8800C4F81431D4F8E03520469B682946984712
:10BD9800E9E720462946FFF74DFE00207CBD00BF9D
:10BDA800E40E0020EC0E002030B5C8B10023DDB24F
:10BDB8000133C41814F8014C002CF8D16B1C5B003B
:10BDC80013800B7003234B70022305E0CA545A1CDE
:10BDD800D2B202338C54DBB210F8012B002AF5D111
:10BDE80030BD00BF70477047704770477047704755
:10BDF800704700000EB403B070470A2810B5044617
:10BE080002D10D20FFF7F9FF064A13681BB103F8AA
:10BE1800014B136010BD044B1B680BB120469847BB
:10BE280010BD00BFF40E0020E451002010B50446F8
:10BE380001E0FFF7E2FF14F8010B0028F9D110BD6B
:10BE48002DE9F04F044685B00D464FF00A0A00E090
:10BE580035462078002800F0C480252801D0013418
:10BE680067E06078302803D1A0780123033407E025
:10BE78002D2802D00234002302E0A07802230334E4
:10BE88004FF0000805E00AFB080814F8010BA8F1B8
:10BE98003008A0F13002D2B2092AF4D96C2801D0B6
:10BEA8004C2803D114F8010B43F00403002800F0D8
:10BEB8009880602886BFA0F12002D2B202464F2A9D
:10BEC8003DD006D8432A2DD0442A09D0422A30D161
:10BED80033E0552A04D0582A29D0532A29D101E021
:10BEE8000A272DE02E1D2F68002500E001357A5D18
:10BEF800002AFBD104E02020FFF77FFF4D4601E038
:10BF0800980704D4454505F10109F4D34D46384650
:10BF1800FFF78CFF03E02020FFF76FFF0135454551
:10BF2800F9D395E728782E1DFFF767FF90E71027CC
:10BF380006E0FFF762FF2E468AE7022700E008279F
:10BF48002E1D442A296804D1002902DA494243F007
:10BF58000803002200E02A46B1FBF7FE07FB1E118A
:10BF6800CDB2092D714607D9782814BF4FF0070CB8
:10BF78004FF0270C6544EDB230350DF80250551CD2
:10BF8800BEF1000F02D0102DE5D10F22190705D5FB
:10BF980004A94D192D2105F8101C951C13F0010F4B
:10BFA8000CBF4FF0200B4FF0300B9B072F4604D5EA
:10BFB80008E05846FFF721FF4F46474507F10109BA
:10BFC800F7D34F46013D1DF80500FFF716FF002D7A
:10BFD800F8D103E02020FFF710FF01374745F9D3D8
:10BFE80036E705B0BDE8F08F70B5064D0C462E68F3
:10BFF800286001E0FFF701FF14F8010B0028F9D1D0
:10C008002E6070BDE45100200FB407B504A951F8A3
:10C01800040B0191FFF714FFBDE80E4004B0704710
:10C028000EB417B505A9084C51F8043B2060184612
:10C038000191FFF705FF2268002313702360BDE814
:10C048001E4003B0704700BFF40E00200EB433B595
:10C0580005A9074C51F8043B256820601846019152
:10C06800FFF7EEFE2560BDE83C4003B0704700BF17
:10C07800E451002070B51E4604461C481546FFF7DB
:10C08800C3FF022E1FD0042E25D0012E2AD105E091
:10C09800A15D1748FFF7B8FF013600E00026AE4261
:10C0A800F6DB2020FFF7A9FE002609E0A05DA0F13D
:10C0B8002003DBB25E2B88BF2E20FFF79EFE0136E1
:10C0C800AE42F3DB0EE034F8021B0A48FFF79CFF90
:10C0D800013DF8D106E054F8041B0748FFF794FF28
:10C0E800013DF8D10A20BDE8704086E6CEA00508DB
:10C0F800D5A00508DBA00508E1A0050808B50121C1
:10C108004FF4807001F07CFA4FF480700021BDE894
:10C11800084001F075BA43680A6823F0407323F4B5
:10C12800807313430A7943EA02234360CA680B69A0
:10C1380030B51A4384688D68084B2A43234013435B
:10C148004A7943EA420383600B7DC26A013B22F4C9
:10C158007002DBB242EA0353C36230BDFDF7FFC091
:10C1680000230360037143718360C360036101238B
:10C1780003757047074A084B516810B50B4090E8A3
:10C18800120021438468C068214301430B43536074
:10C1980010BD00BF00230140E030FCFF0023036016
:10C1A80043608360C3607047836811B143F0010343
:10C1B80001E023F0010383607047436823F44003E0
:10C1C80023F400730B4343607047416282627047F7
:10C1D800436823F01F030B4343607047044B5A68BE
:10C1E80010B142F4000201E022F400025A607047E4
:10C1F80000230140044B5A6810B142F4800201E068
:10C2080022F480025A60704700230140092970B562
:10C218000CB20CD904EB44041E3CC6680725A540A3
:10C2280026EA0505A34045EA0304C4600AE0066956
:10C2380004EB44040725A54026EA050513FA04F48F
:10C248002C430461062A0CD80523013A5A43446B4F
:10C258001F23934024EA0303914043EA0102426307
:10C2680070BD0C2A12B20CD802EB8202233A046B7E
:10C278001F23934024EA0303914043EA0102026327
:10C2880070BD02EB8202413AC46A1F23934024EA3C
:10C298000303914043EA0102C26270BD836843F020
:10C2A8008043836070478068C0F38050704783681C
:10C2B80011B143F4806301E023F480638360704725
:10C2C800836811B143F0020301E023F002038360A5
:10C2D80070474368013923F4604343EA41334360BC
:10C2E8007047436811B143F4006301E023F400632D
:10C2F80043607047C06C80B27047014B1868704744
:10C3080008230140836811B143F4807301E023F4EA
:10C31800807383607047836811B143F4007301E050
:10C3280023F4007383607047044B5A6810B142F4D9
:10C33800005201E022F400525A6070470023014085
:10C34800092970B50CB20CD904EB44041E3CC6682C
:10C358000725A54026EA0505A34045EA0304C4606D
:10C368000AE0066904EB44040725A54026EA05050A
:10C3780013FA04F42C430461836BC3F30154121BB6
:10C388000232D2B202EB82021F24944023EA040351
:10C3980091400B43836370BD836B013923F44013D1
:10C3A80043EA01538363704782B0002301930190ED
:10C3B800019BCB180193019B1A6002B070478368F8
:10C3C80023F470230B4383607047836823F440137E
:10C3D8000B4383607047836843F48003836070472E
:10C3E8008068C0F380507047436811B143F480639C
:10C3F80001E023F4806343607047436811B143F45C
:10C40800805301E023F480534360704782B00023D7
:10C4180001930190019B28335B180193019B1868D5
:10C4280080B202B070470123C9B213FA01F1436820
:10C438000AB1194301E023EA01014160704703682A
:10C4480019420CBF002001207047C94301607047A2
:10C458004368006810EA112007D00122C9B212FA15
:10C4680001F119420CBF0020012070476FEA112129
:10C4780001607047036823F0010303600023036031
:10C4880043608360C3600361212343612C4B98425E
:10C498001CD02C4B984220D02B4B984225D02B4BAC
:10C4A80098422AD02A4B98422FD02A4B984233D010
:10C4B800294B984237D0294B984204D14FF03D522E
:10C4C80043F8AC2C7047264B984203D13D2243F8E1
:10C4D800082C7047234B984204D14FF4746243F8F8
:10C4E800202C7047204B984204D14FF4741243F823
:10C4F800382C70471D4B984204D14FF0746243F8B2
:10C50800502C70471A4B984203D11A4A43F8642CAE
:10C518007047194B984203D1184A43F87C2C70474E
:10C52800174B984203D1174A43F8942C7047164B7F
:10C53800984204BF4FF03D5243F8AC2C704700BFFF
:10C54800106002402860024040600240586002408B
:10C558007060024088600240A0600240B8600240FB
:10C56800106402402864024040640240586402405B
:10C57800706402403D00002088640240400F0020A3
:10C58800A064024000003D20B86402400268134BDA
:10C5980010B51340CC680A6822434C6922438C6961
:10C5A8002243CC6922430C6A22434C6A22438C6A98
:10C5B80022434C6B22438C6B224313430360426932
:10C5C8000C6BCB6A22F007022343134343610B69C8
:10C5D80043604B6883608B68C36010BD3F801CF06C
:10C5E8000023036043608360C36003614361836128
:10C5F800C361036243628362C36203634363836309
:10C608007047036811B143F0010301E023F001030F
:10C6180003607047036811B143F4004301E023F459
:10C62800004303607047036811B143F0200301E041
:10C6380023F020030360704741607047406880B270
:10C648007047036812B143F4002301E023F4002388
:10C65800036001617047036811B143F4802301E06E
:10C6680023F48023036070470AB101617047C160F9
:10C6780070470068C0F3C0407047006800F00100D0
:10C688007047406900F0380070470A4A0A4B10B5F5
:10C698000A4CA04288BF13468A004CBF5B681B68DF
:10C6A80021F0F02121F0821119420CBF0020012055
:10C6B80010BD00BF00640240006002400F640240E9
:10C6C80010B5084B084A094CA04288BF134611F020
:10C6D800005F21F0F02121F0821114BFD960996028
:10C6E80010BD00BF00600240006402400F640240B9
:10C6F8000B0607D5436912B143F0800301E023F02C
:10C7080080034361802909D001F01E01036812B13A
:10C7180019430160704723EA010101607047124B19
:10C72800124A10B5124CA0428CBF14461C4621F088
:10C73800F02323F0C3132BB1026802F01E0202EAB1
:10C74800D12202E0426902F0800288004CBF63688F
:10C75800236821F0F02121F08210184002D0101C2B
:10C7680018BF012010BD00BF0060024000640240F5
:10C778000F64024010B5084B084A094CA04288BF14
:10C78800134611F0005F21F0F02121F0821114BF4F
:10C79800D960996010BD00BF00600240006402408B
:10C7A8000F640240044B00221A605A609A60DA60F3
:10C7B800024A5A61704700BF003C0140FFFF7F00FA
:10C7C800837910B5002B29D01A4B01681C68CA431D
:10C7D80014401C605C6822405A60027902F1804271
:10C7E80002F59E3214682143116002689C68D143A7
:10C7F8000C409C60DC682140D9604179102906D141
:10C80800996811439960D9680A43DA6010BD01F14B
:10C81800804303F59E3319680A4308E003790168E9
:10C8280003F1804303F59E331A6822EA01021A6075
:10C8380010BD00BF003C014000230C2203600371BF
:10C84800427183717047024B1A6902431A6170473B
:10C85800003C0140034B5B6918420CBF00200120DB
:10C86800704700BF003C0140014B5861704700BF52
:10C87800003C0140054B1A685B69034004D0104234
:10C888000CBF00200120704718467047003C01404B
:10C89800014B5861704700BF003C01404FF02043F6
:10C8A80018B943F2DB021A6003E043F2D20243F8FC
:10C8B80020204FF02042411C6FF0704342F8213095
:10C8C80002F5827242F82030704770B58468456876
:10C8D800C368C16A026825431D4303691D43436950
:10C8E8001D4383691D43C3691D43036A1D43436A8E
:10C8F8001D43836A1D43036B0D431D434FF02043C3
:10C90800082C43F8225005D153F8224044F0400443
:10C9180043F82240436B9E691D6835435E6845EACB
:10C9280006159E6845EA0625DE6845EA06451E693D
:10C938005B6945EA0655541C45EA03654FF02043F8
:10C94800B1F5804F43F8245010D1836B986919686A
:10C958000143586841EA0011986841EA00211869C2
:10C968005B6941EA005141EA036101E06FF07041FF
:10C97800014B43F8221070BD040100A0022242605E
:10C988004FF480524262416B4FF4005210B58262FC
:10C9980000230F22FF2403608360C36003614361A7
:10C9A8008361C3610362C36203630A604A608C6087
:10C9B800CA600A614A618B61816B0A604A608C6057
:10C9C800CA600A614A618B6110BD4FF0204321B1F2
:10C9D80053F8202042F0010203E053F82010024AE5
:10C9E8000A4043F820207047FEFF0F0010280CBFB4
:10C9F800064B074B4FF040024FF0180119605A6080
:10CA08004FF0FC329A60DA60704700BF600000A007
:10CA1800800000A030B5836844681C43C36844F0B4
:10CA280008041C4303691C43436944EA432483699B
:10CA380044EA4334C36999685A68090441EA0221FF
:10CA48001A68DB68114341EA0361036A9A685D6802
:10CA5800120442EA05221D68DB682A4342EA03629F
:10CA68000368102B0CBF034B034B1C609960DA6002
:10CA780030BD00BF600000A0800000A0102303604C
:10CA8800C269002343608360C360036143618361BB
:10CA9800FC23136053609360D360026A1360536091
:10CAA8009360D360704741B110280CBF074B084B07
:10CAB8001A6842F004021A60704710280CBF034A33
:10CAC800034A044B11680B4013607047600000A0D4
:10CAD800800000A0FBFF0F0041B110280CBF084BDD
:10CAE800084B1A6842F040021A60704710280CBFC1
:10CAF800034A044A044B11680B401360704700BF97
:10CB0800600000A0800000A0BFFF0F00102802D125
:10CB1800024B58697047024B58697047600000A083
:10CB2800800000A0054B18221A6000225A604FF0BE
:10CB3800FC329A60DA601A61704700BFA00000A05A
:10CB48000268436842F0100242EA4322836842EADC
:10CB58004332144B10B51A60C268916854680904CE
:10CB680041EA04211468D268214341EA02629A60CA
:10CB7800026991685468090441EA04211468D2687A
:10CB8800214341EA0262DA60426991685068090407
:10CB980041EA00211068D268014341EA02621A6141
:10CBA80010BD00BFA00000A0C2680023036043605E
:10CBB8008360FC23136053609360D3600269136041
:10CBC80053609360D3604269136053609360D3608D
:10CBD8007047054B18B11A6842F0040202E0196860
:10CBE800024A0A401A607047A00000A0FBFF0F002D
:10CBF80062B1102801D10E4B03E0B0F5807F03D15C
:10CC08000C4B5A68114311E00B4BFAE7102804D17A
:10CC1800074B5A6822EA010108E0B0F5807F0CBF93
:10CC2800044B054B5A686FEA01011140596070477F
:10CC3800600000A0800000A0A00000A0102801D182
:10CC4800064B04E0B0F5807F0CBF054B054B5B68D5
:10CC58000B420CBF00200120704700BF600000A0FD
:10CC6800800000A0A00000A0102804D1074B5A683B
:10CC780022EA010108E0B0F5807F0CBF044B054BA8
:10CC88005A686FEA0101114059607047600000A0BE
:10CC9800800000A0A00000A0102801D1084B04E0EB
:10CCA800B0F5807F0CBF074B074B5B6813EA0100A8
:10CCB80004D013EAD1010CBF00200120704700BF47
:10CCC800600000A0800000A0A00000A0102804D1EF
:10CCD800084B5A6822EAD10109E0B0F5807F0CBF01
:10CCE800054B064B5A684FEAD10122EA0101596007
:10CCF800704700BF600000A0800000A0A00000A056
:10CD080008B52C4B984205D10120014600F048FC9B
:10CD1800012048E0284B984205D10220012100F06B
:10CD28003FFC02203FE0254B984205D10420012119
:10CD380000F036FC042036E0214B984205D108204B
:10CD4800012100F02DFC08202DE01E4B984205D152
:10CD58001020012100F024FC102024E01A4B9842F6
:10CD680005D12020012100F01BFC20201BE0174BDF
:10CD7800984205D14020012100F012FC402012E029
:10CD8800134B984205D18020012100F009FC802036
:10CD980009E0104B98420BD14FF48070012100F04C
:10CDA800FFFB4FF480700021BDE8084000F0F8BB9D
:10CDB80008BD00BF00000240000402400008024015
:10CDC800000C02400010024000140240001802400B
:10CDD800001C0240002002402DE9F0470023D1F852
:10CDE80000801A464FF0010C03270CFA02F404EAFB
:10CDF8000805A5422ED1066817FA03F4E443264035
:10CE080006600E79D0F8009006FA03FA013E4AEA65
:10CE18000909012EC0F8009014D8866891F8059089
:10CE280026408660866809FA03F949EA060686609C
:10CE3800466826EA050545608D7946689540ADB295
:10CE480035434560C5682C40C460CC79C5689C40B2
:10CE58002C43C46001320233102AC6D1BDE8F087E2
:10CE68004FF6FF7303600023037143718371C3712D
:10CE7800704782B04FF480330193019B0B430193B9
:10CE8800019BC361C161019BC361C3690193C3690C
:10CE9800019302B07047036919420CBF00200120BA
:10CEA8007047006980B27047436919420CBF00207F
:10CEB80001207047406980B2704701837047418301
:10CEC80070470AB1018370474183704741617047D9
:10CED80043694B404361704701F00703C9080831B3
:10CEE80030B59B0050F821500F249C4025EA0404DB
:10CEF80040F8214050F8214012FA03F31C4340F84F
:10CF0800214030BD08B5134B984207D14FF40010AB
:10CF1800012100F069FB4FF4001014E00E4B984219
:10CF280007D14FF48000012100F05EFB4FF4800030
:10CF380009E00A4B98420BD14FF40000012100F0A0
:10CF480053FB4FF400000021BDE8084000F04CBB43
:10CF580008BD00BF0054004000580040005C00407D
:10CF68007FB50446868868460D4600F06DFA02993A
:10CF78002C482B6826F03F063604B1FBF0F0360C3F
:10CF880080B20643A680228822F001021204120C05
:10CF98002280254A93420AD85B00B1FBF3F30130A3
:10CFA8009BB280B22084032B98BF042321E0EE8833
:10CFB8004BF6FF72964205D103225343B1FBF3F3BC
:10CFC8009BB206E019225343B1FBF3F39BB243F43F
:10CFD80080431A054FF4967208BF43F0010350438B
:10CFE8004FF47A7290FBF2F0013080B243F40043C0
:10CFF8002084A38323886989AA889BB243F001030C
:10D008002380238823F4816323F002031B040A434B
:10D018001B0C13439BB223802A89AB8913439BB211
:10D0280023817FBD40420F00A086010041F2883372
:10D038000360002383804BF6FF72038143814FF422
:10D048008043C28083817047038819B19BB243F043
:10D05800010303E023F001031B041B0C038070474A
:10D06800038819B19BB243F4807303E023F48073FF
:10D078001B041B0C03807047038819B19BB243F44F
:10D08800007303E023F400731B041B0C0380704738
:10D0980012B141F0010101E001F0FE010182704787
:10D0A800038819B19BB243F4806303E023F48063DF
:10D0B8001B041B0C0380704783899BB201F0FE019F
:10D0C80023F0FE030B4383817047838919B19BB218
:10D0D80043F0010303E023F001031B041B0C8381CD
:10D0E8007047038819B19BB243F0400303E023F073
:10D0F80040031B041B0C03807047038829B16FEAA7
:10D1080043436FEA53439BB201E05B045B0C03802B
:10D118007047038819B99BB243F0800303E023F0FA
:10D1280080031B041B0C03807047B1F5804F838B71
:10D1380004D023F480431B041B0C02E09BB243F48D
:10D14800804383837047B1F5006F038803D19BB296
:10D1580043F4006303E023F400631B041B0C038007
:10D168007047B1F5005F038803D19BB243F40053C5
:10D1780003E023F400531B041B0C0380704703884F
:10D1880019B19BB243F0100303E023F010031B0412
:10D198001B0C0380704701827047008AC0B2704739
:10D1A800038819B19BB243F4805303E023F48053FE
:10D1B8001B041B0C03807047B1F5006F038803D173
:10D1C8009BB243F4006303E023F400631B041B0CCD
:10D1D80003807047038819B19BB243F0200303E032
:10D1E80023F020031B041B0C03807047008BC0F343
:10D1F80007207047838819B19BB243F4006303E0AA
:10D2080023F400631B041B0C83807047838819B1C7
:10D218009BB243F4805303E023F480531B041B0C9C
:10D228008380704782B0002301930190019BCB1843
:10D238000193019B188880B202B0704783889BB223
:10D248000AB1194301E023EA010181807047838A0A
:10D25800008B9BB243EA0040084020F07F40431A0D
:10D26800584240EB03007047838A008B9BB243EA25
:10D27800004020F07F40704782B000230093019364
:10D288000B0F01900093009B21F07F4113B1019B8C
:10D29800143302E0019B090C18330193019B1B68AE
:10D2A80019420CBF0020012002B07047C94389B25F
:10D2B800818270478388808A80B208409BB206D0FA
:10D2C80001F0E06113EA11410CBF00200120704712
:10D2D800C94389B2818270470A4B1A6842F0010239
:10D2E8001A6000229A60196821F0847121F4803153
:10D2F800196005495960196821F480211960DA60BC
:10D30800704700BF0038024010300024024B002252
:10D318001A701870704700BF02380240034B1A6831
:10D3280022F0F80242EAC0021A6070470038024050
:10D33800014B1860704700BF00004742064B0022AF
:10D3480001281A701A7002D0042804D101E018705C
:10D35800704705221A70704770380240014B1860F8
:10D36800704700BF800E4742014341EA821200998C
:10D378005B08013B42EA016141EA0341014B596004
:10D38800704700BF00380240014B1860704700BF6B
:10D39800600047428001034B40EA0171C3F88410E2
:10D3A800704700BF00380240014B1860704700BF4B
:10D3B80068004742014B1860704700BF4C00474265
:10D3C800034B9A6822F0EC6202430A439A60704762
:10D3D80000380240034B9A6822F0784202430A431D
:10D3E8009A60704700380240034B9A6822F00302A3
:10D3F80002439A60704700BF00380240024B9868A9
:10D4080000F00C00704700BF00380240034B9A68D8
:10D4180022F0F00202439A60704700BF00380240D1
:10D42800034B9A6822F4E05202439A60704700BFA7
:10D4380000380240034B9A6822F4604242EAC00274
:10D448009A607047003802401E4B9A6802F00C023E
:10D45800042A10B503D0082A03D01B4B18E01B4B35
:10D4680016E059685A6811F4800F596814BF174BB1
:10D47800154B02F03F02B3FBF2F3124A5268C2F3B3
:10D488000142C1F3881101324B435200B3FBF2F35E
:10D498000C4903608B680E4A0468C3F30313D35C1A
:10D4A80034FA03F343608C68C4F38224145D33FABE
:10D4B80004F484608968C1F34231525CD340C3608C
:10D4C80010BD00BF003802400024F40000127A00AA
:10D4D8002804002000F44073B3F5407F084B08D1BE
:10D4E800996820F0704221F4F81122F440720A433E
:10D4F8009A601A6F000542EA10501867704700BF1B
:10D5080000380240014B1860704700BF3C0E47428C
:10D51800014B1860704700BF400E4742014B18602E
:10D52800704700BF5C014742044B1A6B09B11043B6
:10D5380001E022EA00001863704700BF003802408B
:10D54800044B5A6B09B1104301E022EA000058630A
:10D55800704700BF00380240044B9A6B09B1104372
:10D5680001E022EA00009863704700BF00380240DB
:10D57800044B1A6C09B1104301E022EA0000186458
:10D58800704700BF00380240044B5A6C09B1104381
:10D5980001E022EA00005864704700BF00380240EA
:10D5A800044B1A6909B1104301E022EA000018612E
:10D5B800704700BF00380240044B5A6909B1104354
:10D5C80001E022EA00005861704700BF00380240BD
:10D5D800044B9A6909B1104301E022EA00009861FE
:10D5E800704700BF00380240044B1A6A09B1104363
:10D5F80001E022EA00001862704700BF00380240CC
:10D60800044B5A6A09B1104301E022EA000058624B
:10D61800704700BF00380240044B1A6D09B110432F
:10D6280001E022EA00001865704700BF0038024098
:10D63800044B5A6D09B1104301E022EA0000586515
:10D64800704700BF00380240044B9A6D09B110437F
:10D6580001E022EA00009865704700BF00380240E8
:10D66800044B1A6E09B1104301E022EA0000186663
:10D67800704700BF00380240044B5A6E09B110438E
:10D6880001E022EA00005866704700BF00380240F7
:10D69800044B1A7809B1104301E022EA000018701F
:10D6A800704700BF0D3802404309012B074A01D1DA
:10D6B800136803E0022B0CBF136F536F00F01F00B9
:10D6C80033FA00F000F00100704700BF0038024054
:10D6D80007B5002301933120FFF7E6FF019B0133D3
:10D6E8000193019BB3F5A06F01D00028F3D031203E
:10D6F800FFF7DAFF003018BF01200EBD024B5A6F4A
:10D7080042F080725A67704700380240034BDB686A
:10D7180018420CBF00200120704700BF00380240AB
:10D72800014B1870704700BF0E38024008B5154B02
:10D7380098420BD101214FF48050FFF761FF4FF45D
:10D7480080500021BDE80840FFF75ABF0E4B9842B1
:10D7580007D14FF480400121FFF746FF4FF4804086
:10D7680009E00A4B98420BD14FF400400121FFF722
:10D778003BFF4FF400400021BDE80840FFF734BFED
:10D7880008BD00BF0030014000380040003C0040A8
:10D798000B88028810B54C8823438C882343CC8897
:10D7A80023430C8923434C8923438C892343CC8905
:10D7B80002F44152234313439BB20380838B23F427
:10D7C80000631B041B0C83830B8A038210BD838BAD
:10D7D80023F47B6323F00F031B041B0C83830223B6
:10D7E80003848B68F0B5858B022BADB238D0294AFB
:10D7F8008E889468002E14BF02260126240203D5C1
:10D80800946824F400049460D2F88440D2F88470B8
:10D818005268DFF884C002F03F02BCFBF2F2C4F3A6
:10D8280088145443C7F30272B4FBF2F4CA88B2F501
:10D83800007F4FF00A0201D1240A02E07601B4FB0E
:10D84800F6F46243B2FBF3F305330A229BB2B3FB4F
:10D85800F2F303F001021202C3F34F0392B200E0A5
:10D8680000229C1EA4B2FE2C28BF0022CC8828BF10
:10D878000223134323439BB203840B884A882B4318
:10D8880043F4006313438A8813438A8913439BB282
:10D898008383F0BD0038024000127A000023038021
:10D8A80043808380C380038143818381C3810723AD
:10D8B8000382704700230222038043808380C38051
:10D8C800826083817047038819B19BB243F040039B
:10D8D80003E023F040031B041B0C03807047838B79
:10D8E80019B19BB243F4806303E023F480631B0403
:10D8F8001B0C83837047038823F400631B041B0CF1
:10D90800038003889BB20B4303807047B1F5804FB7
:10D91800038803D19BB243F4804303E023F480439C
:10D928001B041B0C038070474FF6FF639942038862
:10D9380003D09BB243F4807303E023F480731B0489
:10D948001B0C03807047838819B19BB243F0040312
:10D9580003E023F004031B041B0C838070478388B7
:10D9680019B19BB243F0100303E023F010031B042A
:10D978001B0C83807047838B23F47B6323F00F0396
:10D988001B041B0C8383022303840B88828BB3F54F
:10D99800007F10B592B205D0002B0CBF4FF48073F6
:10D9A800002301E04FF480734C8822438C888989D6
:10D9B80042F4006222430A4392B21343838310BDA8
:10D9C800808980B2704781817047038819B19BB202
:10D9D80043F4005303E023F400531B041B0C03809F
:10D9E800704703889BB243F4805303807047012932
:10D9F80002D0008B80B27047808A80B27047008A5C
:10DA080080B2704783889BB20AB1194301E023EAC8
:10DA1800010181807047090901238B409BB21AB12B
:10DA2800828892B2134303E0828892B222EA030307
:10DA380083807047038919420CBF0020012070477A
:10DA4800C94389B20181704710B5848800890123D0
:10DA580001F00F0280B213FA02F21040A4B205D00E
:10DA680009098B401C420CBF0020012010BD01F0A9
:10DA78000F0101238B40DB439BB20381704700BF3A
:10DA880008B501214FF48040FFF7BAFD4FF48040FC
:10DA98000021BDE80840FFF7B3BD014B186070478F
:10DAA8000038014001F0030289080A4B023130B501
:10DAB800920053F821500F24944025EA040443F8B7
:10DAC800214053F8214010FA02F2144343F8214050
:10DAD80030BD00BF00380140014B1860704700BFDF
:10DAE800DC002742014B1860704700BF0004274242
:10DAF800024B186AC0F30020704700BF003801408D
:10DB080030B5048C24F001042404240C0484058B0F
:10DB1800048CADB2A4B225F0F305154324F00A0431
:10DB280045EA031544F00104ADB20C4305830484AF
:10DB380030BD30B5048C24F010042404240C048473
:10DB4800048B058C24F44074ADB22405240D25F013
:10DB5800A00544EA022445F0100544EA033445EAE6
:10DB68000115A4B2ADB20483058430BD08B5474B96
:10DB7800984205D101200146FFF742FD01203DE012
:10DB8800B0F1804F05D101200146FFF72DFD01209E
:10DB980076E03F4B984205D102200121FFF724FD92
:10DBA80002206DE03B4B984205D104200121FFF78C
:10DBB8001BFD042064E0384B984205D10820012160
:10DBC800FFF712FD08205BE0344B984205D1102086
:10DBD8000121FFF709FD102052E0314B984205D191
:10DBE80020200121FFF700FD202049E02D4B98421D
:10DBF80009D102200121FFF703FD02200021BDE821
:10DC08000840FFF7FDBC284B984207D14FF48030FD
:10DC18000121FFF7F5FC4FF48030EFE7234B9842E2
:10DC280007D14FF400300121FFF7EAFC4FF4003030
:10DC3800E4E71F4B984207D14FF480200121FFF7FA
:10DC4800DFFC4FF48020D9E71A4B984205D14020D9
:10DC58000121FFF7C9FC402012E0174B984205D17B
:10DC680080200121FFF7C0FC802009E0134B984277
:10DC78000BD14FF480700121FFF7B6FC4FF4807090
:10DC88000021BDE80840FFF7AFBC08BD0000014017
:10DC98000004004000080040000C00400010004054
:10DCA80000140040000401400040014000440140CD
:10DCB8000048014000180040001C004000200040BF
:10DCC8001C4A038890429BB212D002F580629042AF
:10DCD8000ED0B0F1804F0BD0A2F58032904207D021
:10DCE80002F58062904203D002F58062904203D12F
:10DCF8004A8823F0700313430F4A904208D002F574
:10DD08008062904204D023F440730A899BB2134383
:10DD180003804B68C3620B880385064B984203D087
:10DD280003F58063984201D18B7A038601238382AD
:10DD3800704700BF00000140001000404FF0FF3363
:10DD48004360002303800381438083727047018509
:10DD580082827047038823F070031B041B0C0B435B
:10DD68000380704741627047C1627047406A7047DC
:10DD7800008D80B27047038819B19BB243F002034B
:10DD880003E023F002031B041B0C03807047038885
:10DD980019B19BB243F0040303E023F004031B040E
:10DDA8001B0C03807047038819B19BB243F08003B2
:10DDB80003E023F080031B041B0C038070470388D7
:10DDC80023F008031B041B0C038003889BB20B433E
:10DDD80003807047038823F440731B041B0C0380E3
:10DDE80003889BB20B4303807047038819B19BB229
:10DDF80043F0010303E023F001031B041B0C038021
:10DE08007047038C23F001031B041B0C038470B5BB
:10DE1800038C8488028B0D884E8822F073021204CA
:10DE2800120C2A438D8923F002031B0435431B0C73
:10DE3800ADB22B430E4DA842A4B203D005F58065C0
:10DE4800A8420ED1CD894E8A23F008032B438D8832
:10DE580023F004032B430D8A354324F44074ADB2F8
:10DE68002C43848002838A684263038470BD00BFA8
:10DE780000000140038C23F010031B041B0C0384D7
:10DE8800038C828830B5048B0D8824F4E64424047E
:10DE9800240C23F0200344EA05241B048D891B0C61
:10DEA80043EA05134D8843EA0513134DA84292B27D
:10DEB800A4B29BB203D005F58065A84215D1CD89DF
:10DEC80023F080039BB243EA05134FF6BF751D404C
:10DED8008B8845EA03130D8A22F4406242EA8502E0
:10DEE8004D8A42EA85029BB292B282808A68048394
:10DEF8008263038430BD00BF00000140038C23F41B
:10DF080080731B041B0C0384038C828830B5848BBC
:10DF18000D8824F073042404240C23F400731B04D8
:10DF28002C438D891B0C43EA05234D8843EA0523BE
:10DF3800124DA84292B29BB203D005F58065A84263
:10DF480015D1CD8923F400639BB243EA05234FF62C
:10DF5800FF351D408B8845EA03230D8A22F4405281
:10DF680042EA05124D8A42EA05129BB292B28280B9
:10DF78008A688483C263038430BD00BF0000014007
:10DF8800038C23F480531B041B0C0384038C30B5CF
:10DF98008488828B0D8822F4E6421204120C23F442
:10DFA800005342EA05221B048D891B0C43EA053302
:10DFB8004D8843EA05330B4DA842A4B292B29BB2F6
:10DFC80003D005F58065A84205D10D8A24F4804464
:10DFD80044EA8514A4B2848082838A680264038434
:10DFE80030BD00BF000001400023038043808380D0
:10DFF80083608381C38103824382704730B5058C77
:10E008000124ADB28C4025EA040400F1180304840D
:10E0180009B1082907D149084FF68F70CC5820401C
:10E02800C850C8580AE00439C1F34E0148F6FF70D9
:10E03800CC582040C8501202C85892B20243CA5065
:10E0480030BD4163704781637047C16370470164A5
:10E058007047038B23F070031B041B0C0B430383D3
:10E068007047038B23F4E0431B041B0C43EA012392
:10E078009BB203837047838B23F070031B041B0C34
:10E088000B4383837047838B23F4E0431B041B0CEF
:10E0980043EA01239BB283837047038B23F0080371
:10E0A8001B041B0C0B4303837047038B23F400638F
:10E0B8001B041B0C43EA01239BB203837047838B29
:10E0C80023F008031B041B0C0B4383837047838BCB
:10E0D80023F400631B041B0C43EA01239BB28383D4
:10E0E8007047038B23F004031B041B0C0B430383AF
:10E0F8007047038B23F480631B041B0C43EA012342
:10E108009BB203837047838B23F004031B041B0C0F
:10E118000B4383837047838B23F480631B041B0C9E
:10E1280043EA01239BB283837047038B23F0800368
:10E138001B041B0C0B4303837047038B09025B040E
:10E1480041EA53439BB203837047838B23F08003D8
:10E158001B041B0C0B4383837047838B09025B04EE
:10E1680041EA53439BB283837047038C23F0020335
:10E178001B041B0C0B4303847047038C23F0080318
:10E188001B041B0C0B4303847047038C23F02003F0
:10E198001B041B0C43EA01139BB203847047038CD6
:10E1A80023F080031B041B0C43EA01139BB2038476
:10E1B8007047038C23F400731B041B0C43EA0123F0
:10E1C8009BB203847047038C23F400631B041B0C6D
:10E1D80043EA01239BB203847047038C23F4005362
:10E1E8001B041B0C43EA01339BB20384704710B530
:10E1F800048C01238B40A4B224EA03030384038C18
:10E2080012FA01F10B439BB2038410BD10B5048CC4
:10E2180004238B40A4B224EA03030384038C12FA78
:10E2280001F10B439BB2038410BD0023012203803C
:10E2380043808280C38003817047406B7047806B46
:10E248007047C06B7047006C7047038B23F00C035A
:10E258001B041B0C0383038B9BB20B430383704784
:10E26800038B23F440631B041B0C0383038B9BB2B7
:10E2780043EA01239BB203837047F8B50C464988EB
:10E28800A288B4F800E02389054600290CBF0227BC
:10E298000027012A14BF01260226BEF1000F10D163
:10E2A800FFF72EFC2846E188FFF7CFFF28463946BE
:10E2B80032462389FFF73DFCE1882846BDE8F8404F
:10E2C800CEE7FFF736FC2846E188FFF7C9FF284666
:10E2D800394632462389FFF713FCE1882846BDE812
:10E2E800F840B2E7838B23F00C031B041B0C8383D9
:10E2F800838B9BB20B4383837047838B23F44063E8
:10E308001B041B0C8383838B9BB243EA01239BB2C0
:10E3180083837047F8B50D460B88AA884988044658
:10E328003BB92B89FFF7ECFBE9882046BDE8F840AC
:10E338008BE7042B07D12B89FFF7FBFBE9882046E5
:10E34800BDE8F8408CE7082BB5F808C0078C1DD14C
:10E3580027F480773F043F0C0784868B038CB6B282
:10E368009BB226F0F30623F4206346EA0C1C43EA2A
:10E3780001211FFA8CFC89B24CEA020241F4807137
:10E3880082830184E988BDE8F840ABE727F4805729
:10E398003F043F0C0784868B038C26F4407623F4D5
:10E3A800005336055B04360D5B0C46EA022243EA4D
:10E3B800013342EA0C329BB2E98892B243F48053AB
:10E3C80082830384BDE8F84097E74A880B881343A3
:10E3D8008A881343CA8813430A8913434A89134313
:10E3E8008A8913439BB2A0F8443070470023038006
:10E3F80043808380C3800381438183817047B0F861
:10E40800443029B16FEA43436FEA53439BB201E0BA
:10E418005B045B0CA0F844307047838819B19BB249
:10E4280043F0040303E023F004031B041B0C838064
:10E438007047838819B19BB243F0010303E023F0CE
:10E4480001031B041B0C8380704783899BB20AB1AC
:10E45800194301E023EA01018181704781827047F5
:10E46800038A19420CBF002001207047C94389B2B2
:10E4780001827047038A828911EA030092B203D0AD
:10E4880011420CBF002001207047C94389B20182A4
:10E4980070470A43A0F84820704783899BB20AB1A5
:10E4A800194301E023EA010181817047838819B18A
:10E4B8009BB243F0080303E023F008031B041B0C82
:10E4C80083807047038923F007031B041B0C038117
:10E4D8007047038923F070031B041B0C0B43038153
:10E4E80003899BB243F007030381704738B50D4693
:10E4F80011460122602D044602D1FFF71AFB01E004
:10E50800FFF7FEFA238923F070031B041B0C1D433D
:10E51800258123899BB243F00703238138BD0389F2
:10E5280023F070031B041B0C0B4303817047838883
:10E5380023F070031B041B0C838083889BB20B435E
:10E5480083807047038923F007031B041B0C038196
:10E5580003899BB20B4303817047038923F080032F
:10E568001B041B0C038103899BB20B430381704777
:10E5780010B50489E4B20C43144344EA0324A4B25A
:10E58800048110BD10B50446FFF7F2FF23899BB242
:10E5980043F48043238110BD10B50446FFF7E8FF1C
:10E5A800238923F077031B041B0C43F07703238193
:10E5B80010BD70B50489068B058C26F44076ADB283
:10E5C80026F0030624F00704360425F02205240467
:10E5D800360C1543240C46F4807645EA031521438E
:10E5E80046F00106ADB201810683058470BD8388BB
:10E5F80019B19BB243F0800303E023F080031B04AE
:10E608001B0C83807047A0F85010704708B5234B47
:10E61800984205D110200121FEF7F2FF102037E0C3
:10E628001F4B984207D14FF400300121FEF7DCFF61
:10E638004FF4003009E01B4B98420BD14FF4802077
:10E648000121FEF7D1FF4FF480200021BDE80840EA
:10E65800FEF7CABF144B984207D14FF4002001219E
:10E66800FEF7C2FF4FF40020EFE7104B984207D1A6
:10E678004FF480100121FEF7B7FF4FF48010E4E754
:10E688000B4B984209D120200121FEF7B9FF202029
:10E698000021BDE80840FEF7B3BF08BD00100140E7
:10E6A8000044004000480040004C0040005000403A
:10E6B80000140140038ACA889BB223F4405330B542
:10E6C80013430D46038283890989AA8823F4B0532A
:10E6D8000A43698923F00C031B040A431B0C92B2FA
:10E6E80013438381838AAA899BB223F4407313431B
:10E6F80085B0838204466846FEF7A6FE1A4B9C4204
:10E7080003D003F580639C4201D1039B00E0029B88
:10E71800A28912B2002A4FF019012A6801FB03F1FD
:10E7280001DA520000E092006423B1FBF2F1B1FB80
:10E73800F3F21201100903FB1011A08900B200289E
:10E7480006DAC9003231B1FBF3F303F0070305E041
:10E7580009013231B1FBF3F303F00F031A4392B20C
:10E76800228105B030BD00BF001001404FF41653A0
:10E7780003600C2200238380C3800381428183814C
:10E7880070470B88028A10B54C8823438C88C98847
:10E79800234392B20B4322F470629BB21343038269
:10E7A80010BD0023038043808380C3807047838922
:10E7B80019B19BB243F4005303E023F400531B0444
:10E7C8001B0C83817047038B03F47F430383038B04
:10E7D8009BB20B4303837047838929B16FEA434394
:10E7E8006FEA53439BB201E05B045B0C8381704783
:10E7F800838A19B19BB243F4006303E023F40063F6
:10E808001B041B0C83827047C905C90D81807047A2
:10E818008088C005C00D7047038A23F00F031B04CE
:10E828001B0C0382038A9BB20B43038270478389C4
:10E8380019B19BB243F0020303E023F002031B0467
:10E848001B0C83817047838923F400631B041B0C12
:10E85800838183899BB20B4383817047038A23F0AA
:10E8680020031B041B0C0382038A9BB20B43038205
:10E878007047038A19B19BB243F4804303E023F441
:10E8880080431B041B0C0382704783899BB243F0AF
:10E89800010383817047838A19B19BB243F008034F
:10E8A80003E023F008031B041B0C83827047038BCF
:10E8B800DBB20383038B9BB243EA012303837047D4
:10E8C800838A19B19BB243F0200303E023F02003AD
:10E8D8001B041B0C83827047838A19B19BB243F0D7
:10E8E800100303E023F010031B041B0C8382704702
:10E8F800838A23F004031B041B0C8382838A9BB244
:10E908000B4383827047838A19B19BB243F0020399
:10E9180003E023F002031B041B0C83827047838AE5
:10E928009BB20AB1194301E023EA010181827047D1
:10E93800C1F3421310B501F01F01012414FA01F1CB
:10E94800A34201D10C3004E0022B01D1103000E0C9
:10E95800143003680AB1194301E023EA0101016098
:10E9680010BD038819420CBF002001207047C9431D
:10E9780089B201807047012210B501F01F03C1F36D
:10E9880042149A40012C01D1838903E0022C0CBF68
:10E99800038A838A9BB21340028892B243B1090A60
:10E9A800012313FA01F111420CBF0020012010BD10
:10E9B800184610BD090A01238B40DB439BB2038034
:10E9C800704700BF81F0004102E000BF83F00043C0
:10E9D80030B54FEA41044FEA430594EA050F08BFF2
:10E9E80090EA020F1FBF54EA000C55EA020C7FEAB6
:10E9F800645C7FEA655C00F0E2804FEA5454D4EB33
:10EA08005555B8BF6D420CDD2C4480EA020281EAFC
:10EA1800030382EA000083EA010180EA020281EA34
:10EA28000303362D88BF30BD11F0004F4FEA013186
:10EA38004FF4801C4CEA113102D0404261EB410195
:10EA480013F0004F4FEA03334CEA133302D052421B
:10EA580063EB430394EA050F00F0A780A4F10104D7
:10EA6800D5F1200E0DDB02FA0EFC22FA05F2801811
:10EA780041F1000103FA0EF2801843FA05F35941F7
:10EA88000EE0A5F120050EF1200E012A03FA0EFC76
:10EA980028BF4CF0020C43FA05F3C01851EBE371A0
:10EAA80001F0004507D54FF0000EDCF1000C7EEBBD
:10EAB80000006EEB0101B1F5801F1BD3B1F5001FFB
:10EAC8000CD349085FEA30004FEA3C0C04F101041A
:10EAD8004FEA445212F5800F80F09A80BCF1004F43
:10EAE80008BF5FEA500C50F1000041EB045141EAC5
:10EAF800050130BD5FEA4C0C404141EB010111F4C6
:10EB0800801FA4F10104E9D191F0000F04BF014670
:10EB18000020B1FA81F308BF2033A3F10B03B3F14E
:10EB280020020CDA0C3208DD02F1140CC2F10C02DE
:10EB380001FA0CF021FA02F10CE002F11402D8BF3C
:10EB4800C2F1200C01FA02F120FA0CFCDCBF41EA08
:10EB58000C019040E41AA2BF01EB0451294330BDD7
:10EB68006FEA04041F3C1CDA0C340EDC04F11404B4
:10EB7800C4F1200220FA04F001FA02F340EA03008B
:10EB880021FA04F345EA030130BDC4F10C04C4F1D1
:10EB9800200220FA02F001FA04F340EA03002946B1
:10EBA80030BD21FA04F0294630BD94F0000F83F4FB
:10EBB800801306BF81F480110134013D4EE77FEADE
:10EBC800645C18BF7FEA655C29D094EA050F08BF2A
:10EBD80090EA020F05D054EA000C04BF194610460B
:10EBE80030BD91EA030F1EBF0021002030BD5FEA4F
:10EBF800545C05D14000494128BF41F0004130BD77
:10EC080014F580043CBF01F5801130BD01F00045CA
:10EC180045F0FE4141F470014FF0000030BD7FEA3D
:10EC2800645C1ABF194610467FEA655C1CBF0B4638
:10EC3800024650EA013406BF52EA033591EA030F4F
:10EC480041F4002130BD00BF90F0000F04BF002147
:10EC5800704730B54FF4806404F132044FF000057A
:10EC68004FF0000150E700BF90F0000F04BF0021F3
:10EC7800704730B54FF4806404F1320410F0004559
:10EC880048BF40424FF000013EE700BF42004FEA54
:10EC9800E2014FEA31014FEA02701FBF12F07F43D1
:10ECA80093F07F4F81F06051704792F0000F14BFCE
:10ECB80093F07F4F704730B54FF4607401F0004512
:10ECC80021F0004120E700BF50EA010208BF704769
:10ECD80030B54FF000050AE050EA010208BF70475E
:10ECE80030B511F0004502D5404261EB41014FF4C7
:10ECF800806404F132045FEA915C3FF4DCAE4FF0CB
:10ED080003025FEADC0C18BF03325FEADC0C18BFB1
:10ED1800033202EBDC02C2F1200300FA03FC20FA02
:10ED280002F001FA03FE40EA0E0021FA02F114444F
:10ED3800C1E600BF70B54FF0FF0C4CF4E06C1CEA64
:10ED480011541DBF1CEA135594EA0C0F95EA0C0FD9
:10ED580000F0DEF82C4481EA030621EA4C5123EA4C
:10ED68004C5350EA013518BF52EA033541F480117B
:10ED780043F4801338D0A0FB02CE4FF00005E1FB2E
:10ED880002E506F00042E0FB03E54FF00006E1FB78
:10ED980003569CF0000F18BF4EF0010EA4F1FF04BB
:10EDA800B6F5007F64F5407404D25FEA4E0E6D41FB
:10EDB80046EB060642EAC62141EA55514FEAC5200C
:10EDC80040EA5E504FEACE2EB4F1FD0C88BFBCF588
:10EDD800E06F1ED8BEF1004F08BF5FEA500E50F139
:10EDE800000041EB045170BD06F0004646EA0101FF
:10EDF80040EA020081EA0301B4EB5C04C2BFD4EB31
:10EE08000C0541EA045170BD41F480114FF0000E29
:10EE1800013C00F3AB8014F1360FDEBF002001F097
:10EE2800004170BDC4F10004203C35DA0C341BDC11
:10EE380004F11404C4F1200500FA05F320FA04F0E3
:10EE480001FA05F240EA020001F0004221F0004117
:10EE580010EBD37021FA04F642EB06015EEA430E8A
:10EE680008BF20EAD37070BDC4F10C04C4F12005BA
:10EE780000FA04F320FA05F001FA04F240EA02006D
:10EE880001F0004110EBD37041F100015EEA430E3E
:10EE980008BF20EAD37070BDC4F1200500FA05F25E
:10EEA8004EEA020E20FA04F301FA05F243EA0203DD
:10EEB80021FA04F001F0004121FA04F220EA0200EC
:10EEC80000EBD3705EEA430E08BF20EAD37070BD32
:10EED80094F0000F0FD101F00046400041EB010112
:10EEE80011F4801F08BF013CF7D041EA060195F0F4
:10EEF800000F18BF704703F00046520043EB0303AE
:10EF080013F4801F08BF013DF7D043EA060370479A
:10EF180094EA0C0F0CEA135518BF95EA0C0F0CD0A5
:10EF280050EA410618BF52EA4306D1D181EA0301EB
:10EF380001F000414FF0000070BD50EA410606BFE5
:10EF48001046194652EA430619D094EA0C0F02D12A
:10EF580050EA013613D195EA0C0F05D152EA03366F
:10EF68001CBF104619460AD181EA030101F000418D
:10EF780041F0FE4141F470014FF0000070BD41F0D6
:10EF8800FE4141F4780170BD70B54FF0FF0C4CF4B0
:10EF9800E06C1CEA11541DBF1CEA135594EA0C0FCF
:10EFA80095EA0C0F00F0A7F8A4EB050481EA030E1C
:10EFB80052EA03354FEA013100F088804FEA033303
:10EFC8004FF0805545EA131343EA12634FEA0222D1
:10EFD80045EA111545EA10654FEA00260EF0004192
:10EFE8009D4208BF964244F1FD0404F5407402D2E4
:10EFF8005B084FEA3202B61A65EB03055B084FEA75
:10F0080032024FF480104FF4002CB6EB020E75EB71
:10F01800030E22BFB61A754640EA0C005B084FEA99
:10F028003202B6EB020E75EB030E22BFB61A754616
:10F0380040EA5C005B084FEA3202B6EB020E75EB61
:10F04800030E22BFB61A754640EA9C005B084FEAD9
:10F058003202B6EB020E75EB030E22BFB61A7546E6
:10F0680040EADC0055EA060E18D04FEA051545EAD5
:10F0780016754FEA06164FEAC30343EA52734FEA7E
:10F08800C2025FEA1C1CC0D111F4801F0BD141EAF7
:10F0980000014FF000004FF0004CB6E711F4801F5C
:10F0A80004BF01430020B4F1FD0C88BFBCF5E06F3C
:10F0B8003FF6AFAEB5EB030C04BFB6EB020C5FEA4C
:10F0C800500C50F1000041EB045170BD0EF0004EA1
:10F0D8004EEA113114EB5C04C2BFD4EB0C0541EAD3
:10F0E800045170BD41F480114FF0000E013C90E6D0
:10F0F80045EA060E8DE60CEA135594EA0C0F08BF94
:10F1080095EA0C0F3FF43BAF94EA0C0F0AD150EA92
:10F1180001347FF434AF95EA0C0F7FF425AF104625
:10F1280019462CE795EA0C0F06D152EA03353FF44D
:10F13800FDAE1046194622E750EA410618BF52EACA
:10F1480043067FF4C5AE50EA41047FF40DAF52EA9E
:10F1580043057FF4EBAE12E74FF0FF3C06E000BF3B
:10F168004FF0010C02E000BF4FF0010C4DF804CD48
:10F178004FEA410C7FEA6C5C4FEA430C18BF7FEA08
:10F188006C5C1BD001B050EA410C0CBF52EA430C36
:10F1980091EA030F02BF90EA020F0020704710F1B6
:10F1A800000F91EA030F58BF994208BF90422CBF45
:10F1B800D8176FEAE37040F0010070474FEA410C3E
:10F1C8007FEA6C5C02D150EA013C07D14FEA430C5C
:10F1D8007FEA6C5CD6D152EA033CD3D05DF8040BCD
:10F1E800704700BF8446104662468C4619466346FF
:10F1F80000E000BF01B5FFF7B7FF002848BF10F1D6
:10F20800000F01BD4DF808EDFFF7F4FF0CBF01201A
:10F2180000205DF808FB00BF4DF808EDFFF7EAFF96
:10F2280034BF012000205DF808FB00BF4DF808ED51
:10F23800FFF7E0FF94BF012000205DF808FB00BF46
:10F248004DF808EDFFF7CEFF94BF012000205DF8D0
:10F2580008FB00BF4DF808EDFFF7C4FF34BF0120DD
:10F2680000205DF808FB00BF4FEA410212F50012CA
:10F2780015D211D56FF47873B3EB625212D94FEAF5
:10F28800C12343F0004343EA505311F0004F23FADF
:10F2980002F018BF404270474FF00000704750EA34
:10F2A800013005D111F0004008BF6FF000407047F1
:10F2B8004FF00000704700BF4A0011D212F500124B
:10F2C80011D20DD56FF47873B3EB62520ED44FEAB6
:10F2D800C12343F0004343EA505323FA02F0704736
:10F2E8004FF00000704750EA013002D14FF0FF3074
:10F2F80070474FF0000070474FEA4102B2F1E04317
:10F3080024BFB3F5001CDCF1FE5C0DD901F0004C04
:10F318004FEAC0024CEA5070B2F1004F40EB830054
:10F3280008BF20F00100704711F0804F21D113F180
:10F338003872BCBF01F00040704741F480114FEAB9
:10F348005252C2F11802C2F1200C10FA0CF320FA42
:10F3580002F018BF40F001004FEAC1234FEAD3235F
:10F3680003FA0CFC40EA0C0023FA02F34FEA4303C9
:10F37800CCE77FEA625307D150EA01331EBF4FF052
:10F38800FE4040F44000704701F0004040F0FE406D
:10F3980040F40000704700BF4BB942B9002908BFCC
:10F3A800002802D04FF0FF31084600F037B882B08D
:10F3B800EC462DE9005000F01BF8DDF804E002B03F
:10F3C8000CBC7047F8B5144606460F461D4600F0BB
:10F3D80027F804FB01F300FB0535A4FB0023EB1819
:10F3E800069CB21A67EB0303C4E90023F8BD00BF0B
:10F3F800F8B5144606460F461D4600F075F900FBA1
:10F4080005F5A0FB042304FB0155EB18069CB21A72
:10F4180067EB0303C4E90023F8BD00BF704700BFD2
:10F4280000292DE9F0071D46C0F29E800024002D1A
:10F43800C0F2958007460D4616469C46002B3ED1E5
:10F448008A4254D9B2FA82F343B1C3F1200620FAB2
:10F4580006F501FA03F19A4029439840160CB1FBCE
:10F46800F6F597B206FB15114FEA104C07FB05F3AA
:10F478004CEA01418B4209D9891805F1FF3C80F01B
:10F4880015818B4240F21281023D8918C3EB010CB1
:10F49800BCFBF6F306FB13C180B207FB03F740EA97
:10F4A8000140874207D9591E821880F0058197428A
:10F4B80040F20281023B43EA0542002303E08B420B
:10F4C8000AD900231A461046194614B1404261EB86
:10F4D8004101BDE8F0077047B3FA83F3002B40F011
:10F4E80087808C4501D38242ECD80122EBE712B920
:10F4F8000123B3FBF2F2B2FA82F6002E3AD1891A4E
:10F50800150C1FFA82FC0123B1FBF5F705FB171157
:10F518004FEA10480CFB07F648EA01418E4207D92A
:10F52800891807F1FF3802D28E4200F2DA80474686
:10F53800891BB1FBF5F605FB161180B20CFB06FC26
:10F5480040EA0140844507D9711E821880F0B080D6
:10F55800944540F2AD80023E46EA0742B3E7E443F1
:10F56800524263EB430365E7404261EB41014FF0D0
:10F57800FF345CE7B240C6F1200521FA05F320FA12
:10F5880005F701FA06F9150CB3FBF5F847EA09097E
:10F598001FFA82FC05FB18374FEA19410CFB08F3E8
:10F5A80041EA0747B040BB420AD9BF1808F1FF310A
:10F5B80080F09580BB4240F29280A8F10208BF1803
:10F5C800FE1AB6FBF5F305FB13611FFA89F90CFB6C
:10F5D80003F649EA01418E4206D95F1E891878D29E
:10F5E8008E4276D9023B8918891B43EA08438BE788
:10F5F800C3F1200726FA07F80CFA03F248EA020CCE
:10F6080021FA07F105FA03FA4FEA1C4920FA07F52F
:10F61800B1FBF9F845EA0A0509FB18172A0C1FFA85
:10F628008CFA0AFB08F142EA0747B94206FA03F6E0
:10F6380009D917EB0C0708F1FF324ED2B9424CD961
:10F64800A8F1020867447F1AB7FBF9F209FB1271A7
:10F65800ADB20AFB02FA45EA01418A4507D9551EAF
:10F6680011EB0C0137D28A4535D9023A614442EA96
:10F6780008424FEA124C1FFA86F808FB0CF7360CC2
:10F6880095B208FB05F806FB057505EB184506FB62
:10F698000CFCAF4288BF0CF5803CCAEB01010CEBB7
:10F6A8001546B14212D309D000230CE76546EDE6B2
:10F6B8000E4646EA074206E70B46FCE61FFA88F8BC
:10F6C80000FA03F308EB0545AB42EDD2013A0023FB
:10F6D800F9E63B4688E72A46C9E79046B3E78846F5
:10F6E8006EE7023F891823E72DE9F00F1446054617
:10F6F8000E46002B3FD18A424AD9B2FA82F343B16F
:10F70800C3F1200025FA00F201FA03F69C401643E3
:10F718009D40210CB6FBF1F22F0CA0B201FB126C3C
:10F7280000FB02F347EA0C46B34208D9571E3619C4
:10F7380080F0FF80B34240F2FC80023A3619F61A94
:10F74800B6FBF1F301FB1361ADB200FB03F045EA30
:10F758000141884207D95E1E091980F0EC80884271
:10F7680040F2E980023B43EA024200231046194670
:10F77800BDE8F00F70478B4243D8B3FA83F4002CEE
:10F7880042D18B42234601D382423BD80122EDE786
:10F7980012B90123B3FBF2F4B4FA84F2002A40F060
:10F7A8008A80091B260CA7B20123B1FBF6F006FBE1
:10F7B80010114FEA154C07FB00F24CEA01418A424E
:10F7C80007D9091900F1FF3C02D28A4200F2D3801E
:10F7D8006046C2EB010CBCFBF6F206FB12C1ADB2EF
:10F7E80007FB02F745EA0145AF4207D9511E2C191C
:10F7F80080F0A380A74240F2A080023A42EA004289
:10F80800B4E700231A46B1E7C4F1200722FA07F645
:10F8180003FA04F3334321FA07FA4FEA134C01FAC7
:10F8280004FB20FA07F141EA0B0BBAFBFCF70CFBCF
:10F8380017A61FFA83F84FEA1B4508FB07F945EAA4
:10F848000645A94502FA04FA04D97A1EED18C0F053
:10F8580088801746C9EB0505B5FBFCF60CFB16526C
:10F868001FFA8BFB08FB06F84BEA0241884503D9CF
:10F87800721EC91870D3164646EA0742170C1FFABB
:10F888008AFC0CFB07F695B24FEA1A430CFB05FC01
:10F8980003FB056505EB1C4503FB07F3AE4288BF78
:10F8A80003F58033C8EB010103EB1543994250D3AC
:10F8B80047D000235AE79440C2F12008260C20FACA
:10F8C80008F721FA08F501FA02F9B5FBF6F847EA54
:10F8D800090906FB1855A7B24FEA194C4CEA054C22
:10F8E80007FB08F3634500FA02F509D91CEB040C81
:10F8F80008F1FF323DD263453BD9A8F10208A44480
:10F90800C3EB0C02B2FBF6F306FB13201FFA89F9CE
:10F9180007FB03F249EA00418A4206D9581E091931
:10F9280025D28A4223D9023B0919891A43EA084396
:10F938003BE73A4603E7334615E70A4642EA004200
:10F9480014E71FFA8CF100FA04F001EB0545A84210
:10F95800AFD2013A002309E788458CD9023EC9187D
:10F968008AE7A9457FF675AF023FED1872E70346AF
:10F97800DBE79046C4E7023809192AE7002103E0CB
:10F988000A4B5B584350043109480A4B42189A42C3
:10F99800F6D3094A02E0002342F8043B074B9A4297
:10F9A800F9D3FAF7C5F900F00DF87047E4A5050892
:10F9B80000000020FC0C0020000D0020EC5100206D
:10F9C800FEE70000A34BF7B54FF4FA661E60A24AA3
:10F9D800A24BA34F1A60A34AA34B1A60A34B42F24F
:10F9E80010721A60A24B64241C6001233B70F8F764
:10F9F800CAFFA04B00251D70F8F764F9F6F764FA02
:10FA0800F6F76EFAF6F77CFAF7F778F82046F7F784
:10FA1800F5FCF7F799F82046F7F7F0FCF8F738F90E
:10FA2800F7F76EFFF7F7F8FC2046F7F7E7FCFAF769
:10FA3800C1FA2046F7F7E2FC4FF4FA50F7F74AFC10
:10FA48002046F7F7DBFCF6F7B1FF2046F7F7D6FCC0
:10FA58002846F7F7B5FD8848F7F7D0FCF4F7E8FA39
:10FA68002046F7F7CBFC854B03F1100229468DE8B9
:10FA7800240028465A681B68F4F7E0FC3046F7F77C
:10FA8800BDFC2846F4F75AFF4FF6FF70F4F76CFFF9
:10FA9800032132207A4A2B46F5F77EF89620794AD8
:10FAA8008C212B46F5F778F89620A021764A2B462C
:10FAB800F5F772F8754A2B469620B421F5F76CF8DD
:10FAC800F8F718FF5021DC20F8F7E7FE3046F7F783
:10FAD80095FC6F4A2B46DC212846F5F75DF86D4802
:10FAE800F7F78CFC2046F7F789FCF6F707FD204668
:10FAF800F7F784FC9FED680AF7F77AFD2046F7F7D9
:10FB08007DFCF7F7A3FCF5F711FB2046F7F776FC29
:10FB180014200146F6F760FA2846F6F7B3FA2046AD
:10FB2800F7F76CFCF6F734FC2046F7F767FCF6F7B6
:10FB3800DDFF2046F7F762FCF6F730FD00B13D70B7
:10FB4800F6F738FD08B1F8F77FFE544B00241C7017
:10FB5800F1F702FDF5F7A0FA08B9514802E0514B58
:10FB680051481C70F1F713FDF5F70AFFF8F7C5FBCC
:10FB7800F8F7F8FBF9F75EF9F8F7ACF9F8F787FE4C
:10FB8800FAF78AF9F8F7D6FE484B494D494C8028D0
:10FB980014BF4FF480504FF480601880324B1A68BD
:10FBA8002E4B1B68D21A314B1B6892FBF3F2424B67
:10FBB8002E461A80F6F714FD2B7833B1012B02D1AB
:10FBC800F7F7CCFE01E0F7F7F1FE00273770F8F7FA
:10FBD80047F8F3F7AFFCF9F715FA237813B1277054
:10FBE800F2F72AF9334B5B781BB100236370F1F706
:10FBF800C5FD324B1A8812B2012A13D130484FF48E
:10FC08000051FDF75EF9A3780BB9F9F727FAF7F772
:10FC1800B9FF00222A484FF40051FDF752F9274B4B
:10FC280000221A80E37843B1F8F764FEF0209621A9
:10FC3800F8F733FE2348F7F7D7F9234F3846FBF791
:10FC4800A4FC0028B6D03B78112BB3D1F8F774FD8B
:10FC5800B0E700BF803E0020E0673500B03E0020DE
:10FC6800380F002080C3C901CC440020A4440020E0
:10FC7800603E00202446002000127A00607D0108C2
:10FC8800389E0508529E05085F9E05086B9E05086C
:10FC9800749E0508002D31010000FA44903E0020B2
:10FCA80068110020483E002054130020AC3E00207C
:10FCB800A8440020080E0020EC470020EC0D00208E
:10FCC8000008024040420F00493E002010B4314C69
:10FCD8000180B1F5807F44608270C37052D00DD925
:10FCE800B1F5806F39D017D9B1F5006F2ED0B1F5C5
:10FCF800805F24D0FF2040B210BC704720293AD042
:10FD080014D9402930D08029F4D123494FF020124A
:10FD1800C26081600020EEE7B1F5007FEAD11F4B99
:10FD28004FF00811C16083600020E4E71029E1D199
:10FD38001B494FF00122C26081600020DBE7194BAC
:10FD48004FF00111C16083600020D4E7164A4FF0DC
:10FD58000213C36082600020CDE714494FF00412FB
:10FD6800C26081600020C6E7114B4FF04011C160AE
:10FD780083600020BFE70F4A4FF08013C3608260A2
:10FD88000020B8E70C4A4FF01013C36082600020CF
:10FD9800B1E700BF889C0408C68C0508968C050846
:10FDA800868E0508888C05088A8C05088E8C0508BF
:10FDB800068D0508868D0508A68C05082DE9F00F27
:10FDC800B2B02E9030932E9B00882E9C5B68309F9B
:10FDD800A4682D90451E03EB4506BF082093289480
:10FDE8002C952F911F921E96319700F03A814FEA79
:10FDF800900A4FEACA0B00F003002F99299003F1EB
:10FE0800080504EB0B00CDF884A0CDF8A8B019952F
:10FE18001A921B97189617912B90179A189E138869
:10FE28003380B2F802C0A6F802C09488B480D7889C
:10FE3800F78008361896219F199E0832179256F8AF
:10FE4800041C56F8082C4FF0000A4FF0000B002F46
:10FE580000F06982CDE904ABCDE906ABCDE902AB90
:10FE6800CDE900AB289CBC46029BDDF80C902568C8
:10FE7800C2FBC5394FF0000848EA030ACB46CDE972
:10FE880002AB049BDDF814B0C1FBC53BCDF824B030
:10FE9800CDF82080DDE908ABC1EA02004AEA030A8E
:10FEA800CDE904AB069BDDF81CB03268C0FBD53B3E
:10FEB800CDF82CB0CDF82880DDE90AABC2EA0107FD
:10FEC8004AEA030ACDE906AB9DE80108C7FBD50B52
:10FED800CDF834B0CDF83080DDE90CAB4AEA000A41
:10FEE80063680298CDE900AB0834DDF80CB0C1FBBB
:10FEF800C30BCDF83CB0CDF83880DDE90EAB4AEA4B
:10FF0800000ACDE902AB71680498DDF814B0C2FBB1
:10FF1800C30BCDF844B0CDF84080DDE910AB4AEA18
:10FF2800000ACDE904AB0698DDF81CB0C7FBD30B7B
:10FF3800CDF84CB0CDF84880DDE912ABC1EA020536
:10FF48004AEA000ACDE906AB9DE80108C5FBD30BD8
:10FF5800CDF854B0CDF85080DDE914AB08364AEA44
:10FF6800000ABCF1010CCDE900AB7FF47DAF2A9DFE
:10FF780019982B9B2E18299F002F35D01868039F9E
:10FF8800029BC2FBC03700241D971C94DDE91C4569
:10FF980044EA0304CDE90245049B059DC1FBC03535
:10FFA800002723952297DDE9224544EA0304CDE999
:10FFB8000445C1EA0203079D069AC3FBD02525958F
:10FFC8002497DDE9244544EA02043368C3EA0101C1
:10FFD800CDE9064553465D46C1FBD03527952697A2
:10FFE800DDE926AB4AEA030A069A029C0499039DB6
:08FFF800079FD30B059AE60BED
:020000040801F1
:10000000C90B46EA454043EA474441EA424604F305
:100010000F0500F30F0C199BCCEA054706F30F0000
:100020001A9D1B9E2F604FEADA3A08334AEA4B4B7F
:100030000BF30F04C0EA04426A600835711E19937D
:100040001A951B917FF4EDAE319A2F9E1E991F9B3E
:10005000DDF880B0D00037180D182F970BEB000A91
:100060001F181E951F97CDF880A0DDF8C0C01CF0AA
:10007000030BCDF820B000F086802D9BDDF8BC800E
:10008000CDF808B05808DDF880A0DDF8A0B00690E3
:10009000CDF81080049A1E9E32F8025B069826F86E
:1000A000025B0492BAF80270BBF80230BAF8002082
:1000B000BBF800401E9617FB03F112FB04F6451E29
:1000C0004FEAE17711EB06082B4605F0010047EBFC
:1000D000E6790AF104020BF10401002D3BD0A8B12E
:1000E000B2F800C0BBF80470548848881CFB07F5C0
:1000F00018EB050749EBE57614FB00F917EB090847
:1001000046EBE97904320431013B24D00F88B2F880
:1001100000C0568848888C8895881CFB07FC18EB23
:100120000C0816FB00F7D088CE8849EBEC7C15FB59
:1001300004F518EB07084CEBE77918EB050710FB03
:1001400006FC49EBE57417EB0C0844EBEC7908323C
:100150000831023BDAD11F9A02994FEAD83545EAB5
:10016000494404F30F0322F8023B4F1E0AF1020A2E
:100170001F9202978ED1DDF880A0DDF820B00AEB47
:100180004B0ACDF880A02C9E2E98B50840683FD031
:10019000209F47EA000212F0030F00F1080307F165
:1001A000080214BF002101219F4298BF904294BFD2
:1001B00000260126314277D097E8420001600121F4
:1001C0006C1EA942466004EA010419D044B192E8C9
:1001D0001200196002215C6008320833A9420FD076
:1001E00092E850001C605E60966802F1080BD268CD
:1001F0009E600231DA601033A9420BF10802EFD1A0
:10020000DDF880C0ED000CEB050B4019CDF880B097
:100210002C9C14F0030343D05A085400002A00F029
:100220008E80209D40EA050717F0030F209F14BF22
:1002300000250125011D3E1D012B94BF002505F061
:1002400001058F4298BFB04294BF002101210D42A9
:1002500075D039689200BF18A342016020971044FE
:10026000C4EB03011CD0209B013933F8024B0A4632
:1002700020F8024B01F0010192B129B133F8021BC1
:10028000013A20F8021B0BD01C46014634F802CB81
:1002900021F802CB5D88A31C4580881C023AF3D16B
:1002A00032B0BDE8F00F7047B7F800C0A0F800C04A
:1002B0007C884480BE888680691EFE880C46BA46CB
:1002C00001F00101C680002C9AD089B1B2F800B0CB
:1002D000A3F800B051885980B2F804C0A3F804C054
:1002E000B2F806B00832A3F806B00833013C87D054
:1002F00016881E8051885980B2F804B0A3F804B063
:10030000B2F806C0A3F806C016891E8103F1080BD7
:100310005189ABF802109389ABF80430D6891032BA
:10032000023C0BF10803ABF80660E1D168E7289BBB
:10033000CDE904ABCDE906ABCDE902AB1FE619462A
:1003400091E700BF2DE9F00F9CB006780F900F9C4D
:1003500040880F9DA4686D681990B3FBF6FA471E9C
:100360004FEA5A0804EB4709AAEB480340460A94AF
:100370000D951A97CDF86C800C911492CDF82C90B5
:100380001193002800F0B5811746199A199CCDF8F1
:1003900048809108CA00159104F00303A918179228
:1003A000169310971891760075084FEA450C002DAA
:1003B00000F03B840B9FDDF8308047EA080010F026
:1003C000030F14BF0021012108F10404381D012E80
:1003D00094BF002101F00101804598BFA74294BF5E
:1003E0004FF000094FF0010911EA090F00F01D84D8
:1003F000BB46D8F8002001236F1EAB42CBF800208B
:1004000007EA03072146024614D237B124680223C3
:100410000431021DAB4204600CD20C46104654F865
:10042000047B40F8047B496802335160211D021DA2
:10043000AB42F2D3DDF83080DDF82CB04FEA4C054A
:10044000664508EB05020BEB0503CCEB06001DD05F
:10045000013832F802CB014623F802CB00F001004C
:10046000A1B128B132F8029B013923F8029B0DD0CB
:1004700014461F4634F8029B27F8029BB2F802A0EC
:10048000A21CA3F802A0BB1C0239F1D10C9ADDF822
:100490003CC00B989CF80080710053180A9E0C9386
:1004A000159BCDF84C80451806EB48020B950E9233
:1004B000002B00F0B18300240025CDE90445CDE9EF
:1004C000024507930D9913460A9AB3F804A0B2F8AF
:1004D00006B0CDF804A0B3F806A00E881588CDF8B4
:1004E00020B0CDF824A0DDE902AB15FB06F51AEB30
:1004F000050A4BEBE57BCDE902AB1F884888B2F8D3
:1005000002C0B3F80290B2F804808C88CDF818804D
:10051000DDE904AB16FB07F61AEB060A4BEBE67BAC
:10052000DDE902671CFB00F5761910FB09F047EBCB
:10053000E5771AEB000A4BEBE07BCDE902ABDDF887
:1005400018B0DDF804C0B1F80680099D1BFB04F06B
:1005500016EB000A47EBE07BDDE9026714FB0CF4C5
:10056000361947EBE477089C14FB08F00831083291
:1005700008331AEB000418FB05F84BEBE0750798FD
:1005800016EB080A47EBE87B0138CDE90245CDE9D7
:1005900004AB079099D1179E0E9C0A9B1899A71936
:1005A0009A190E97169F002F73D00E9B31F8020BED
:1005B00032F8024B33F8026BDDE90289DDE904AB66
:1005C00014FB00F47D1E10FB06F618EB040849EB43
:1005D000E4791AEB060A4BEBE67B2F4605F00100A7
:1005E000CDE90289CDE904AB002D52D0002873D0AB
:1005F00031F8024B32F8020B33F8025B10FB04F6C1
:1006000014FB05F0DDE90245DDE90489A41945EB99
:10061000E67518EB000849EBE079013FCDE90245AA
:10062000CDE9048935D0C246CB46DDE902890D46C5
:1006300014460497214628461A4630F8026B31F8D2
:10064000027B32F802CB6D8864885B8817FB06F763
:1006500018EB070816FB0CF649EBE7791AEB0607CF
:1006600014FB05FA4BEBE67B15FB03FC8C1C931C7F
:100670000499851C18EB0A0849EBEA7917EB0C0A78
:100680004BEBEC7B8A1ECDE902890492D2D1CDE9F5
:1006900004AB029D03990498DDF828A0059BEA0BA2
:1006A000109D42EA4148129908F30F09A5F80090FD
:1006B000DDF84C90C70B0AEB8908281D4A1E47EA53
:1006C0004346CDF8288006F30F0410906C801292F8
:1006D0000AD00F9C267866E6DDE904AB0D46144689
:1006E0000497DDE90289A5E7149F1B9B07EB8306AE
:1006F0001496119F002F00F0A681DDF864B0DDF89C
:100700006480DDF834C04FEA9B09CDF81C904FEAB5
:10071000C90908F0030A0CEB090BCDF82090CDF8BD
:1007200010A0CDF824B0DDF83CC09CF8006075083E
:100730004FEA450C002D00F07E820C990B980B9F20
:1007400040EA010414F0030F14BF002201220C1D23
:100750000430012E94BF002202F00102814298BFB2
:10076000A74294BF002301231A4200F06482BA46D4
:1007700001230F68691EAB42CAF80070024601EA05
:100780000307214614D237B127680223211D021D19
:10079000AB4207600CD20C46104654F8047B40F87C
:1007A000047B496802335160211D021DAB42F2D324
:1007B000DDF83090DDF82C804FEA4C05664509EBFA
:1007C000050208EB0503CCEB06001DD0013832F81A
:1007D00002BB014623F802BB00F00100A1B128B121
:1007E00032F8025B013923F8025B0DD014461F4634
:1007F00034F802AB27F802ABB2F802C0A21CA3F88F
:1008000002C0BB1C0239F1D1DDF82CA0DDF830B0FC
:10081000079876000AEB060C0BEB0608CDF82CC007
:10082000CDF83080002800F0F0810A9ADDF834809D
:100830005788B2F800A0DDF828909488B9F806909F
:10084000B8F8062084460D9841880588B8F8040059
:1008500017FB01F61AFB05F3B3461BEB03014FEA46
:10086000E67714FB00F047EBE3750F180A9B19FBC2
:1008700002F145EBE0750CF1FF3617EB010AB146CA
:1008800006F0010008F1080203F1080345EBE17BE3
:10089000002E00F0858048B3DDF834C01E88BCF817
:1008A00008405888518897889D88B2F80680B3F828
:1008B00006C016FB04F41AEB040A10FB01F14BEB23
:1008C000E4761AEB010415FB07FB46EBE17014EB31
:1008D0000B011CFB08F640EBEB740832083311EBFC
:1008E000060A44EBE67BB9F1010959D0CDE902AB28
:1008F000CB46B3F80080B3F808901688CDF838904E
:1009000018FB06F6DDE902895D885488988891888D
:10091000B2F806C0DF88B2F808A015FB04F418EBA3
:10092000060810FB01F149EBE67918EB040817FB08
:100930000CF749EBE47918EB010849EBE17918EB86
:10094000070849EBE779CDE90289DDF838905D8940
:10095000548998899189B2F80EC0DE8919FB0AF78B
:10096000DDE9028915FB04F418EB070810FB01F11F
:1009700049EBE77918EB040849EBE47916FB0CF630
:1009800018EB010449EBE17510321033A01945EB67
:10099000E671BBF1020BCDE90201AAD182468B467A
:1009A0000DF1200898E816006318049D9DB332F8F5
:1009B00002CB33F8026B16FB0CF4013D1AEB040A70
:1009C000294605F001004BEBE47B25B358B132F822
:1009D000028B33F8020B10FB08F71AEB070A4BEBFC
:1009E000E77B691E17D01446184634F8025B30F8CE
:1009F000027B52885B8817FB05F81AEB08064BEB65
:100A0000E87713FB02FBA21C831C16EB0B0A47EBD7
:100A1000EB7B0239E7D10F9DDDF8508095F800C0DF
:100A20000A9A119E4FEADA3343EA4B4404F30F006B
:100A300028F8020B02EB4C07711E0A97CDF8508084
:100A400011917FF470AE1A9E0F9CB508A06842D039
:100A50000A9F47EA000616F0030F07F1080200F1AB
:100A6000080314BF002101219F4298BF904294BF08
:100A70004FF0000A4FF0010A11EA0A0F7FD097E801
:100A80004200016001216C1EA942466004EA010493
:100A900019D044B192E81200196002215C6008325A
:100AA0000833A9420FD092E850001C605E6096683F
:100AB00002F10804D2689E600231DA601033A94264
:100AC00004F10802EFD1DDF828A0ED000AEB0509DA
:100AD0004019CDF82890DDF868A01AF003034AD039
:100AE0005A085400002A00F0A480DDF828B040EA3B
:100AF0000B0515F0030F14BF002501250BF10406AB
:100B0000011D012B94BF002505F001058B4598BF01
:100B1000B04294BF4FF0000C4FF0010C15EA0C0FDF
:100B200000F08780DBF8001092009344A34201603C
:100B3000CDF828B01044C4EB03011CD00A9B013946
:100B400033F8024B0A4620F8024B01F0010192B142
:100B500029B133F8021B013A20F8021B0BD01C46C6
:100B6000014634F802CB21F802CB5D88A31C4580F6
:100B7000881C023AF3D11CB0BDE8F00F7047B7F8FB
:100B80000090A0F800907C884480BE888680691E12
:100B9000FE880C46B84601F00101C680002C92D0B8
:100BA00091B111881980B2F802C0A3F802C0B2F85E
:100BB00004A0A3F804A0B2F806900832A3F80690A7
:100BC0000833013C3FF47FAF11881980B2F802C0AE
:100BD000A3F802C0B2F80490A3F80490B2F806A0FB
:100BE000A3F806A016891E8103F1080C5189ACF800
:100BF00002109389ACF80430D6891032023C0CF113
:100C00000803ACF80660DFD15DE70D9A0A9B4FF050
:100C1000000A4FF0000BC8E600260027CDE9046764
:100C20000A9A0D99CDE90267BCE430460B9B0C9AF9
:100C30000EE4194682E730460B9B0C9AC6E500BFCE
:100C400000B553EC102B42F2FB1223F00043C3F625
:100C5000E972934285B026DD4FF6FF72C7F6EF7258
:100C600093420BDD51EC100B02460B46FDF7B2FE32
:100C700002460B4643EC102B05B000BD684600F061
:100C8000BFFB00F0030001289DED000B9DED021B52
:100C90001AD0022810D0F8B900F0D2FE53EC102B75
:100CA00010461946E4E79FED101B00F0C9FE53EC17
:100CB000102B10461946DBE700F0C2FE53EC102B58
:100CC000104603F10041D3E701F0F6FB53EC102B83
:100CD000104603F10041CBE7012001F0EDFB53EC9E
:100CE000102B10461946C3E700000000000000006A
:100CF0002DE9F04759EC108BC9F30A56A6F57E741E
:100D0000073C132C4D46CA46474626DC002C4FDBD9
:100D10004FF6FF76C0F20F0646FA04F606EA09051A
:100D200055EA080517D044A3D3E9002351EC100B72
:100D3000FDF752FE00220023FEF790FA00284AD069
:100D4000B9F1000F6EDB2AEA060A4FF0000853469D
:100D5000424643EC102BBDE8F087332C0CDDB4F594
:100D6000806FF8D151EC100B3A460B46FDF734FE7C
:100D700041EC100BBDE8F087A6F58265033D4FF00E
:100D8000FF3323FA05F515EA080FE4D02AA3D3E9C7
:100D9000002351EC100BFDF71FFE00220023FEF78D
:100DA0005DFAC0B1B9F1000F1CDB28EA050813E0B9
:100DB00021A3D3E9002351EC100BFDF70DFE002217
:100DC0000023FEF74BFA38B1B9F1000F1BDB4FF0EF
:100DD0000008C24600E0CA465346424643EC102B88
:100DE000BDE8F087142C09D0C6F5866303334FF0B5
:100DF000010808FA03F818EB0708D6D30AF1010A2C
:100E000028EA0508E8E729F0004848EA07084FF013
:100E1000000AD045CBF6F07A08BFCA4618BF4FF09B
:100E20000008D9E74FF4801343FA04F409EB040AED
:100E300089E700BFAFF300809C7500883CE4377EF3
:100E400000B553EC102B42F2FB1223F00043C3F623
:100E5000E972934285B027DD4FF6FF72C7F6EF7255
:100E600093420BDD51EC100B02460B46FDF7B2FD31
:100E700002460B4643EC102B05B000BD684600F05F
:100E8000BFFA00F0030001289DED000B9DED021B51
:100E90001DD0022812D008BB012001F00DFB53EC3D
:100EA000102B10461946E3E700209FED111B01F0BF
:100EB00003FB53EC102B10461946D9E7012001F033
:100EC000FBFA53EC102B104603F10041D0E700F081
:100ED000B7FD53EC102B10461946C9E700F0B0FDE2
:100EE00053EC102B104603F10041C1E7AFF3008033
:100EF000000000000000000000F0E6B8D0B52DEDC5
:100F0000048BB0EE408AF0EE608A3C4C8AB000F070
:100F1000DBF994F90030B0EE409AF0EE609A0133BC
:100F200035D0B0EE480AF0EE680A01F04FFD002817
:100F30002DD051EC180B00220023FEF77BF930B3C3
:100F40002F4B24780193002308938DED028B8DEDB8
:100F5000048B002C23D000270026CFF6F07751EC2D
:100F6000180B00220023CDE90667FEF74FF9002891
:100F700025D002239C42009336D0684601F05EFDE6
:100F8000002831D0089B002B27D19DED069BB0EEA9
:100F9000490AF0EE690A0AB0BDEC048BD0BD4FF6E9
:100FA000FF774FF06046CCF2EF7751EC180B002240
:100FB0000023CDE90667FEF729F90028D9D10123DE
:100FC000022C009315D0684601F038FD88B10D4819
:100FD00001F036FD8DED060BD4E701F0EFFF089B25
:100FE0009DED069B0360D2E701F0E8FF222303603A
:100FF000C8E701F0E3FF21230360E8E7380400209D
:10100000E8A0050848A3050810B52DED048BB0EE47
:10101000408AF0EE608A294C8AB000F02DFC94F9E9
:101020000030B0EE409AF0EE609A01332BD0B0EE73
:10103000480AF0EE680A01F0C9FC20B351EC180B25
:1010400000220023FEF7ECF8E8B11D4B2478019351
:1010500001230093002308938DED048B8DED028B0B
:10106000CCB10020002102460B46FDF791FF022C77
:10107000CDE9060115D101F0A1FF21230360089BF2
:10108000ABB99DED069BB0EE490AF0EE690A0AB0D5
:10109000BDEC048B10BD0022002343EC172B8DED1B
:1010A000067B684601F0CAFC0028E8D1E3E701F0BE
:1010B00085FF089B9DED069B0360E4E73804002054
:1010C000F0A0050800000000F8B5B0EE407AF0EEA0
:1010D000607A53EC112B544210461D46002125F036
:1010E0000047044353EC102B47EAD474C7F6F07161
:1010F0008C4216463DD85442344323F0004242EA23
:10110000D4748C4235D805F1404101F5801101437A
:101110004FD0AC1704F00204164344EAD37435D020
:10112000384341D00021C7F6F0718F424FD00021E3
:10113000C7F6F0718A4237D0D21B12153C2A42DC26
:10114000002D7DDB53EC112B51EC170BFDF720FF2D
:1011500041EC100B01F030FC01F06AFA51EC100B7D
:10116000012C68D0022C57D0002C48D141EC170B31
:1011700007E051EC170B53EC112BFDF72DFC41EC64
:10118000170BB0EE470AF0EE670AF8BD032CC7D87C
:1011900001A151F824F000BF831101088311010857
:1011A000C1110108BB110108002B25DB9FED307B2D
:1011B000E7E7BDE8F84001F03BBA9FED2F7BE0E7A1
:1011C0009FED2F7BDDE72AA1D1E90001C8E7BA42F4
:1011D0003CD0032CABD801A151F824F0F311010845
:1011E000ED110108C1110108BB1101089FED267B1B
:1011F000C7E79FED277BC4E79FED277BC1E730A3BF
:10120000D3E90023FDF7E6FB1DA3D3E90023FDF797
:10121000E1FB41EC170BB4E729A3D3E90023FDF769
:10122000D9FB02460B4616A1D1E90001FDF7D2FB1E
:1012300041EC170BA5E701F1004141EC170BA0E7CA
:101240003C32BFF67FAF0020002189E7032CABD8EA
:10125000DFE804F00B0805029FED117B91E79FED9D
:10126000127B8EE79FED127B8BE79FED137B88E768
:10127000182D4454FB21F93F182D4454FB2109C07B
:10128000182D4454FB21094000000000000000809C
:101290000000000000000000182D4454FB21F9BF9D
:1012A000D221337F7CD902C0D221337F7CD9024046
:1012B000182D4454FB21E9BF182D4454FB21E93F6C
:1012C000075C143326A6A13C2DE9F84F55EC104BD2
:1012D000B5F5801F2F4622DA25F00043234368D05E
:1012E000002D2046294670DB00230022C4F2503333
:1012F000FDF724FD4FF6FF730F46C7F6EF739F42CD
:1013000004460D466FF0350210DD20462946224680
:101310002B46FDF761FB41EC100BBDE8F88F4FF653
:10132000FF73C7F6EF7300229F42EEDC3B15A3F577
:101330007E73073B9A18D60F901927F07F47C6F5A2
:101340007E76FDF795FC073627F4700747EA0655C9
:1013500045EC104B8046894601F00AFC4046494660
:1013600021A3D3E9002355EC104BFDF7E7FC20A3A4
:10137000D3E9002382468B4640464946FDF7DEFC12
:101380001DA3D3E9002306460F4620462946FDF754
:10139000D5FC02460B4630463946FDF71DFB02469A
:1013A0000B4650465946FDF717FB41EC100BBDE8C4
:1013B000F88F00210020CCF2503100220023FDF7ED
:1013C000E7FD41EC100BBDE8F88F22462B46FDF7F8
:1013D00001FB00220023FDF7DBFD41EC100BBDE813
:1013E000F88F00BFAFF3008000609F501344D33FDD
:1013F000362BF111F3FE593D0EE526157BCBDB3F75
:101400002DE9F04F53EC102B42F2FB1223F0004475
:10141000C3F6E97294428FB01E46074640F3AA8095
:101420004DF67B13C4F202039C422ADC002E51ECE1
:10143000100BDDA3D3E9002340F3CA81FDF7CAFAFC
:1014400042F2FB13C3F6F9739C428046894600F0D2
:10145000AA80D7A3D3E90023FDF7BCFA0D460446C2
:101460002B462246C7E9004540464946FDF7B2FAF9
:10147000CFA3D3E90023FDF7ADFA0125C7E90201A7
:1014800081E042F2FB13C4F239139C4240F3AA807C
:101490004FF6FF73C7F6EF739C4278DC4FEA245A8D
:1014A000AAF5826AAAF1060A51EC100BA4EB0A53C2
:1014B00019461D460446FDF7DBFEFDF7D9FB8046C5
:1014C000894642464B4620462946CDE90889FDF724
:1014D00081FA00230022C4F27013FDF72FFC0D46A1
:1014E0000446FDF7C5FEFDF7C3FB8046894620464E
:1014F000294642464B46CDE90A89FDF76BFA00239F
:101500000022C4F27013FDF719FC002204460D46B8
:101510000023CDE90C45FDF779FE002800F07B8122
:101520004046494600220023FDF770FE03240AAD21
:10153000013C40B175E9020100220023FDF766FE7F
:10154000013C0028F6D12346022400949E4C08A8B2
:1015500039465246019400F0ABFB002E054612DAE4
:101560007A68FB6802F1004203F100437A60FB6095
:10157000454208E00022002343EC172B87ED000BC7
:1015800080ED027B002528460FB0BDE8F08F51ECBE
:10159000100B02460B46FDF71DFA0025C7E90201B4
:1015A000C7E90001EFE77AA3D3E90023FDF712FAB8
:1015B00079A3D3E9002380468946FDF70BFA0D464F
:1015C00004462B462246C7E9004540464946FDF7FA
:1015D00001FA71A3D3E90023FDF7FCF90125C7E95E
:1015E0000201D0E701F0E8F959EC108B6CA3D3E9C4
:1015F000002340464946FDF7A1FB00230022C3F625
:10160000E073FDF7E9F9FDF733FE0546FDF730FB22
:1016100065A3D3E90023CDE90201FDF78FFB024664
:101620000B4640464946FDF7D5F961A3D3E90023AF
:1016300082468B46DDE90201FDF780FB1F2DCDE9D7
:101640000401504659462BDC6A1E604B53F8223089
:10165000A34225D0DDE90423FDF7BCF902460B4681
:10166000C7E90023814688464A46434650465946C4
:10167000FDF7B0F9DDE90423FDF7ACF9002E0246D1
:101680000B46C7E90223BFF67EAF08F1004301F124
:101690000041C7F800907B60B860F9606D4272E766
:1016A000DDE90423FDF796F988462415C8F30A53AB
:1016B000E31A102B8146C7E90001D5DD34A3D3E935
:1016C0000023DDE90201FDF739FB804689464246E9
:1016D0004B4650465946FDF77DF9CDE90601DDE957
:1016E000062350465946FDF775F942464B46FDF72D
:1016F00071F929A3D3E9002380468946DDE9020177
:10170000FDF71CFB42464B46FDF764F9CDE90401A9
:10171000DDE90423DDE90601FDF75CF98846C8F33D
:101720000A53E41A312C8146C7E9000140F3958041
:1017300021A3D3E90023DDE90201FDF7FFFA80468A
:10174000894642464B46DDE90601FDF743F98246EC
:101750008B4652465B46DDE90601FDF73BF9424602
:101760004B46FDF737F916A3D3E900238046894697
:10177000DDE90201FDF7E2FA42464B46FDF72AF9A0
:10178000CDE904015046594664E700BFAFF300803D
:101790000000601A61B4D03D7370032E8A19A33B18
:1017A00083C8C96D305FE43F00004054FB21F93F1E
:1017B0003163621A61B4D03D0000002E8A19A33B48
:1017C000C14920259A837B3978A10508F8A005082E
:1017D000FDF702F942F2FB13C3F6F9739C4280460F
:1017E00089461AD01EA3D3E90023FDF7F5F80D466C
:1017F00004462B462246C7E9004540464946FDF7C8
:10180000E9F817A3D3E90023FDF7E6F84FF0FF3519
:10181000C7E90201B7E6032495E613A3D3E9002341
:10182000FDF7DAF812A3D3E9002380468946FDF7D5
:10183000D3F80D4604462B462246C7E900454046EC
:101840004946FDF7C7F80AA3D3E90023FDF7C4F81A
:101850004FF0FF35C7E9020195E6DDE906AB03E786
:101860003163621A61B4D03D0000601A61B4D03DAA
:101870007370032E8A19A33B2DE9F84353EC102B08
:1018800000242546C7F6F074C7F6F0751C40AC423C
:101890002DED028BB0EE408AF0EE608A19461046BC
:1018A00000F0AB80002B7FDD1A1500F08980A2F5D7
:1018B0007E7721F07F4323F47003073FD20743F480
:1018C000801366D5C20F4FF0000C02EB43037F106C
:1018D0004200654616204FF400116C18D60F9C424A
:1018E0004FEA420202DC65181B1B8C444908013890
:1018F00006EB4303F1D1202680464FF0004107E07C
:1019000043D0D40F49085200013E04EB43031BD0DF
:10191000AB4208EB0104F3DD04F00049B9F1004FDC
:1019200004EB01082BD0A9469442C5EB0303C4EB9A
:10193000020288BF013B4018D40F49085200013E03
:101940004D4604EB4303E3D11A4327D146084FEA3F
:101950006C0101F17E511CF0010F01F5C00118BFAF
:1019600046F0004601EB0753324643EC182BB0EE2D
:10197000480AF0EE680ABDEC028BBDE8F883B8F1C6
:10198000000FD0DB05F10109CEE79442C4D91D4612
:10199000B7E7C20F02EB4303400093E7431C39D083
:1019A00000F001031818D1E723F000441443DED0FF
:1019B000002B36D11A46C10A153A40050029FAD043
:1019C00011F4801329D149000133CC02FBD5C3F1B6
:1019D0000105C3F1200420FA04F452192143984070
:1019E000A2F57E7721F07F4323F47003073FD207EF
:1019F00043F480133FF566AFCBE751EC100BFDF7D6
:101A00009DF902460B4651EC180BFCF7E5FF41EC43
:101A1000180BACE70CF1010C99E7202401250023F9
:101A2000D9E751EC100B0B46FCF7D4FF02460B46EE
:101A3000FDF7AEFA41EC180B99E700BF000000007B
:101A40002DE9F04F5BEC10AB2DED028BB0EE418A2F
:101A5000F0EE618A2BF00044B4F1795F85B071DA61
:101A600050465946FDF704FC002800F0FD80524620
:101A70005B4650465946FDF761F981A3D3E900233F
:101A800006460F46FDF75AF97FA3D3E90023FCF77A
:101A9000A3FF32463B46FDF751F97DA3D3E900236E
:101AA000FCF798FF32463B46FDF748F97AA3D3E9A5
:101AB0000023FCF791FF32463B46FDF73FF978A340
:101AC000D3E90023FCF786FF32463B46FDF736F9A3
:101AD00075A3D3E90023FCF77FFF32463B46FDF7B1
:101AE0002DF98046894600230022C3F6E073304674
:101AF0003946FDF723F94246CDE900014B46304611
:101B00003946FDF71BF953EC182B04460D46504699
:101B10005946FDF713F902460B4620462946FCF7C5
:101B200059FF02460B46DDE90001FCF753FF0B4667
:101B300000210246C3F6F0710020FCF74BFF41EC98
:101B4000100B83E052465B4650465946FDF7F6F8C7
:101B50004BA3D3E9002306460F46FDF7EFF84AA34F
:101B6000D3E90023FCF738FF32463B46FDF7E6F8A1
:101B700047A3D3E90023FCF72DFF32463B46FDF790
:101B8000DDF845A3D3E90023FCF726FF32463B46A8
:101B9000FDF7D4F842A3D3E90023FCF71BFF32463C
:101BA0003B46FDF7CBF840A3D3E90023FCF714FF35
:101BB0003B463246FDF7C2F843F23233C3F6D373E5
:101BC0009C42804689468EDD0023C3F6E9739C4221
:101BD00041DC0021A4F5001300220020C3F6F071BF
:101BE00014461D46FCF7F6FECDE902010023002253
:101BF000C3F6E07330463946FDF7A0F822462B467F
